:10000000544649531228012800000800000000004F
:10001000000000800100000058919D0400001000C5
:100020000000000000000000400000000000000090
:1000300000000000010000000000000000000000BF
:10004000544643530000100000D501004051CD8AB2
:10005000000001200101100007011000090110003B
:100060000B0110000D0110000F0110001F01100006
:100070001F0110001F0110001F01100011011000CE
:10008000130110001F01100015011000D3361000DD
:10009000CF3710001901100019011000617B110009
:1000A00019011000E7121000ED12100019011000E4
:1000B000190110004333100019011000F312100051
:1000C000E7381000F90210004D1F10001901100050
:1000D0000000000000000000000000000000000020
:1000E0000000000000000000000000000000000010
:1000F0000000000000000000000000000000000000
:1001000000000000000000000000000000000000EF
:1001100000000000000000000000000000000000DF
:1001200000000000000000000000000000000000CF
:1001300000000000000000000000000000000000BF
:1001400000000000000000000000000000000000AF
:1001500000F010F8FEE7FEE7FEE7FEE7FEE7FEE749
:10016000FEE7FEE7FEE7FEE701480047FEE7FEE7A1
:100170001F01100000F002F800F04AF80AA090E811
:10018000000C82448344AAF10107DA4501D100F052
:100190003FF8AFF2090EBAE80F0013F0010F18BFD5
:1001A000FB1A43F0010318478C960100AC9601003E
:1001B0000A4410F8014B14F00F0508BF10F8015B5A
:1001C000240908BF10F8014B6D1E05D010F8013B43
:1001D0006D1E01F8013BF9D1641E03D0641E01F8C5
:1001E000015BFBD19142E4D370470000002300245F
:1001F00000250026103A28BF78C1FBD8520728BF37
:1002000030C148BF0B6070471FB51FBD10B510BD92
:10021000DFF80CD0FFF7F8FF04F07AFC17F0BBFC16
:100220000000012003B4FFF7F1FF03BC17F0BAFC94
:1002300000210028D8BF704700BF491C8842FBDC62
:100240007047704770477047704770477047017834
:10025000002908BF704710F8011F0029FBD1704723
:1002600082B0010F8DF80010C0F303618DF801100A
:10027000C0F303518DF80210C0F303418DF8031051
:10028000C0F303318DF80410C0F303218DF805107D
:10029000C0F303118DF8061000F00F008DF8070071
:1002A00000206A46115C0A2934BF303137311154BD
:1002B000401CC0B2082828BF0020F3D3401CC0B2A5
:1002C0000828FBD302B0704782B001098DF80010F6
:1002D00000F00F008DF8010000206A46115C0A2929
:1002E00034BF303137311154401CC0B2022828BF0E
:1002F0000020F3D3401CC0B20228FBD302B07047E9
:1003000082B0010B8DF80010C0F303218DF80110AD
:10031000C0F303118DF8021000F00F008DF80300F8
:1003200000206A46115C0A2934BF3031373111543C
:10033000401CC0B2042828BF0020F3D3401CC0B228
:100340000428FBD302B0704712484FF6FF710160DA
:1003500070471048104A0021016012681020506157
:100360000E48012203685A6003684022DA6003687D
:100370004FF40C621A6102685161026840F6FF7125
:1003800011620068EA21016305A010F8011F00292D
:10039000FBD1704700700020609011005090110058
:1003A00055415254204F50454E21210D0D00000063
:1003B0000B0ACAB2F849D1F800C0CCF81C0043F4CB
:1003C000FE400B6858610868006840F00103086847
:1003D00003600868C06810F0010FFAD008688068F0
:1003E0000B6840F00100986002F07F024FF400407B
:1003F00040EA022208684261086800680B6840F021
:10040000010018600868C06810F0010FFAD0086891
:1004100080680B6840F001009860086842610868D5
:1004200000680A6840F0010010600868C06810F0B9
:10043000010FFAD0086880680A6840F001009060F7
:1004400008688069C0B2704700F07F0041EA00216F
:10045000D1480268516101680968026841F00101F0
:1004600011600168C96811F0010FFAD0016889684C
:10047000006841F001018160704700F07F014FF496
:10048000004040EA0122C44801684A6101680968E5
:10049000036841F0010119600168C96811F0010F9A
:1004A000FAD001688968036841F001019960016828
:1004B0004A6101680968026841F001011160016840
:1004C000C96811F0010FFAD001688968026841F02B
:1004D0000101916000688069C0B2704710B58C4618
:1004E0000446FFF7CAFF20EA0C01E0B2BDE8104065
:1004F000AAE7704770B5A848002401210268C2F835
:10050000141302686FF0FE21C2F8201302689921CB
:10051000C2F8301300680321C161A048A04DA14E6C
:1005200000684FF0010390F8800190B935F823007E
:10053000C0F307217F20FFF787FFF01890F8C0165F
:1005400015F82300FFF780FF5B1CB3F5A67FEDDBFA
:1005500070BD35F82300C0F3072C644505D0644610
:100560000CF00F017F20FFF76FFFF01890F8C01616
:1005700015F82300FFF768FF5B1CB3F5A67FE8DBE7
:1005800070BD10B504F0CCFA834B84464FF00430B4
:100590001968086219680014486219680120086126
:1005A000196888601968486000217F20FFF74CFFB8
:1005B00040210120FFF748FFBCF1050F18BF10BD17
:1005C00000201968C1F8100310BD734A00B5126805
:1005D0000321D16100284FF000014FF07F0006D0C9
:1005E000FFF732FF032100205DF804EB2CE7FFF753
:1005F0002BFF012100205DF804EB25E7664A00B5DA
:1006000012680321D16100284FF000014FF07F00F4
:1006100006D0FFF719FF012100205DF804EB13E776
:10062000FFF712FF03210020FFF70EFF002108460D
:100630005DF804EB08E7584900B509680320C86174
:1006400000217F20FFF700FF00205DF804EB14E796
:10065000514900B509680320C86100217F20FFF7D8
:10066000F3FE082102205DF804EBEDE64A490A6832
:10067000926C0123096803FA00F010438864704704
:10068000704745490968896D80F001000122801C8E
:1006900002FA00F0084070473F480168496C026860
:1006A00041F4006151640168496C006821F4006103
:1006B00041647047384A012303FA00F000291168A9
:1006C000096C03D0084311680864704721EA0000F0
:1006D000116808647047304900280868C06D0AD066
:1006E0000A6840F00200D0650868C06D096840F0F3
:1006F0001000C86570470A6840F00100D0650868BE
:10070000C06D096840F00800C86570472DE9F043E6
:10071000DFF8849080462025D9F8001009270220B0
:10072000C861002404217F20FFF78EFEA44611E05B
:10073000BCF1030F03D0BCF1060F0BD105E005217E
:100740007F20FFF781FE002404E006217F20FFF7D1
:100750007BFE00240023002D88BF08EB4C1608D92F
:10076000F15C2046FFF770FE601C5B1CC4B29D422A
:10077000F6D80CF1010C6745DAD8D9F80010012041
:10078000C861002404217F20FFF75EFEA446002FED
:100790001CD8BDE8F083000064901100E80600203A
:1007A000000000209C5D0020BCF1030F03D0BCF1D1
:1007B000060F0BD105E005217F20FFF745FE002441
:1007C00004E006217F20FFF73FFE00240023002DD8
:1007D00088BF08EB4C160AD9F01890F82011204673
:1007E000FFF732FE601C5B1CC4B29D42F4D80CF1D2
:1007F000010C6745D8D8CCE770B5D449044603202E
:100800000968C8610425E9B27F20FFF71DFE0023B7
:10081000E1B2D8B2FFF718FE03F12000E1B2C0B296
:10082000FFF712FE03F14000E1B2C0B2FFF70CFE89
:100830005B1C202BECDB0CF0E3F9002808BF002444
:100840006D1C072DDFDB70BDC04803210268D1613C
:1008500002681121C2F8301300684FF00111C0F88E
:10086000201300217F20EFE5B84B00B51968032065
:10087000C86101467F20FFF7E7FD09210320FFF74C
:10088000E3FD01210F20FFF7DFFD19680120C1F80A
:10089000140319689920C1F8300319686FF0FE201D
:1008A000C1F8200303217F20FFF7CEFDFF210020A8
:1008B000FFF7CAFD03210120FFF7C6FD2121052016
:1008C000FFF7C2FD01217F20FFF7BEFD002175204B
:1008D000FFF7BAFD012176205DF804EBB4E59B4BF0
:1008E00000B519680320C86100217F20FFF7ACFD27
:1008F00040210120FFF7A8FD00210320FFF7A4FD00
:1009000002217F20FFF7A0FD15210220FFF79CFDAB
:1009100089210420FFF798FD0F217F20FFF794FD28
:1009200001210320FFF790FD19680120C1F814038D
:1009300019681120C1F8300319684FF00110C1F88F
:10094000200303217F20FFF77FFD01210020FFF717
:100950007BFD00210120FFF777FD21210520FFF716
:1009600073FD04216D20FFF76FFD08216E20FFF756
:100970006BFD10216F20FFF767FD01217F20FFF73E
:1009800063FD08210020FFF75FFD04210120FFF730
:100990005BFD1868406C196840F400604864186892
:1009A000406C196820F40060486400BD2DE9F047F0
:1009B000664E0546012730680024C0F8147304F021
:1009C000AFF86FF0FE294FF0990A4FF003080228A4
:1009D00004D004F0A5F805281DD028E00CF010F98B
:1009E00038B130685A4CC0F820933068C0F830A352
:1009F0001DE03068574CC0F81C8031681120C1F8E8
:100A0000300331684FF00110C1F8200300217F202E
:100A1000FFF71AFD0BE009F084FA78B330684C4C0C
:100A2000C0F820933068C0F830A3FFF71DFF30688E
:100A3000406C316840F4006048643068406C316854
:100A400020F40060486404F06BF8034630684FF00F
:100A50000431016208143168486230680761306807
:100A600087603068476000217F20FFF7EDFC402160
:100A70000120FFF7E9FC052B09D104E0FFE7354C25
:100A8000FFF72DFFD3E731680020C1F8100330686D
:100A9000C0F81C80DFF8C0C001233CF82300C0F37D
:100AA00007217F20FFF7D0FCE95C1CF82300FFF74B
:100AB000CBFC1CB1E118E85C81F8C0065B1CB3F507
:100AC000A67FEADBBDE8F0877047244B00211A4679
:100AD000E0FB03214809C0EB0010800070470020B4
:100AE000704700207047002070470020704708467C
:100AF000704700207047704700207047704770476C
:100B000000207047704770470020704700207047F2
:100B100000207047002070477047704700207047E2
:100B2000704770477047002070470020704770473B
:100B300070477047002070470020704770470020C2
:100B4000704770477047704770470000649011000D
:100B50009C5D0020E2070020000000205BB0055BE8
:100B6000FF4910B509680320C86100217F20FFF705
:100B70006BFC02210020FFF767FC01210220FFF738
:100B800063FC0121BDE810400020FFF75DBCF44983
:100B900010B509680320C86100217F20FFF754FCCD
:100BA00002210020FFF750FC01210220FFF74CFC3E
:100BB0000121BDE810400020FFF746BCE94808B518
:100BC00001684969C1F30721009101684969009AE8
:100BD000C1F307219142F8D0E1480168D1F82C1304
:100BE000006841F00401C0F82C13FFF724FD002831
:100BF00008BF08BD0020BDE80840FFF7FFBCD9488A
:100C000008B501684969C1F3072100910168496984
:100C1000009AC1F307219142F8D0D1480168D1F878
:100C20002C13006841F00401C0F82C13FFF703FDFA
:100C3000002808BF08BD0020BDE80840FFF7DEBC63
:100C400010B503F06DFF052809D0C5480068D0F83D
:100C50002C0310F0040F0CBF0120002010BDC2486F
:100C60000068006810BD70B50546FFF7E9FF012870
:100C700018BF70BD03F054FFB94C0326052827D0D8
:100C8000FFF7BDFF012D18BF70BD2068406C2168C3
:100C900040F40060486400BF00BF00BF2068406CA3
:100CA000216820F4006048642068C66100217F202C
:100CB000FFF7CAFB02210020FFF7C6FB012102203B
:100CC000FFF7C2FBBDE8704001210020FFF7BCBB6D
:100CD0000020FFF793FCD8E710B5FFF752FC012086
:100CE000FFF7C1FF102004F080FA0121052002F077
:100CF0004AFA0121062002F046FA9C490120887038
:100D000010BD10B5602002F094FA602002F084FA61
:100D1000934903200968C86410BD944A014650797C
:100D2000002818BF0120002918BF01215171704708
:100D30008E4A11691061084670478C480021017184
:100D4000C17001898A4816F088BE88480021017167
:100D5000C1700189864816F080BE00B583B00020BE
:100D60008DF80000ADF8040003F0DAFE02281CBF85
:100D700003B000BD0BF044FF02281CBF03B000BD50
:100D8000012077490968C86103217F20FFF75CFBD8
:100D900089210520FFF758FB67210620FFF754FB48
:100DA00045210720FFF750FB23210820FFF74CFBCC
:100DB00003B0F12109205DF804EBFFF745BB2DE9F5
:100DC000F14F88B0002004464FF0100B02900090C5
:100DD00003F0A6FE022806D003F0A2FE052808BFF5
:100DE00009F09FF801E00BF00BFF03F099FE614959
:100DF00005280BD0086890B1012808BF01240ED047
:100E000002280BD0032808BF032408E00868022842
:100E100014BF4FF0360B4FF0000BEBD102245648B5
:100E200056494FF0200900680969406BFF3100F511
:100E3000E03021F0FF01503004FB010512200026B4
:100E4000069001E0032E01D214271AE0F01E0328B9
:100E500038BF152715D3B01F032838BF162710D366
:100E6000A6F10900032838BF24270AD3A6F10C00F5
:100E7000032838BF252704D3A6F10F00032838BF65
:100E800026270298B84209D03548029739090068E8
:100E9000C16107F00F017F20FFF7D6FA0BF0B0FE1B
:100EA00000280CBF4FF07F084FF048080024B9F12C
:100EB000000F35D9380905903148A0FB06104008CD
:100EC000A0EB800000EB060A2E48A0FB06104008AD
:100ED000404200EBC0008119089800EB41100490DB
:100EE000089800EB461003900598012820D0C4F123
:100EF0001F0000EB4A1080B201900122694628468B
:100F000001F0DEF86D1C03F00BFE02284BD050E020
:100F1000202C45F10005E7D3601CC4B24C45F7D343
:100F2000701CC6B2069886428CD309B0BDE8F08F1B
:100F300004EB4A1080B2019001226946284601F074
:100F4000BFF86D1C03F0ECFD022805D10098804528
:100F500002D880384F281BD203F0E2FD052813E0A9
:100F600064901100809011006890110030050020FD
:100F7000D0100020CC050020A4060020A8060020E8
:100F8000ABAAAAAA398EE33804BF0098FF2801D182
:100F9000CDF800B00098C1B2039801550198C0B2D5
:100FA000FFF752FAB8E70098804502D880384F28FA
:100FB00006D203F0B5FD052804BF0098FF2801D133
:100FC000CDF800B0049800992044C9B280F82011EF
:100FD0000198C0B2FFF738FA9EE7F749C86070473A
:100FE00010B503F09DFD052802D0BDE8104006E6CF
:100FF000FFF726FE012818BF10BD0020BDE81040F5
:10100000FFF7FCBA70472DE9F041064682B00C4666
:101010000120FFF728FE03F083FDE84FE64D4FF077
:10102000000824B303F07CFD052815D0FFF7E7FD89
:10103000606800281CBF2168002918D0FFF7B6FCA3
:101040003868C0F82883EE600BF0DAFD02280BD078
:101050000BF086FC40B10AE0FFF7F2FD012804BF67
:101060000020FFF7CBFAE3E7A068FFF7A8FE8DF8B2
:101070000080ADF8048003F053FD02281ED10BF070
:10108000BFFD02281AD139680120C86103217F20E1
:10109000FFF7DAF989210520FFF7D6F96721062045
:1010A000FFF7D2F945210720FFF7CEF923210820C9
:1010B000FFF7CAF9F1210920FFF7C6F985F8048086
:1010C00085F803802989BE4816F0C7FCC5F8108052
:1010D000687900206871602002F0ABF8602002F0AF
:1010E0009BF839680320C86402B0BDE8F081602035
:1010F00002F096B810B5602002F092F8BDE81040FA
:101100000120B0E5AC48C0687047AB4800780028C3
:1011100018BF0120704738B500240094FFF790FDF8
:10112000002818BF38BDA4480471C4700189A448C0
:1011300016F093FCDFF884C2DCF80000406CDCF8A9
:10114000001040F40060486400BFDCF80000406C10
:10115000DCF8001020F4006048649A4D9A48297821
:1011600000290168496914BFC9B2C1F30721009180
:1011700020D001684969009AC9B29142F9D000684B
:101180000221C161DCF80000D0F82C03DCF800106B
:1011900020F00400C1F82C03DCF80000C0F8104374
:1011A000FFF749FA002818BF38BD0120BDE83840D4
:1011B000FFF724BA01684969009AC1F307219142F7
:1011C000F8D0002301684969C9B2009101684969F2
:1011D000009AC9B29142F9D0591CCBB2042BF1D379
:1011E00001212970CBE770B503F09AFC0025724C01
:1011F000052803D02570BDE870408CE7FFF720FD7F
:10120000002818BF70BD2571E57021896C4816F063
:1012100024FC257069480168D1F82C13006821F07E
:101220000401C0F82C13BDE870400120FFF7E6B9B7
:10123000614901200870704770B503F071FC5E4C85
:101240000125052808D0FFF7FBFC002818BF70BD5A
:101250002570BDE870405EE7FFF7F2FC002818BF7C
:1012600070BD00202071E0702189554816F0F5FB13
:101270002570BDE870400120FFF7C0B90120F2E4FD
:1012800070B54D4C0025E57003F04AFC052803D0ED
:101290002570BDE870403EE7FFF7D2FC002818BF7C
:1012A00070BD2571E5702189454816F0D6FB257083
:1012B00042480168D1F82C13006821F00401C0F8FD
:1012C0002C13BDE870400120FFF798B93A4A5169E4
:1012D00050610846704738498861704736488069D0
:1012E0007047354840787047334948707047012847
:1012F00088BF7047354900280868406E04D00968E7
:1013000040F0020048667047096840F001004866F6
:101310007047012888BF70472C4900280868406E34
:1013200004D0096820F0020048667047096820F080
:10133000010048667047002000F0F6BB012000F075
:10134000F3BB10B51C4CE069401CE0611B48016810
:10135000096D006841F004010165FFF79DF9FFF791
:1013600077F9207800281CBF0120FFF77CFC60691A
:10137000002818BF80471648016841F400610160E9
:1013800010BD10B50120FFF76EFCBDE8104000F065
:1013900014BC10487047104870470748006A7047EF
:1013A0000548406A70470448806A70470249002037
:1013B000086248628862704730050020649011001E
:1013C000D0100020AA05002080901100609011002C
:1013D00064050020A4100020AD100020F84900EBA7
:1013E000C00001EBC010704748434FF6FF7101EA9F
:1013F0004000F44908817047F34A107051707047FB
:10140000F149085C7047F0B50746A1B020240121DE
:101410000220FFF74FF9ED4D00216E46286830F8A5
:10142000110026F81100491CA142F7D30021022027
:10143000FFF740F901210020FFF73CF90021002CC3
:1014400009D9286806EB410230F81100491CA2F8BE
:1014500040008C42F5D800210846FFF72BF9A20086
:101460006946384616F058FA21B0F0BD70B50E4600
:10147000D4490500E0B04FF0800008814FF020040F
:101480004FF001010CBF05200420FFF713F9CF49ED
:1014900000206B46096801EB053101EB800202F583
:1014A0008052D2F800C043F820C003EB800CD2F881
:1014B0008020401CCCF88020A042EED3002D4FF0BD
:1014C000000114BF04200520FFF7F4F8E20069468C
:1014D000304616F021FA60B070BD70B50400B9480E
:1014E0000E464FF0010105890CBF05200420FFF7CF
:1014F000E1F8B6482A46006800EB043000F5805158
:10150000304616F009FA4FF0000124B1BDE87040F2
:101510000420FFF7CFB8BDE870400520FFF7CAB838
:1015200010B590B020220021009101910291039109
:101530000491059106910791089109910A910B91E7
:101540000C910D910E91EC460F9100EB410430F897
:101550001130B4F8404223442CF81130491CC9B270
:101560009142F2D35200614616F0D6F910B010BD88
:10157000F0B5944F954EADF2844D00243D89002C7A
:101580004FF001010CBF05200420FFF793F83068ED
:101590002A4600EB043000F58051684616F001FA47
:1015A000002C4FF000010CBF05200420FFF782F84B
:1015B000641C022CE2DB0020FFF7ABFE0120FFF7EA
:1015C000A8FE0DF2844DF0BD814A824900201368C7
:1015D00003EB8003D3F8C03021F81030401C0728FB
:1015E000F5D31068D0F8E40048827047784A7A4B07
:1015F000002818BF00201DD0116801EB8001D1F830
:1016000080110904090C18BF23F81010401C202871
:10161000F2D30020116801EB8001D1F88012090497
:10162000090C1CBF03EB400CACF84010401C2028F8
:10163000F0D37047116801EB8001D1F80011090463
:10164000090C18BF23F81010401C2028F2D30020EA
:10165000116801EB8001D1F800120904090C1CBFCC
:1016600003EB400CACF84010401C2028F0D370472E
:101670002DE9F84304460020009003F051FA0127B9
:10168000504EDFF84C81534D052809D00BF0B8FAC5
:101690000028204650D0FEF7F4FF002859D061E022
:1016A00008F03FFC0228204603D0FEF7EAFF68B3AB
:1016B00035E0FEF7E6FF40B984F001042046FEF76E
:1016C000E0FF002808BFBDE8F8833D492046FFF74A
:1016D00004FF0020D8F8001001EB8001D1F8C01001
:1016E00025F81010401C0728F4D3D8F80000D0F8D3
:1016F000E40068822046FFF779FF2046FFF709FEE5
:10170000377184F00100F070BDE8F88384F00104C3
:101710002046FEF7B6FF002808BFBDE8F883284939
:101720002046FFF7DAFE2046FFF7F3FD377184F01D
:101730000100F070BDE8F883FEF7A3FF0028EED1AA
:1017400084F001042046FEF79CFF0028E7D1BDE8A5
:10175000F88384F001042046FEF793FF002808BFB9
:10176000BDE8F88316492046FFF7B7FE0020D8F8F9
:10177000001001EB8001D1F8C01025F81010401CBA
:101780000728F4D3B1E770B50E4D044668790028F8
:1017900004BFE878FFF76CFF2879002808BF70BD08
:1017A000074AAB6902F5A060A0F18001A0610020AA
:1017B000C4E9021020616061C4E90032012070BDFB
:1017C000D010002030050020360500208890110040
:1017D00064901100D015002050150020E849002029
:1017E000087170472DE9F14F82B00020009012205F
:1017F0004FF020080025019001E0032D01D21426AE
:101800001AE0E81E032838BF152615D3A81F0328A1
:1018100038BF162610D3A5F10900032838BF2426A7
:101820000AD3A5F10C00032838BF252604D3A5F15F
:101830000F00032838BF26260098B04209D0D148AF
:10184000009631090068C16106F00F017F20FEF7A4
:10185000FBFD0024B8F1000F28D902984FEA161BAF
:1018600000EB451AC848A0FB05104008A0EB80001B
:101870004719C648A0FB05104008404200EBC000D5
:101880000299284401EB4019BBF1010F16D0C4F1B5
:101890001F0000EB471080B2FEF7EFFD09EB0401DB
:1018A00081F82001601CC4B24445EDD3681CC5B268
:1018B00001988542A1D303B0BDE8F08F04EB471037
:1018C00080B2FEF7DAFD0AF80400EBE7012070476A
:1018D0007047002070472DE970431C4616460D46A0
:1018E0008046FFF7ADF95FEA00091CBF0120FFF752
:1018F000BAF92819A84288BF01210FD9002344460C
:10190000B34238BF202C06D201FA04F23A4218BF83
:101910005B1C641CF4E76D1C8542EFD3B9F1000F2A
:1019200008BFBDE87083BDE87043A9E42DE9F04726
:10193000994614460E460746089DFFF781F95FEA6F
:1019400000081CBF0120FFF78EF903F047FADFF80B
:1019500040C206EB0903B342CCF8000088BF381937
:1019600013D93C460AE0DCF80010097825F8021B80
:10197000DCF80010491C641CCCF80010844238BF0D
:10198000202CF0D3761C9E42EBD3B8F1000F08BF99
:10199000BDE8F087BDE8F04772E4704710B5FFF787
:1019A000ABF87749488110BD754AC1B200F4706345
:1019B0005289914288BF11464FF0640C01FB0CF133
:1019C000B1FBF2F11A0A02FB0C1189B210F4805F2C
:1019D00012BF08B2484200B270470028B8BF404268
:1019E00080B2B4BF00214FF4805100F47062114303
:1019F000634AC0B25289504341EA1020704708B58B
:101A00000921732000F030F9BDF8001000F01F002C
:101A100021F0FF010843ADF800000D21732000F014
:101A200023F9BDF8001000F01F0021F47F4141EAC6
:101A30000020ADF80000BDF8000008BD7047FFF7BA
:101A400071B854484FF41071006800F5405016F01A
:101A500004B82DE9F84F12204FF0200800900BF049
:101A6000CFF8DFF82CB102280CBF4B484B4800F5EB
:101A700090600024CBF8000001E0032C01DA14266A
:101A80001AE0E01E032838BF152615D3A01F03282F
:101A900038BF162610D3A4F10900032838BF242626
:101AA0000AD3A4F10C00032838BF252604D3A4F1DF
:101AB0000F00032838BF2626B24509D03148310926
:101AC000B2460068C16106F00F017F20FEF7BCFC42
:101AD0000025B8F1000F1EDD31484FEA161980FBD2
:101AE0000410A0EBE070A0EB80000719B9F1010F22
:101AF0000EBF05EB4710C5F11F0000EB4710DBF8E8
:101B00000020C0B212F8011BCBF80020FEF79CFCAD
:101B10006D1C4545EADB0098641C8442ADDBBDE8E2
:101B2000F88F0020FEF7DDBF70B5044601280AD803
:101B30001C48002C0168496E14BF41F0020141F0BD
:101B40000101006841660E4DA869401CA861296921
:101B500000291CBF20468847287800281CBF012088
:101B6000FFF781F80748002C0CBF02210121006813
:101B700001650D48016841F02001016070BD000061
:101B80003005002064901100ABAAAAAA398EE33870
:101B9000E0050020889011009C5D0020E2070020F5
:101BA00056555555609011006405002005490028E0
:101BB00014BF0020012008707047704770477047BD
:101BC000704700005C050020704710B501F017FE5B
:101BD000234B244900224C6824B14A6001F014FED2
:101BE000204610BD1878002818BF0A80F3D1088855
:101BF000B0F57A7F87BF30BF0A80401C0880EAE7D3
:101C000010B501F0FCFD17484468002C08BF30BF38
:101C1000FAD00021416001F0F7FD204610BD70B5FB
:101C200001F0EDFD0F4D6C682CB10020686001F0F3
:101C3000EBFD204670BD30BF01F020FB0028F2D044
:101C400001F020FBA860EEE70020704730BF70472E
:101C500072B662B670477047704772B662B6704728
:101C60003406002060050020EE4BC2081B681A6491
:101C700001F0FC0141EA002040F4704040F0804057
:101C800000687047E74BC2081B681A6401F0FC0249
:101C900042EA002040F4704040F08040890700682C
:101CA000C90EC840C0B27047DF4900200870DD4946
:101CB0000E2009680864DD48007810F0800018BF25
:101CC0000120704710B44FEAD00CD64B1C68C4F802
:101CD00040C001F0FC0141EA002040F4704040F0B7
:101CE000804002601868006C10F4007F04BF10BCD4
:101CF000704700BF1868006C10F4007FF9D110BC69
:101D00007047DFF820C310B4DCF800C0C308CCF87B
:101D1000403001F0FC0343EA002343F4704343F0F6
:101D20008043FF24D3F800C08B07DB0E9C402CEAD5
:101D3000040C9A4010BC42EA0C02C3E7BC484FF4C2
:101D4000F4610268116101684968026841F00201AA
:101D500051600068032181617047B54810B5026881
:101D60001021116002684FF4F46111610168496843
:101D7000026841F00201516000680321816107227D
:101D800008217120FFF7BDFF0E2001F02BFABDE8FE
:101D900010400E2001F033BAA24910B50968A548D9
:101DA0000862072201217020FFF7ABFFA048102135
:101DB0000268116002684FF4F461116101684968BA
:101DC000026841F00201516000680321816107222D
:101DD00008217120FFF795FF0E2001F003FABDE8FE
:101DE00010400E2001F00BBA9148002102681160EA
:101DF00002684FF4E0611161006801218161704760
:101E00008B4900200A6810600A68106109688861BF
:101E100070478748062102681160026802215160FC
:101E20000068816170478248002102681160006883
:101E3000816170477E49002009680860704710B5CD
:101E40007B4C0820216808602168022088610722F5
:101E500008217120FFF755FF2068C06810F0080FB7
:101E6000FAD021680F20886010BD10B504460246E4
:101E70000021F020FFF726FF22460121F020FFF786
:101E800021FF22460021F120FFF71CFF22460121FD
:101E9000F120FFF717FF22460021FC20FFF712FF79
:101EA00022460121BDE81040FC200BE74FF4807171
:101EB00041EAD0025B490B681A645F4A42EA002299
:101EC00010600868006C10F4007F08BF704700BF06
:101ED0000868006C10F4007FF9D17047514A4FF444
:101EE000807141EAD00112681164534941EA00202F
:101EF0000068704708227020002102E7002270204D
:101F00001146FEE647480168496E026821F40071F7
:101F100051660168496E026841F48071516601683A
:101F2000496E026841F4806151660168496E00683B
:101F300021F480614166002270201146E1E63948B3
:101F40000168496E026841F4806151660168496E1A
:101F5000026821F4806151660168496E026821F4CB
:101F6000807151660168496E006841F400714166F4
:101F700070472C480168496E026841F480615166DF
:101F80000168496E006821F4806141667047254808
:101F90001B210268116400680164704710B5244C6D
:101FA0002068C0682549086025484FF6FF71006821
:101FB00001602068C06810F0100F0BD019491B2079
:101FC0000A6810640968086420688068216840F025
:101FD000100088602068C06810F0080F05D02068E5
:101FE0008068216840F0080088602068C06810F0B0
:101FF000040F0AD020688068216840F004008860DF
:10200000FF2200217020FFF77CFE2068C06810F0DE
:10201000010F08BF10BD20688068216840F00100F2
:10202000886010BD609011006C05002000F2004037
:10203000809011002222A26000F00040EC060020F7
:1020400048901100704770B5FF4D0446C0F307413A
:10205000286801F0CEFAC4F30721286801F0C9FA14
:10206000E1B22868BDE8704001F0C3BA2DE9F04143
:10207000F64F0446164638680D46806A396840F0C7
:1020800003008862DFF8C0830321D8F8000001F064
:10209000B0FA2046FFF7D7FF0024002E07D9D8F862
:1020A000000001F0D4FA2855641CA642F7D838681D
:1020B000806A396820F0030088620120BDE8F08161
:1020C00070B514460D46064601F0A3FB224629468C
:1020D0003046BDE87040C9E72DE9F0410024DC4DF1
:1020E000042601F096FB324629462046FFF7BEFF44
:1020F00004242F463D1D264601F08BFB324629461F
:102100002046FFF7B3FF08242D1D042601F081FBB4
:10211000324629462046FFF7A9FF202507F10C0487
:1021200001F077FB324621462846FFF79FFF0C3728
:1021300024243E1D042501F06CFB2A46314620462E
:10214000FFF794FF2824361D01F063FB2A46314631
:102150002046FFF78BFFBF4E07F10C0401F059FB3F
:102160002A4621463046FFF781FF371D25462C1DA4
:10217000042601F04EFB324621463846FFF776FF33
:102180003E1D0424083501F044FB22462946304612
:10219000FFF76CFF4FF4FC342D1D042601F039FBD2
:1021A000324629462046FFF761FF271D2C46251D94
:1021B00001F02FFB324629463846FFF757FFA64F5E
:1021C0002D1D01F026FB324629463846FFF74EFF0B
:1021D0003F1D2D1D01F01DFB324629463846FFF7F5
:1021E00045FF2E1D3F1D042501F013FB2A463146F5
:1021F0003846FFF73BFF351D3F1D042601F009FB64
:10220000324629463846FFF731FF3E1D0425183473
:1022100001F0FFFA2A4621463046FFF727FF8F4E8E
:102220008F4C012501F0F5FA2A4621463046BDE8DB
:10223000F0411BE77047F8B50E0005464FF000046B
:1022400017D0042269462846FFF710FF9DF80000CA
:102250009DF801109DF8032008409DF802101140E0
:102260000840FF2801D00020F8BD641C2D1DB44299
:10227000E7D30120F8BD2DE9F84391460D4680468D
:10228000002401F0C6FA0027B9F1000F88BF6E469E
:1022900019D9042269464046FFF7E8FE0023F05CA6
:1022A000E95C88421CBF601C84B25B1C042BF6D323
:1022B0002D1D7F1C08F104084F45EAD3002C1CBFDC
:1022C0000020BDE8F8830120BDE8F88301207047B5
:1022D00070B55E4C06462068806A216840F00300B5
:1022E0008862594D0521286801F083F9286801F0BA
:1022F000AEF92168896A226821F003019162307089
:10230000012070BD38B5514C2068806A40F003014F
:10231000206881624C4D0521286801F06AF928681F
:1023200001F095F92168896A226821F00301916220
:102330008DF8000010F0010018BF012038BD10B565
:10234000424C2068806A216840F0030088623E4861
:102350000621006801F04DF92068806A216820F0AC
:1023600003008862012010BD70B50546FFF7CAFF63
:1023700000281CBF022070BDFFF7E1FF334C20682E
:10238000806A216840F0030088622F48202100689D
:1023900001F02FF92846FFF756FE2068806A216871
:1023A00020F003008862FFF7ADFF28B100BF00BF37
:1023B000FFF7A8FF0028F9D1012070BD2DE9F84FE3
:1023C0008046032701F025FADFF88090DFF878A037
:1023D000FFF798FF10BBFFF7B2FFD9F80000806A43
:1023E000D9F8001040F0030088622021DAF80000DC
:1023F00001F0FFF84046FFF726FED9F80000806A9A
:10240000D9F8001020F003008862FFF77BFF28B1A5
:1024100000BF00BFFFF776FF0028F9D145464FF413
:1024200080660024042269462846FFF71FFE9DF8B7
:1024300000009DF801109DF8032008409DF802104F
:1024400011400840FF280DE07C90110060901100C1
:10245000F015002068C0010010F8010004300300EE
:102460007005002006D0381EA7F10107B0DC02205D
:10247000BDE8F88F641C2D1DB442D3D30120BDE804
:10248000F88F2DE9F04117460E460446FFF73AFF54
:1024900000281CBF0220BDE8F081FFF750FFDFF8E5
:1024A0000C84D8F80000806AD8F8001040F00300CF
:1024B0008862FF4D0221286801F09BF82046FFF753
:1024C000C2FD0024002F06D9315D286801F091F883
:1024D000641CA742F8D8D8F80000806AD8F8001029
:1024E00020F003008862FFF70DFF28B100BF00BF96
:1024F000FFF708FF0028F9D10120BDE8F0812DE9A0
:10250000F043C1B08846814603276E4601F081F949
:102510004FF4807241464846FFF7B3FF002445461A
:102520004FF4807269464846FFF7A0FD305D295D93
:10253000884205D07F1EE9D241B00220BDE8F08379
:10254000641CB4F5807FF1D341B00120BDE8F08375
:102550002DE9F041D74C0646D44FDFF8548360682C
:10256000C0B00D4650B1D8F8000001F042F86268E2
:10257000FF2AB8BF501C1BDA606035E001F049F952
:10258000FFF7DDFE3868806A396840F00300886232
:102590000221D8F8000001F02CF83046FFF753FD77
:1025A0002946D8F8000001F024F86068401CE3E7F1
:1025B000002060603868806A396820F00300886213
:1025C00000244FF4807269463046FFF74FFD68469D
:1025D0002A5D015D914203D040B00220BDE8F08148
:1025E000641CB4F5807FF3D340B00120BDE8F081D6
:1025F00070B50C46054601F00CF9B4F5807F88BF34
:1026000070BDAA490A68926A096842F003028A62A8
:10261000A7480321006800F0ECFF2846BDE87040A1
:1026200011E5A348006801F012B8A0480168896A62
:10263000006821F003018162704770B50C460546C1
:1026400001F0E7F821462846BDE870404FF480725B
:102650000CE570B5954D04462868806A296840F0FD
:1026600003008862924E9F21306800F0C2FF3068FC
:1026700000F0EDFF2070306800F0E9FF6070306816
:1026800000F0E5FFA0702868806A296820F0030048
:102690008862012070BD70B5044601F0BAF8834D20
:1026A0002868806A296840F003008862804E9F2174
:1026B000306800F09EFF306800F0C9FF207030687D
:1026C00000F0C5FF6070306800F0C1FFA07028689E
:1026D000806A296820F003008862012070BD2DE91E
:1026E000F047DFF8C89104461746D9F8000088463D
:1026F000806AD9F8001040F0030088626C4D032115
:10270000286800F076FF2046FFF79DFC0024B4EB1C
:10271000970F18D2286800F09AFF0646286800F044
:1027200096FF46EA0026286800F091FF46EA004638
:10273000286800F08CFF46EA006048F82400641C1A
:10274000B4EB970FE6D3D9F80000806AD9F80010EF
:1027500020F0030088620120BDE8F08770B51446C0
:102760000D46064601F055F8224629463046BDE89A
:102770007040B4E710B5FFF7C5FD00281CBF02206C
:1027800010BDFFF7DCFD494C2068806A216840F0ED
:102790000300886246486021006800F02AFF206834
:1027A000806A216820F003008862FFF7ABFD28B142
:1027B00000BF00BFFFF7A6FD0028F9D1012010BD22
:1027C00010B501F026F8FFF79DFD00281CBF022080
:1027D00010BDFFF7B4FD354C2068806A216840F0D9
:1027E0000300886232486021006800F002FF206820
:1027F000806A216820F003008862FFF783FD28B11A
:1028000000BF00BFFFF77EFD0028F9D1012010BDF9
:1028100070B50C46054600F0FCFF002600F0F9FFFD
:102820004FF4807221462846FFF720FC761C04F501
:10283000807405F58075102EF0D3012070BD2DE950
:10284000F047C0B08846814600F0E3FF4FF0000A31
:10285000464603276D4600F0DCFF4FF48072314698
:102860004846FFF70EFE00244FF480726946484642
:10287000FFF7FCFB295D305D814205D07F1EEAD267
:1028800040B00220BDE8F087641CB4F5807FF1D32E
:102890000AF1010A08F5807809F58079BAF1100F7C
:1028A000D6D340B00120BDE8F08700006090110051
:1028B0007C901100700500202DE9F04F81B0054695
:1028C000ADF5804D000514468846000DEB4633D02B
:1028D0002F466FF30B07BA465E4600F09AFF4FF0A3
:1028E000000900F096FF4FF4807231463846FFF73A
:1028F000BDFB09F1010906F5807607F58077B9F18E
:10290000100FEED3C5F30B00C0F58056A64288BF6A
:10291000264658443246414614F0FEFF5046FFF723
:102920004DFD022850D059465046FFF788FF022837
:102930004CD03544B044A41BB4F5805F19D34FF498
:1029400080524146584614F0E7FF2846FFF736FD0F
:10295000022839D059462846FFF771FF022835D0A2
:10296000A4F5805405F5805508F58058B4F5805FCE
:10297000E5D21CB3D9462E4600F04BFF002700F0ED
:1029800048FF4FF4807259463046FFF76FFB7F1CBB
:1029900006F580760BF5807B102FF0D3224641465A
:1029A000484614F0B9FF2846FFF708FD02280BD06F
:1029B00049462846FFF743FF022807D0012001B00F
:1029C0000DF5804DBDE8F08F0A20F8E70B20F6E703
:1029D00010B5ADF5806D0446AAB1684614F09CFFB1
:1029E0002046FFF7EBFC022802BF0A200DF5806DA0
:1029F00010BD69462046FFF782FD022802BF0B206A
:102A00000DF5806D10BD01200DF5806D10BD70B508
:102A10000646FFF777FC00281CBF022070BDFFF7B9
:102A20008EFCB44C2068806A216840F00300886204
:102A3000B14D0121286800F0DCFD3146286800F026
:102A4000D8FD2068806A216820F003008862FFF7C3
:102A500059FC28B100BF00BFFFF754FC0028F9D192
:102A6000012070BDF8B500F0D4FEA24D2868806A40
:102A7000296840F0030088629F4E0521306800F00D
:102A8000B8FD306800F0E3FD2968896A2A6821F002
:102A90000301916240F040048DF80040FFF732FCE2
:102AA000002818BFF8BDFFF74AFC2868806A29682B
:102AB00040F0030088620121306800F09AFD214651
:102AC000306800F096FD2868806A296820F00300CD
:102AD0008862FFF717FC002808BFF8BD00BF00BFE1
:102AE000FFF710FC0028F9D1F8BD70B505460024A9
:102AF000FFF708FC40B1AC4201D9002070BD641C56
:102B0000FFF700FC0028F6D1012070BD70B5794CAC
:102B100006462068806A216840F003008862764D8E
:102B20000921286800F065FD286800F090FD216803
:102B3000896A226821F0030191623070012070BD22
:102B400038B5FFF7DFFB002836D1FFF7F8FB694CFB
:102B50002068806A40F0030120688162664D2F2161
:102B6000286800F046FD2068806A216820F0030094
:102B70008862FFF7C7FB28B100BF00BFFFF7C2FBA9
:102B80000028F9D12068806A216840F0030088623B
:102B90000921286800F02DFD286800F058FD216803
:102BA000896A226821F0030191628DF8000010F01B
:102BB000020F1CBF012038BD022038BD4E4810B5A1
:102BC0000421006800F015FD012010BD70B5FFF76D
:102BD00099FB00281CBF022070BD464C2068806A0B
:102BE000216840F003008862434D0521286800F009
:102BF00000FD286800F02BFD06462068806A2168E9
:102C000020F0030088622068806A216840F0030099
:102C10008862FFF794FB0121286800F0EAFC26F0A7
:102C20004001286800F0E5FC2068806A216820F0F7
:102C300003008862012070BD70B50546FFF762FB96
:102C400000281CBF022070BDFFF779FB294C2068CB
:102C5000806A216840F0030088622748522100689A
:102C600000F0C7FC2846FFF7EEF92068806A21686B
:102C700020F003008862FFF745FB28B100BF00BFCA
:102C8000FFF740FB0028F9D1012070BD10B50446C4
:102C9000FFF738FB00281CBF022010BDFFF74FFBD9
:102CA0001548D821006800F0A4FC2046FFF7CBF9B6
:102CB00010480168896A006821F003018162FFF70A
:102CC00021FB28B100BF00BFFFF71CFB0028F9D192
:102CD000012010BD084810B5B921006800F089FC3A
:102CE000012010BD044810B5AB21006800F081FC44
:102CF000012010BD609011007C901100012101FAAB
:102D000000F041490A6810430860404909680860BA
:102D10007047012101FA00F03B490A6822EA0000ED
:102D200008603A490968086070473749096821FA1C
:102D300000F000F001007047334A116821FA00F3F7
:102D400013F0010F4FF0010303FA00F02F4B05D0F1
:102D500021EA00001060196808607047084310609D
:102D600019680860704729490968096821FA00F064
:102D700000F00100704725490A685268012309687C
:102D800003FA00F010434860704720490A6852680F
:102D90000123096803FA00F022EA00004860704746
:102DA0001A490A68126A0123096803FA00F01043FD
:102DB0000862704715490A68126A0123096803FA14
:102DC00000F022EA00000862704710490868406875
:102DD0000A6840F001005060086840680A6840F0E6
:102DE00002005060084A106840F0010010600B6853
:102DF0001860106840F0020010600968086004491B
:102E000000200968C86070477805002058901100BC
:102E10006090110070477047B24810B502683F21BA
:102E2000D1600268002191640068C0F8B4100321E9
:102E30000A2000F0A8F9BDE810400A2000F0C7B948
:102E4000A84A13681860136859604843116888607D
:102E50007047A44A1368186013685960484310F01B
:102E6000010F18BF401C1168886070479D490968B0
:102E7000C1F8B40070479B4918B109680120886403
:102E80007047096800208864704796480168C968DF
:102E9000006841F00201C1607047DFF848C210B419
:102EA000DCF800402062DCF800004162DCF8000041
:102EB0008262DCF80000C362DCF8001001200863C5
:102EC000DCF80000406B10F0010F09D000BF00BF1C
:102ED00000BF00BFDCF80000406B10F0010FF5D11F
:102EE00010F0020018BF4FF0FF3010BC70477D4853
:102EF0000168C968006821F00201C1607047794823
:102F00000168C968006841F00101C1607047754BF4
:102F1000D3F800C0CCF820001868416218688262BB
:102F20001968012008641868406C10F0010F08D07F
:102F300000BF00BF00BF00BF1868406C10F0010F59
:102F4000F6D110F0060018BF4FF0FF30704765480B
:102F50000168C968006821F00101C16070476148DB
:102F60000168C968006841F00401C1607047027CD3
:102F7000017B02F03F0241EA02415A4A1368996517
:102F8000136801685962136841689962136881681F
:102F9000D9621368012119651168496D11F0010F9B
:102FA00008D000BF00BF00BF00BF1168496D11F01D
:102FB000010FF6D11368DB6D83821368DB6D1B0C88
:102FC000C38213681B6E038313681B6E1B0C438341
:102FD00013685B6E83831268526EC2F30E42C28323
:102FE00011F0020018BF4FF0FF3070473D480168F4
:102FF000C968006821F00401C160704701684FEAA8
:10300000314238490B68C3F89C200A684068C2F80E
:10301000A0000868C068096840F02000C8607047D8
:10302000304A136818621068416211680120C1F8C3
:1030300090001068D0F8980010F0010F09D000BF80
:1030400000BF00BF00BF1068D0F8980010F0010F5B
:10305000F5D110F0060018BF4FF0FF30704721483F
:103060000168C968006821F02001C16070471D48EF
:103070000168C968006841F01001C1607047A3F1A0
:10308000050C184B10B41C68C4F888C0D3F800C0F5
:10309000CCF8200018684262186881621968012023
:1030A000C1F880001868D0F8840010F0010F09D032
:1030B00000BF00BF00BF00BF1868D0F8840010F048
:1030C000010FF5D110F0060018BF4FF0FF3010BC13
:1030D000704704480168C968006821F01001C160A8
:1030E000704700006C901100234810B50268012160
:1030F0001166026810215167026841F206015166AB
:1031000002680021916602680A21C2F888100268EC
:103110009021C2F884100168D1F88410026841F04F
:103120000101C2F8841002684FF4817111660068D1
:103130000166032000F04BF80021032000F023F883
:103140000E49022009688862002010BD10B50320D6
:1031500000F048F808484FF4807102681166026870
:1031600000211166006810218167002010BD04490C
:1031700000200870704700005C90110068901100FA
:103180007C050020704700F00303DA004FF0FF0CCD
:103190000CFA02F24FF0050C0CEBC303994000F05F
:1031A0000C03002808DA30480068184443691140CD
:1031B00093431943416170472C4800681844D0F884
:1031C0000033114093431943C0F80013704700F0D7
:1031D0001F01012202FA01F1244A4009126842F853
:1031E0002010704700F01F01012202FA01F11F4A6E
:1031F0004009126802EB8000C0F88010704700F0B0
:103200001F01012202FA01F1184A4009126802EB7B
:103210008000C0F880117047144909680860704741
:1032200012490968C1F880007047104800680068BA
:1032300070470E490968C1F8800170470A48006864
:103240008068704708490A68926809688860104673
:103250007047054A1268926800F1100352F8230083
:1032600042F82310704700004C9011004890110064
:10327000704770477047704770477047002070472D
:103280000020704700207047704770471B4A116844
:10329000106008467047704718484068704710B57E
:1032A00000F0ACF8164804210268C2F888100268E1
:1032B0004FF6FF71C2F88C1072B600684FF40071BF
:1032C000016662B610BD72B60D484FF40031026857
:1032D000116662B60068D0F8040268B14FF6FF715B
:1032E000081A0649074A8860A0F50840B938904294
:1032F0003CBF4FF00110C86000F085B88005002089
:1033000070901100372B1A001A4801684969026849
:1033100041F40071516101680969026821F00601F8
:10332000116101680969006841F01001016170478D
:10333000104801680969026821F0060111610168FD
:103340000969026841F004011161016809690068B6
:1033500041F01001016170470649096888607047B3
:10336000BFF34F8F034904480968C860BFF34F8F0C
:10337000FEE700004C9011000400FA05022824BF6B
:1033800000207047874B53F8202043F82010104648
:10339000704770B5844C2068006F824D10F0010FAB
:1033A00006D021680120C8662868002818BF804719
:1033B0002068006F10F0020F08BF70BD0220216866
:1033C000C8666868002808BF70BDBDE87040004747
:1033D000754810B5026802211165036801221A665A
:1033E00003680322DA66006841650920FFF7EFFEF3
:1033F0000221BDE810400920FFF7C5BE6A4902203E
:10340000096808657047684902200968486570477F
:103410000020704764480168096F11F4007F04D0F0
:1034200000684FF440710166704700684FF4807186
:103430000166704710B55C4C2068C06F10F0020F39
:103440004FF0010018BF0320226850670520B1FB30
:10345000F0F022684FF405710009C2F8801014F0F2
:10346000C5FF524A524B15F011F814F07BFF21684A
:10347000C1F884002068006F10F4007F04D0216838
:103480004FF44070086610BD21684FF480700866E4
:1034900010BD45480168096F11F4807F04D00068B1
:1034A0004FF440710166704700684FF40071016687
:1034B00070473D4B30B41A68D26F12F0010F1DBF38
:1034C0000322D3F800C0CCF874204FF0020C04BFE4
:1034D0001A68C2F874C04FF0020C00EB4005C5EB4F
:1034E000C0104FF49674C1EBC0004C4300EB800059
:1034F000304904EB4010A1FB0010C0080521B0FBCF
:10350000F1F00022B0F5803F05D3511C4008CAB24B
:10351000B0F5803FF9D242EA0C211A6841F010015F
:10352000C2F888101968C1F88C001868006F10F490
:10353000807F05D019684FF44070086630BC704732
:1035400019684FF40070086630BC7047164801686F
:10355000096F11F4003F04D000684FF44031016658
:10356000704700684FF48031016670470E4801686B
:10357000096F11F4803F04D000684FF440310166B8
:10358000704700684FF400310166704706480068D4
:10359000006FC0F30020704703480068006FC0F35D
:1035A0004020704794050020709011007B14AE47B6
:1035B000E17A843FCDCCCCCC30B40025DDE9024C9F
:1035C000056001F00F0141EA8C1101600168D2B27F
:1035D00041EA0221016023F47F4101611021416031
:1035E000416804F0040211436FF3CF11416030BC15
:1035F0007047C26812F0010F18BF8160C16811F0F6
:10360000100FFBD1C16811F0040F08BF704781682B
:10361000C16811F0040FFAD170470023002A0BDDB6
:1036200011F803C0C0F808C0D0F80CC01CF0100F8F
:10363000FAD15B1C9342F3DBC16811F0040F08BFA1
:1036400070478168C16811F0040FFAD17047FF22FA
:10365000C16811F0100FFBD18260C16811F0100F2A
:10366000FBD1C16811F0040FFBD08068C0B2704775
:103670000023002AD8BF704710B4FF24D0F80CC034
:103680001CF0100FFAD18460D0F80CC01CF0100FA1
:10369000FAD1D0F80CC01CF0040FFAD0D0F808C052
:1036A00001F803C05B1C9A42E7DC10BC704741681C
:1036B00041F002016FF3CF1141607047416821F47E
:1036C000C17121F47E41416070470000704702489B
:1036D00000684068704770476090110026490020DC
:1036E0000A6890600968086024494860704710B50E
:1036F000214C216848602168002088600221401E1A
:10370000FFF741FD21680720086010BD1A4900201D
:1037100009680860704719490870704717480078B1
:103720007047164901200870704714488068704738
:103730002DE9F041114C002705466780A0684FF441
:103740007A71B0FBF1F00C4E401E31684860306871
:1037500087600221C81EFFF716FD31680720086048
:103760006188A942FCD330680760BDE8F081044954
:103770004843024988607047449011009C0500202E
:1037800040420F00704770B52C4C05464FF40D5069
:103790002168886621680320C86621682848486631
:1037A00021684CF27100086621682648C1F8800043
:1037B000216842F24630886602210020FFF7E3FCD0
:1037C0000020FFF704FD002D08BF70BD2068806E4B
:1037D00042F2413108432168886670BD174810B530
:1037E00002680121916700684FF40D518166002045
:1037F000FFF7F8FCBDE810400020FFF700BD0F49BF
:1038000001200968486770470C49012009688867EA
:1038100070470A494CF2710009680866704707480A
:1038200081B04CF27101026811660168096F02688B
:10383000D1660068006F009001B07047549011008D
:1038400007383937009C1C9110B500210A20FEF77B
:1038500045FB8B49887110BD024670200121FEF79F
:1038600050BA024670200021FEF74BBA2DE9F04114
:103870000024254672201421FEF7F6F9064610F0C2
:10388000010F18BF012416F0020F18BF44F0020404
:1038900016F0040F18BF44F0040416F0080F0DD002
:1038A000784844F008040168D1F82C13006841F00E
:1038B0000401C0F82C130020FCF7A0FE16F0100F36
:1038C00018BF44F0100416F0200F6D4F06D044F0DE
:1038D000200400210A20FEF701FBB87124B17020FA
:1038E00001212246FEF70DFA300A10F0010F18BF31
:1038F0001025040A14F0010F4FF0010607D045F01F
:1039000020053E7000210A20FEF7E8FAB871200A6F
:1039100010F0010F1CBF45F040057E7025B17020EE
:1039200000212A46FEF7EDF9B8799C281CBF00203B
:10393000B870BDE8F08199E710B500210A20FEF7C4
:10394000CDFAC0B200224E499C2804BFCA700A704A
:1039500008D0C878401CC0B2C870032882BFCA70A3
:10396000012010BD002010BD10B5454C6079401CF1
:10397000C0B26071142818D900210A20FEF7AEFAEF
:10398000A279C0B20021824204BF217161710CD0C2
:103990006079401E60712079401CC0B220710328FC
:1039A00003D921716171012010BD002010BD10B537
:1039B000C9200021FEF758F9002010BD70B574240D
:1039C000002133222046FEF79CF901210D462A46AC
:1039D0002046FEF796F902212A462046FEF791F985
:1039E00003212A462046FEF78CF970200121772218
:1039F000FEF787F90C20FFF7EAFB00210C20FFF708
:103A0000C2FBC82000211422FEF77BF91C4C0020C9
:103A10000146A0700A20FEF761FAA07170BD70B572
:103A2000FFF7A2FF20B10020FFF773F9FEF787FA36
:103A3000134C00252078B0B100210A20FEF74EFA81
:103A4000C0B29C2804BFE57025700CD0E078401C03
:103A5000C0B2E070032806D9E57025700020FFF79A
:103A600058F9FEF76CFA6078002808BF70BD6570E1
:103A70000020FFF74EF9BDE87040FEF760BA000085
:103A8000A80500206490110070B5FE4C00254FF48D
:103A9000906125706570FC4813F0DFFF4FF4906172
:103AA000FA4813F0DAFF4FF49061F94813F0D5FFAC
:103AB0006560A5708021F74813F0CFFFBDE8704026
:103AC0008021F54813F0C9BFEE488078002818BF60
:103AD00001207047EB484078002818BF012070474C
:103AE00070B50546ED48EE490078097800FB01F411
:103AF000FFF7A6F9E64A2B46A2F510610846FFF744
:103B0000CCF962002946E24813F006FFDD490120A6
:103B1000487070BD2DE9F0411D4616460F4680469F
:103B2000069C00F0FDFF022802D109F069F830B1CF
:103B300000F0F6FF052803D106F0F3F900B90224DE
:103B4000FFF768F921462846FFF783F93A463146E0
:103B50004046FFF7DCF9BDE8F041FFF75CB9C94822
:103B600040687047CF4A10B5127801469200C948A4
:103B700013F0D2FEC3490120887010BD2DE9F04F2B
:103B8000DFF800A3002689B09AF801809AF8027045
:103B9000B346FDF7EDFCC4480168496C026841F486
:103BA0000061516400BF0168496C006821F4006144
:103BB0004164BE490220096808660020FDF7ADF89F
:103BC000FDF711FB05F09BFB01280BD06846FDF7C4
:103BD000DAFD0028F6D0684605F0C1FF029870B102
:103BE0001FB10CE04FF0010B69E00146AD480078D1
:103BF0008200A84813F090FE01208AF80200019884
:103C0000002854D0B8F1000F51D104469AF80000B2
:103C1000A8BBDAF8045095B3A04800780790A048F4
:103C200090F8009000F07CFF022802D108F0E8FF35
:103C300030B100F075FF052804D106F072F908B91B
:103C40004FF00209FFF7E6F849460798FFF701F938
:103C500021462A460846FFF75AF9FFF7DCF8DFF855
:103C6000509299F80000022804BF284605F00EFE85
:103C700099F80000092804BF204605F007FE2546F4
:103C8000864887490078097800FB01F4FFF7D8F8E7
:103C90007F4A2B46A2F510610846FFF7FEF8620046
:103CA00029467B4813F038FE01208AF80100FDF711
:103CB00095FD761C042E85D3BBF1000F03D08AF846
:103CC00001808AF802700120FCF7CDFF77480221BD
:103CD0000068016609B05846BDE8F08F69480021C8
:103CE00001704BE738B50F2100F0E6FF654C012865
:103CF00006D100202070FFF741FF009001F05FF82F
:103D0000607800281BBFA07800280020012038BD63
:103D10000F2138B500F0D0FF5A4C012806D1002001
:103D20002070FFF72BFF009001F049F86078002821
:103D30001BBFA07800280020012038BD0021514879
:103D4000417081707047504870475048704770B557
:103D500005464FF490614C4813F07FFE4FF490619C
:103D60004B4813F07AFE474C29464748227800F02A
:103D700038FB22782946BDE87040454800F031BB49
:103D8000F0B4464A404B002114788C4603F5106588
:103D90000022002C13D933F9116030F91170BE42A2
:103DA00053F81160B4BFB61CB61E43F8116033F966
:103DB000116045F81160491C521CA242EBD30CF172
:103DC000010CBCF1020FE3D3F0BC7047002818BF10
:103DD00001202C49487070472DE9F047DFF8A49086
:103DE00082B05FEA00087BD000254FF4107A2C46A1
:103DF00000F096FE052808BF012505D008F000FF59
:103E000000280CBF2B4C2C4C2C482D4F0068796996
:103E1000806BFF3100F5E03021F0FF01503005FBF1
:103E2000010600F07DFE022807D108F0E9FE20B966
:103E30007869FF3020F0FF00064400F071FE022890
:103E400002D108F0DDFEE8B300F06AFE052802D1D9
:103E500006F067F8B0B30025771C304601226946AA
:103E6000FEF72EF97E1C012201A93846FEF728F93B
:103E70000198C1B2009861F31F2000B2414628F8B2
:103E8000150021E0B005002034160020B41A0020EF
:103E9000341F0020B42C0020342D0020BE0500204B
:103EA000BF050020C505002064901100609011003E
:103EB00031060020E20700209C5D0020A4060020BF
:103EC000A806002011E00BE0002C18BF24F8150014
:103ED0006D1C5545C0D30122FD4800F082FAFC4814
:103EE000C9F8040002B0BDE8F087402300208446F2
:103EF000614628F810C0002C18BF24F81010401C90
:103F00009842F5D301224146F24800F06AFAF1489E
:103F1000E6E710B508F074FE02284FF0010207D062
:103F2000ED49EB4800F05DFAEC49E948486010BD06
:103F3000EB49E74800F055FAF6E710B5E74C0028E2
:103F400004BF606010BD01220146E14800F049FA5B
:103F5000DF48606010BDE3487047002818BF0120AB
:103F6000DE4988707047DD49002200284A708A7057
:103F700018BF0120087001E610B54FF44C30142230
:103F8000D949FEF79DF8D84810BD10B54FF44C3014
:103F90001422D549FEF794F8D348006810BD10B537
:103FA0004FF44C301422D049FEF78AF8CE4810BDA9
:103FB0000268B2F1FF3F15D0052904BFC07A7047EF
:103FC00028DC012904BF00797047022904BF007A68
:103FD0007047032904BF407A7047042904BF807AE0
:103FE000704727E0052913D007DC012922D00229D8
:103FF0001CBF032904290BD01CE0142912BF15296A
:104000002D207047162904BF28207047172911D189
:1040100000207047142904BF007B7047152904BF96
:10402000407B7047162904BF807B7047172904BF67
:10403000C07B7047FF20704770B5C0B000244FF4BC
:104040008071684613F009FDFF224FF44C36511C75
:10405000684613F0D8FCFF21254661F307052D22A1
:10406000214662F3070162F30F2128224BF6BB3091
:1040700062F3174164F31F61CDE90005CDE9024108
:1040800004943046FEF722F969463046FEF737FAC7
:1040900040B070BD2DE9F04FC1B00446DDE94A984B
:1040A00092489A4693460D4601602068B0F1FF3F62
:1040B00008BFFFF7C1FFD4E901106BF307006AF3F3
:1040C0000F20266869F31740D4E9037465F30701EC
:1040D00068F31F600D468046FF22511C684613F0AE
:1040E00092FCCDF80880CDE90374CDE900654FF46A
:1040F0004C342046FEF762F969462046FEF7FFF988
:10410000012818BF002041B0BDE8F08F2DE9F04F25
:10411000174688468146C1B000244FF44C30142223
:104120007149FDF7CDFF704B1D68B5F1FF3F02BF30
:10413000204641B0BDE8F08FFF22D3E902A4511C14
:104140006846D3F810B05E6813F05DFC69F30704AD
:1041500068F30F2467F31744012060F31F64CDE96F
:1041600002A4CDE900564FF44C34CDF810B02046EF
:10417000FEF724F969462046FEF7C1F941B0BDE8D3
:10418000F08F2DE9F04F5A4F0025C1B07E42A8466E
:104190004FF44C3014225449FDF792FF524C172132
:1041A00020462368FFF704FF844614212046FFF7CA
:1041B000FFFE4BF6BB3140B28B4204D1BCF1000F85
:1041C0000FD12D280DD02160FF20207100202072FA
:1041D0006072A072E0722D21217361732821A17396
:1041E000E07314212046FFF7E3FE40B2039015214F
:1041F0002046FFF7DDFE40B2029016212046FFF771
:10420000D7FE40B2019016212046FFF7D1FE404272
:1042100040B20090FCF776FF10F0020F70D03548E6
:10422000364A4FF0000990F800C033480078002863
:10423000C8BFACF1010A1EDD0021BAF1000F16DD86
:1042400001F1010B01FB00930BFB009B32F81330D3
:1042500032F81BB0A3EB0B031BB2002BB8BF5B42C1
:104260001BB24345C8BF9846491C5145E8DB09F1DC
:1042700001098145E0DB02994145B8BF45F00205DF
:104280004FF00009CA46BCF1000FC8BFA0F1010BF6
:104290001BDD0021BBF1000F13DD0AFB001332F818
:1042A00013E002EB43035B88AEEB03031BB2002B6E
:1042B000B8BF5B421BB24B45C8BF9946491C594524
:1042C000EBDB0AF1010AE245E3DB0399494518E01B
:1042D000B423002034280020E2070020B00500208D
:1042E0009C5D0020B42C0020B42D0020700500201F
:1042F000F1D8FFFFBF050020BE05002034160020C6
:1043000023E0B8BF45F004054FF0000ABCF1000FF0
:1043100013DD002300280CDD0AFB003132F91110F7
:10432000B942C8BF0F46B142B8BF0E465B1C8342BC
:10433000F2DB0AF1010AE245EBDB0198B84202DB4D
:104340000098B04201DD45F0080509F0FF004090FB
:104350007042C6B2334808F0FF08FFB2056020681B
:10436000B0F1FF3F08BFFFF767FED4E9020A4099AA
:10437000D4E9009B61F3070068F30F2067F317404F
:1043800066F31F600646FF22246965F3070B511C84
:10439000684613F038FBCDF80090CDE903A4CDE9D1
:1043A00001B64FF44C342046FEF708F86946204623
:1043B000FEF7A5F81D208DF8000041208DF80100C2
:1043C00000208DF802508DF804008DF803008DF860
:1043D000050006226946072008F046F841B0BDE80E
:1043E000F08F2DE9F04107460F480E4604780F483C
:1043F000057800F095FB022802D108F001FC78B1A5
:1044000000F08EFB052802D105F08BFD40B104FBC6
:1044100005F0420031463846BDE8F04113F07CBA61
:104420006000F6E770050020BE050020BF050020F3
:104430002DE9FF4FADF2C44D6FF03100CDF8BC0453
:104440000020CDF8B404CDF8B004CDF8B80483460C
:10445000CDF8A0048246CDF8AC04CDF89C04FE480B
:104460004FF0000915460678FC484FF032084F46D9
:104470000078CDF890040220CDF8A894CDF88C04F3
:10448000CDF89494C01ECDF89894CDF88894CDF8CA
:104490008094CDF8A40400F043FB1E246042CDF8C4
:1044A000C004FFF750FCCDF88404DDF8900400232D
:1044B000002840F318810022002E40F3DB8003FB2C
:1044C000062081B2DDF8C40430F91100A04206DDF7
:1044D000DDF8B804401C00B2CDF8B80409E0DDF8FE
:1044E000BCC4604505DADDF8B404401C00B2CDF868
:1044F000B40435F91100A04217DD0BF1010C0FFADD
:104500008CFB4845C8BF8146DDF8A4C46045C8BFE0
:10451000404521DD1FFA83FCCDF880C41FFA82FCE0
:10452000CDF8A404CDF888C416E0DDF8C0C48445F5
:1045300012DD0AF1010C0FFA8CFA8742C8BF074658
:10454000DDF8BCC4604507DADDF8B0C40CF1010C3D
:104550000FFA8CFCCDF8B0C40028B4BFC0F1000C39
:104560008446E04519DADDF8A0C400280CF1010CFE
:104570000FFA8CFCCDF8A0C4ACBF8446C0F1000C8F
:10458000DDF898E4E64508DA0028ACBF8446C0F1BF
:10459000000C0FFA8CFCCDF898C4DDF884C43CF90B
:1045A00011C0C44507DDDDF8A8E40EF1010E0FFAD5
:1045B0008EFECDF8A8E4ACEB0000DFF8A4C200B298
:1045C0003CF811C0ACEB000C2DF811C0DDF8C4C4F0
:1045D0003CF911E0BEF1000F1EDA0028B8BF4042DE
:1045E000DDF884C43CF911C0BCF1000FB8BFCCF1B8
:1045F000000C844510DA1EF11E0F04DADDF8D0C479
:104600000220ACF80000DDF8C40430F811C0DDF879
:10461000C80420F811C004E0DDF8C8C400202CF85C
:1046200011003DF91100A04205DDDDF8AC14491C74
:1046300009B2CDF8AC140028B4BF41420146884508
:1046400013DADDF89C14491C09B2CDF89C1400283B
:10465000ACBF01464142DDF894C48C4505DA002820
:10466000B8BF404200B2CDF89404501C02B2B2422E
:10467000FFF625AF581C03B2DDF890048342FFF625
:104680001AAFBAF10A0F03DBDDF8D004072101806D
:10469000D345B8BFB9F1960F0DDA07F19500B0F523
:1046A000957F08D8002FB4BF784238464845C8BF28
:1046B0004FF0000B19DCD345B8BFB9F1500F0FDA3A
:1046C00007F14F009E280BD866494878401CC0B2BD
:1046D0004870C8283DD9C82048700020087038E0CC
:1046E000002FB8BF7F424F4533DCDDF8B80401210D
:1046F00038B1BBF1000F10D05A48007801282DD0F6
:1047000048E0DDF8B40400280BDC56494878401C2A
:10471000C0B24870C8281CD9DDE7DDF8B004002815
:1047200010DD50480022427001704FF490624C48F6
:10473000DDF8841413F0F0F80DF2D44D4FF0FF3093
:10474000BDE8F08F47494878401CC0B24870C8287F
:10475000C1D800200DF2D44DBDE8F08FDDF8A014D3
:10476000DDF89C04884215DADDF89814DDF894042D
:1047700088420FDA32466946DDF89034DDF8C40429
:1047800005F0B5FFDDF8AC04002804BF0DF2D44DF0
:10479000BDE8F08F4FF00008DDF8A404A6F1010990
:1047A0001FFA89F700287DDDBAF10F0FDCBFDDF8B5
:1047B000A8040F2876DDDDF88C14DDF8800488422B
:1047C00070D3DDF89014DDF88C04091ADDF880044C
:1047D000814267DDDDF88C14DDF88804884261D3FE
:1047E000DDF88804711A88425CDADDF8801401FB78
:1047F000060E35F91E3003EBD370B3F1FF3F4FEADD
:104800006000B8BF404202B201FB06F01FFA80FC14
:10481000DDF8880400B28346012841DB0CEB00017F
:1048200089B2002B20DD35F911A005EB410131F9EA
:10483000021CBAEB010A06D50029B4BFC1F1000A77
:104840008A46924504DB0029B8BF4942A14223DAD7
:10485000401E1FFA80F823E0BE050020BF0500209F
:10486000B42E0020B805002016DA35F911A005EBAA
:10487000410131F9021CAAEB010ABAF1000F06DD71
:104880000029B4BFC1F1000A8A469245E0DB002945
:10489000B8BF4942A142DBDB401E00B20128BDDAAD
:1048A000CB4500E074E036DA0CEB0B0080B2002B55
:1048B00016DD35F9101005EB4000B0F90200091AB9
:1048C00005D50028B4BF41420146914204DB0028CF
:1048D000B8BF4042A04218DA0BF1010087B21AE0DB
:1048E00013DA35F9101005EB4000B0F90200091A8F
:1048F000002905DD0028B4BF414201469142EBDBAF
:104900000028B8BF4042A042E6DB0BF101000FFADD
:1049100080FBCB45C8DBDDF88004DDF8843400FB88
:10492000068082B2DDF8800433F9123000FB067095
:1049300035F812201FFA80FC9A1ADDF8840414B2AC
:104940001FFA8EF1DDF8842430F9110035F81110CA
:1049500032F91C2035F81CC0411A09B2A2EB0C0C2C
:104960000FFA8CFC0D1B48BF651AB1EB0C0448BF55
:10497000ACEB010429190FFA81FCC11A48BF191ABE
:10498000831A48BF131AC81800B28445FFF6E1AE77
:104990000120DFE62DE9F05FDFF864A18046002604
:1049A000DAF80000374690F8241100291CBFB0F84F
:1049B000300100286CD0FCF791FCDAF8001091F877
:1049C0002411B0FBF1F201FB1200002860D101F0CC
:1049D00071FC5FEA00095BD04A480078102804BFE8
:1049E000484604F053FF48484FF0000C444690F806
:1049F00000B04648634690F800E0BEF1000F19DDB4
:104A000034F9020B0125BBF1010F10DD34F9022B43
:104A1000101A01B20029B8BF494208B2604502DD50
:104A200084461E462F466D1C10465D45EEDB5B1C22
:104A30007345E5DBDAF80020B2F83001844527DB66
:104A400006FB0B7008EB400338F8101033F8023CFB
:104A5000C91A39F8103009EB400009B230F8020CDD
:104A6000181A081A00B20028B4BF434203460029AE
:104A7000B8BF49428B420BDA0028B8BF4042B2F8B7
:104A80003211884204DA01F01FFC0020BDE8F09FDB
:104A90000120BDE8F09F70B515460E46044608F0AB
:104AA000AFF8002C18BF70BD042818BF052806D029
:104AB0001348006890F82400A84288BF70BD3046B3
:104AC000BDE87040FFF74EB870B51546044608F0D3
:104AD00097F8B4F1FF3F0AD0002C18BF70BD002D2D
:104AE00008BF70BD2846BDE87040FEF7F9BF002D35
:104AF00008BF70BD2846BDE87040FFF728B9000028
:104B0000E806002031060020BE050020BF05002079
:104B100010B506F0E9FA06F083FB002010BD000096
:104B2000AB4800787047AA480078022805D00528CD
:104B30001CBF0020704705F0F4B908F061B8A44923
:104B40000870704710B50446072C28BF10BDDFE879
:104B500004F013040810130C0800084600F040F994
:104B60000AE0084608F041F806E0084605F0CEF9EC
:104B700002E0084607F0E8FC9548047010BD95492E
:104B800000200968B1F8641011F4807F08BF7047F5
:104B9000FDF71BB88F4900200968B1F8641011F4C3
:104BA000807F08BF7047FDF72BB88A49002009684D
:104BB000B1F8641011F4806F08BF7047FDF744B876
:104BC0008349487800281CBF401E4870704710B5C4
:104BD00072B6FEF703FEBDE81040FEF7C1BB10B58C
:104BE0007D48FDF773FB72B6FEF7F8FDBDE8104097
:104BF000FEF7B6BB7648006970477548C0687047D5
:104C000073494861704772484069704710B5FCF7B6
:104C1000E7F9FBF76FFCFCF774F8FFF77AF9BDE8EA
:104C20001040FCF716BF10B5FCF7DAF9FBF762FC91
:104C3000FBF71AFEFCF765F8BDE81040FCF709BF6A
:104C400030B5ADF2844D05464FF49061684612F0E0
:104C500004FF5F4C2846256106F062F9E060F0B180
:104C60000278A2704178E17083782371531C03F0BD
:104C7000FE0363710023E37123724FF0120C84F87A
:104C800006C004F10A0C8CF800308CF80130007872
:104C900060721046FCF7A8FB0DF2844D30BD4D4804
:104CA0000068B0F8640010F4807F18BFFCF7A8FF1C
:104CB00000200DF2844D30BDF0B5ADF2CC4D0F4665
:104CC00004464FF49061684612F0C7FE404D2046FE
:104CD0002C6106F025F9E860002851D00278AA700E
:104CE00041780446E97080782871501C00F0FE007D
:104CF00068710020E87128721223AB7105F10A0374
:104D000018705870207868721046FCF76DFB0DF52E
:104D10009061204606F021F9608A6E6900281CBF68
:104D20007043060B002017F0040F18BF062017F081
:104D3000080F18BF40F00200616A0840DDF88014D7
:104D4000CDF8C014DDF89C14CDF8C414DDF890142F
:104D5000CDF8C8140DF59861FCF755F9DDF88C0411
:104D600020B13346EA78A97805F0CAFB64213046C1
:104D700005F079FC287802280FD0052810D017E01C
:104D800014480068B0F8640010F4807F18BFFCF786
:104D900037FF00200DF2CC4DF0BD07F031FF01E0F0
:104DA00005F0BFF8022804BFDDF89404FFF714F8FB
:104DB000002001F07EFA0DF2CC4D0120F0BD10B5BF
:104DC000FCF798F902490020C860012010BD0000DE
:104DD000BC050020E806002000FE1100F9487047DD
:104DE000F94948707047F84840787047F74810B460
:104DF000F74A0168914218D14168B1F5887F14D80B
:104E00000022D0F808C003461146B2EB9C0F24BF25
:104E100010BC704753F82140491C2244B1EB9C0F51
:104E2000F8D3002A04BF10BC7047002010BC7047A4
:104E30004FF4FC30FDF7C2BA2DE9F0410446E348D7
:104E40000E46E34F0168B94213D14168B1F5887F3E
:104E50000FD80023D0F808C001461A46B3EB9C0FC8
:104E600008D251F82250521C2B44B2EB9C0FF8D3BD
:104E700003B10020002558B1B0E80E10A4E80E10D0
:104E8000B0E80E10A4E80E100FC884E80F0016E07A
:104E9000FF223021204612F0B6FD4FF48870C4E99D
:104EA00000703020C4E90205AA20C4E904054FF0CF
:104EB000FF30E062A062A5616062C4E9075066B994
:104EC0004FF4FC30FDF77AFAC24805604560856012
:104ED000C560056145618561C5610120BDE8F0815E
:104EE000B949012048707047B749002008707047E1
:104EF00070B5ADF5107D0446FFF77FFE054614F052
:104F0000020F04BF0DF5107D70BD0426FFF70BFEE8
:104F1000002818BFB04C08D095F92C102246304616
:104F200006F040F80DF5107D70BD6C462046FCF78C
:104F300059FCF1E770B50D4606461024FFF75DFEFB
:104F400016F0020F18BF05242A46102C28BF70BD8A
:104F5000002A08BF70BD204490F928102046BDE803
:104F6000704006F01FB82DE9F04F87B0814612203F
:104F700000244FF0200A27460090FFF7D1FD0228B9
:104F800002D107F03DFE30B1FFF7CAFD052804D17C
:104F900004F0C7FF08B902200090009800250028FF
:104FA0009CBF07B0BDE8F08F0026BAF1000F7CD996
:104FB0008A4A681EA2FB00314908A1EB810108441E
:104FC0000590E81E0490A81F0390C01E0290C01E0A
:104FD0000190A2FB05104008A0EB8000A5F10F0B8B
:104FE00000EB0508FFF79CFD022803D107F008FE3F
:104FF00000283AD0FFF794FD052803D104F091FF73
:10500000002832D0032D38BF142417D30498032866
:1050100038BF152412D30398032838BF16240DD3A4
:105020000298032838BF242408D30198032838BFE6
:10503000252403D3BBF1030F38BF2624A7420AD08F
:105040006748C4F3031127460068C16104F00F01EB
:105050007F20FBF7F9F9C4F3031001281CBFC6F148
:105060001F0000EB481018D127E0002D0CBF1424BE
:105070002424A74209D05A48210927460068C16163
:1050800004F00F017F20FBF7DFF92009012814D07D
:105090000598C6F11F0101EB401019F8011BC0B2C1
:1050A000FBF7D2F9761C56459CD300986D1C8542BF
:1050B000FFF47AAF07B0BDE8F08F06EB4810ECE7DD
:1050C0002DE9F84F834640484FF0000A0C46B0F9EE
:1050D00004804FF01209202750460091FCF77EF91A
:1050E0000546CBF10706FFF71BFD022802D107F0AA
:1050F00087FD30B1FFF714FD052804D104F011FF3E
:1051000008B94FF00209BBF1000F1CD0002E55DB8F
:105110004FF0000CB9F1000F49D9012101FA06F353
:10512000701E01FA00FB0021002F3CD935F8020B5C
:105130002278A0EB080000B25FEAD21E23D000283C
:1051400027DA2EBB1BE00023B9F1000F2FD9002175
:10515000002F10D935F8022B2078A2EB080212B2EA
:10516000502AC8BF40F0800040F04000491C04F8BD
:10517000010BB942EED35B1C4B45E8D317E010F1AD
:10518000280F05DB0AE0002803DD0EB9282805DD1D
:105190009A43002EC4BF4BEA0200C2B204F8012BAE
:1051A000491CB942C2D30CF1010CCC45BBD30098C9
:1051B000FFF7D9FE002E08BF4FF0010A5046BDE8A8
:1051C000F88F000034330020D405002000F81100CF
:1051D000544352461416002074350020ABAAAAAAE4
:1051E00064901100FD498880704770B5FB4EFC4902
:1051F000F08009680320C8610425E9B27F20FBF72D
:1052000023F90024B179E0B2FBF71EF904F1200084
:10521000B179C0B2FBF718F904F14000B179C0B21E
:10522000FBF712F9641C202CECDB6D1C072DE4DB72
:1052300070BD2DE9F04F89B00026FBF7D1FEE8499B
:10524000072009680865E748016841F0200101600E
:105250000020FFF7CAFFE1494FF4006088804FF457
:105260001071E14812F0F9FB0020FBF756FDFBF747
:10527000E3FF00252C460795FFF755FC04F03FF8A7
:1052800001281DD06846FCF77EFAB8B10120FBF773
:1052900044FD684604F063FC6D1C012D0ED0002512
:1052A000D1492046FFF70CFF072C1ED00020FBF74A
:1052B00034FDFCF793FAFBF7BFFF641C002EDDD032
:1052C000FFF731FCC54AC948C74BD0600020D16800
:1052D00013F800C0401C01F801CBD160B0F5107F7D
:1052E000F5D3079800283CD135E012200890BB4840
:1052F00000274FF0200BB0F904603846FCF76EF839
:105300000546BA460024BBF1000F18D9304613F009
:1053100056F8B74AB74B13F0B9F88946804635F9C5
:10532000022B901B48BFB01A13F049F842464B4677
:1053300013F0AAF938BF7F1C641C5C45EFD30898B2
:105340000AF1010A8245DDD3002F4FF001061CBF90
:1053500001200790B4E7002E1EBF002009B0BDE871
:10536000F08F012009B0BDE8F08FF0B587B00026BE
:105370000120FBF778FC9B48016841F020010160A7
:105380000020FFF732FF95494FF4006088809A496A
:105390000020C1F88000C1F88400C1F88800C1F87D
:1053A0008C00C1F89000C1F89400C1F89800C1F8D1
:1053B0009C00C1F8A000C1F8A400C1F8A800C1F881
:1053C000AC00C1F8B000C1F8B400C1F8B800C1F831
:1053D000BC00FBF7A2FCFBF72FFF00252C462F4655
:1053E00003F08DFF012835D06846FCF7CCF978B37F
:1053F0000120FBF792FC6D1C012D24D000257F4974
:105400002046FFF75DFE072C06D00020FBF785FC49
:10541000FBF712FF641C1BE0002420252046FBF74D
:10542000DDFF002130F9022BA2F26662B2F54D7F5A
:1054300088BF641C491CB1EB450FF3D3002C08BF97
:1054400001260DD106E00020FBF767FCFBF7F4FE18
:10545000002EC5D027B9002E1EBF002007B0F0BD1A
:10546000012007B0F0BD2DE9F04F82460021ADF5D7
:10547000137D634890910C4600780F460D46022834
:1054800008BF022703D0052804BF02240427DFF841
:105490005091DFF870B100F09AB9204605F040FD58
:1054A000002800F09381008900EA0A0626F0CC006B
:1054B00030F47C4000F08A81DFF84C81D8F800009D
:1054C0004069D8F8001040F400704861D8F8000036
:1054D0000069D8F8001020F006000861D8F8000034
:1054E0000069D8F8001040F0100008613CB1012CB0
:1054F00035D0022C71D0032C55D000F0FBB802211E
:105500000846FFF71FFB0120FBF7ADFB05F06DFB25
:105510000F212046FFF7D0FB002800F05781D9F873
:105520000000406CD9F8001040F40060486400BFEF
:1055300000BF00BFD9F80000406CD9F8001020F47B
:1055400000604864FBF723FB05F03BFB012007F0FC
:1055500011FC0020FBF7E1FBFCF740F9CAE0002159
:105560000220FFF7EFFA0120FBF77DFB0F21204619
:10557000FFF7A2FB002800F02981D9F80000406C59
:10558000D9F8001040F40060486400BF00BF00BFBD
:10559000D9F80000406CD9F8001020F4006048648D
:1055A000FBF7F5FAA6E000210520FFF7CBFAFBF7A1
:1055B00017FDD8F800000069D8F8001020F00600A8
:1055C0000861D8F800000069D8F8001040F0040025
:1055D0000861D8F80000006918E03EE0D40500201A
:1055E00064901100640500207435002034330020DD
:1055F0009A9999999999B93F34370020B437002086
:1056000029060020689011004C901100D8F8001075
:1056100040F01000086109F024FC0F210220FFF780
:105620004BFB00287ED0DBF8001007208860DBF8F9
:1056300000100420486002212020FBF7D5FE002046
:10564000FBF76BFBFBF7CFFDDBF800000068DBF836
:10565000001040F0010008604CE002210520FFF737
:1056600071FAFBF7BDFCD8F800000069D8F800100B
:1056700020F006000861D8F800000069D8F8001092
:1056800040F004000861D8F800000069D8F8001064
:1056900040F01000086109F0E4FB05F092FA0F21D8
:1056A0000320FFF709FB00283CD0DBF800107F2027
:1056B0008860DBF8001002204860D9F80000406CD8
:1056C000D9F8001040F400604864012007F04BF95D
:1056D000D9F80000406CD9F8001020F4006048644C
:1056E000FBF781FDDBF800000068DBF8001040F0FC
:1056F000010008609098002864D116F0010F23D0B3
:105700000120FBF7B0FAFFF70EFA88B1FBF730FF84
:10571000FF210F20FFF78DFD012121EA0000054345
:10572000002000E052E0FBF7F8FA909890BB0BE005
:10573000FBF71EFFFF210F20FFF717FE012121EAD3
:10574000000045EA4005EBE716F0060F22D0FFF710
:10575000EAF902281ED1FEF797F90020FEF703FCB4
:105760000120FBF780FAFEF7EEFA0646FFF745FA4E
:105770000523320004D090F92D10184605F012FCD4
:10578000FEF7E1FAFEF7D9FBFEF7DDFA4FF4906180
:1057900012F041F9FFF731FA804604209190FFF7AB
:1057A000C2F9002818BFFE4E1FD098F92C103246BF
:1057B000919805F0F7FBFB4900200870FA49087042
:1057C000FBF711FDFFF7ACF9FFF7F9FA641CBC42D7
:1057D00003D2909800283FF460AEF449002008708E
:1057E0000DF5137D2846BDE8F08F6E463046FBF779
:1057F000F9FFDAE770B5ED48CCB04578FFF790F9DE
:1058000001287DD1EA480068B0F93610B0F93400BB
:1058100004F09CFF15F0020F73D0002140A8FFF7A1
:105820000BFB4598401C459040F27770FFF71BFE3C
:10583000C0B2032810D0002804BF45F250004490A5
:1058400012D0012808BF4AF250100CD0022808BF1D
:1058500045F2A10007D007E04AF2A1104490469813
:10586000401C469008E0449047980022401C479016
:105870002121072006F0CFFD40AC05F042FB40B1EE
:1058800081694891C169499141694A91C0684B90C9
:1058900005E04FF0FF304B904A9049904890C54842
:1058A00040904FF488704190302042900020439007
:1058B000A3682246014652F820C0401C6144B0EB68
:1058C000930FF8D34E42FF22511C6846E66012F057
:1058D0009AF8A268F4E804018DE847000FCC04AE02
:1058E00086E80F0094E80F0008AE203C86E80F0021
:1058F0004FF4FC306946FCF702FEAF49226801E034
:1059000022E00DE00A6062684A6022698A6062698A
:10591000CA60A2690A61E2694A61226A8A610CE08E
:1059200015F0010F09D040F22220FFF79CFD20B9AD
:1059300000222121072006F06EFDFEF7FFF92A461E
:105940004021072006F067FD4CB0BDE8704003F031
:10595000D2BC70B50C469949054603200968C86158
:1059600001217F20FAF770FD00217520FAF76CFD08
:1059700001217620FAF768FD60210820FAF764FD1E
:1059800000210920FAF760FD30210A20FAF75CFDBA
:1059900000210B20FAF758FD06210E20FAF754FDDE
:1059A000E1B22620FAF750FDE1B22720FAF74CFDCC
:1059B000E1B22820FAF748FDE1B22920FAF744FDC8
:1059C000E1B22A20FAF740FDE1B23020FAF73CFDBF
:1059D000E1B23120FAF738FDE1B23220FAF734FDB6
:1059E000E1B23320FAF730FDE1B23420FAF72CFDB2
:1059F000E1B23620FAF728FDE1B23720FAF724FDAC
:105A0000E1B23820FAF720FDE1B23920FAF71CFDA7
:105A1000E1B23A20FAF718FDE1B24020FAF714FD9E
:105A2000E1B24120FAF710FDE1B24220FAF70CFD95
:105A3000E1B24320FAF708FDE1B24420FAF704FD91
:105A4000E1B24620FAF700FDE1B24720FAF7FCFC8C
:105A5000E1B24820FAF7F8FCE1B24920FAF7F4FC89
:105A6000E1B24A20FAF7F0FCE1B25020FAF7ECFC80
:105A7000E1B25120FAF7E8FCE1B25220FAF7E4FC77
:105A8000E1B25320FAF7E0FCE1B25420FAF7DCFC73
:105A9000E1B25620FAF7D8FCE1B25720FAF7D4FC6D
:105AA000E1B25820FAF7D0FCE1B25920FAF7CCFC69
:105AB000E1B25A20FAF7C8FCE1B26020FAF7C4FC60
:105AC000E1B26120FAF7C0FCE1B26220FAF7BCFC57
:105AD000E1B26320FAF7B8FCE1B26420FAF7B4FC53
:105AE000E1B26620FAF7B0FCE1B26720FAF7ACFC4D
:105AF000E1B26820FAF7A8FCE1B26920FAF7A4FC49
:105B0000E1B26A20FAF7A0FC02217F20FAF79CFCA0
:105B10006A210220FAF798FC8E210420FAF794FCFF
:105B2000F1210720FAF790FC15B1012D05D008E00E
:105B300004210620FAF788FC03E008210620FAF782
:105B400083FC03217F20FAF77FFC21211020FAF744
:105B50007BFC00211120FAF777FC00211220FAF7D4
:105B600073FC00211320FAF76FFC00211420FAF7D0
:105B70006BFC00211520FAF767FC01211620FAF7CB
:105B800063FC02211720FAF75FFC00211820FAF7C6
:105B90005BFC00211920FAF757FC00211A200FE0C6
:105BA000743500201607002017070020D4050020B8
:105BB000E806002054435246141600206490110059
:105BC000FAF742FC00211B20FAF73EFC01212020BD
:105BD000FAF73AFC20212120FAF736FC0021222096
:105BE000FAF732FC00212320FAF72EFC00212420B2
:105BF000FAF72AFC00212520FAF726FC01212620AD
:105C0000FAF722FC00212720FAF71EFC02212820A7
:105C1000FAF71AFC00212920FAF716FC00212A20A5
:105C2000FAF712FC00212B20FAF70EFC012130209C
:105C3000FAF70AFC00213120FAF706FC2021322075
:105C4000FAF702FC00213320FAF7FEFB0021342092
:105C5000FAF7FAFB00213520FAF7F6FB012136208E
:105C6000FAF7F2FB00213720FAF7EEFB002138208B
:105C7000FAF7EAFB02213920FAF7E6FB00213A2085
:105C8000FAF7E2FB00213B20FAF7DEFB012140207E
:105C9000FAF7DAFB00214120FAF7D6FB0021422077
:105CA000FAF7D2FB20214320FAF7CEFB0021442053
:105CB000FAF7CAFB00214520FAF7C6FB012146206E
:105CC000FAF7C2FB00214720FAF7BEFB002148206B
:105CD000FAF7BAFB00214920FAF7B6FB02214A2065
:105CE000FAF7B2FB00214B20FAF7AEFB012150205E
:105CF000FAF7AAFB00215120FAF7A6FB0021522057
:105D0000FAF7A2FB00215320FAF79EFB2021542032
:105D1000FAF79AFBBDE8704000215520FAF794BBD2
:105D200010B50322FD49062828BF10BDDFE800F0AA
:105D30000327FDFCFBFA0868C26101217F20FAF706
:105D400083FBAF210820FAF77FFB73210A20FAF7C3
:105D50007BFB0A210E20FAF777FB02217F20FAF75E
:105D600073FB00210720FAF76FFB1F210120FAF7D0
:105D70006BFB1021BDE810400620FAF765BB0868F0
:105D8000C26101217F20FAF75FFB0F210E20FAF795
:105D90005BFB87210820FAF757FB6E210A20FAF7F0
:105DA00053FB02217F20FAF74FFB71210720FAF7FE
:105DB0004BFB6A210220FAF747FB8E210420FAF7F9
:105DC00043FB03217F20FAF73FFB61211020FAF704
:105DD0003BFB00211120FAF737FB00211220FAF7D4
:105DE00033FB00211320FAF72FFB00211420FAF7D0
:105DF0002BFB00211520FAF727FB01211620FAF7CB
:105E000023FB06211720FAF71FFB00211820FAF7C1
:105E10001BFB00211920FAF717FB00211A20FAF7C3
:105E200013FB00211B20FAF70FFB01212020FAF7BA
:105E30000BFB60212120FAF707FB00212220FAF753
:105E400003FB00212320FAF7FFFA00212420FAF7B0
:105E5000FBFA00212520FAF7F7FA01212620FAF7AC
:105E6000F3FA00212720FAF7EFFA06212820FAF7A3
:105E7000EBFA00212920FAF7E7FA00212A20FAF7A5
:105E8000E3FA00212B20FAF7DFFA01213020FAF79C
:105E9000DBFA00213120FAF7D7FA60213220FAF735
:105EA000D3FA00213320FAF7CFFA00213420FAF791
:105EB000CBFA00213520FAF7C7FA01213620FAF78C
:105EC000C3FA00213720FAF7BFFA00213820FAF789
:105ED000BBFA06213920FAF7B7FA00213A20FAF77F
:105EE000B3FA00213B20FAF7AFFA01214020FAF77C
:105EF000ABFA00214120FAF7A7FA00214220FAF775
:105F0000A3FA60214320FAF79FFA00214420FAF710
:105F10009BFA00214520FAF797FA01214620FAF76B
:105F200093FA03E03FE039E033E02DE00021472021
:105F3000FAF78AFA00214820FAF786FA0021492068
:105F4000FAF782FA06214A20FAF77EFA00214B205E
:105F5000FAF77AFA01215020FAF776FA0021512057
:105F6000FAF772FA00215220FAF76EFA0021532054
:105F7000FAF76AFA60215420FAF766FA0021BDE8C0
:105F800010405520FAF760BAAA21BDE81040002061
:105F9000DFE45521BDE810400020DAE4AA21BDE885
:105FA00010400120D5E45521BDE810400120D0E487
:105FB00010B5FDF7C8FE0446FDF7C7FE2146BDE853
:105FC00010404FF4906211F0A7BC2DE9F041544805
:105FD000047854480578FDF7B8FE0646FDF7B3FE91
:105FE0000022002D98BFBDE8F0810021002C10D9BF
:105FF00002FB04FC06EB4C0300EB4C0C11F0010F10
:106000001CBF33F811702CF81170491CC9B2A142A1
:10601000F4D3511CCAB2AA42E7D3BDE8F08100B55F
:10602000ADF2844DFDF791FE01464FF49062684653
:1060300011F072FC6846FDF78AFE0DF2844D00BD3A
:106040002DE9F04F83B012200190384836494FF0C7
:1060500020090024C16001E0032C01DA14261AE0B3
:10606000E01E032838BF152615D3A01F032838BF0C
:10607000162610D3A4F10900032838BF24260AD31A
:10608000A4F10C00032838BF252604D3A4F10F0087
:10609000032838BF2626B34509D020483109B34626
:1060A0000068C16106F00F017F20FAF7CDF90025E5
:1060B000B9F1000F2ADD1E484FEA161A80FB0410C2
:1060C000A0EBE070A0EB800000EB0408BAF1010F38
:1060D0000EBF05EB4810C5F11F0000EB481087B25A
:1060E0001249C86810F8012B0092C860F8B2114636
:1060F000FAF7AAF900BF00BF00BF00BF00BFF8B2A7
:106100000099FAF7A1F96D1C4D45DFDB0198641C7D
:106110008442A1DB03B0BDE8F08F00006490110061
:10612000BE050020BF05002034330020D405002028
:10613000565555552DE9F84FDFF8D8B174484FF052
:106140002008CBF80C0012200024009001E0032C62
:1061500001DA14261AE0E01E032838BF152615D3ED
:10616000A01F032838BF162610D3A4F10900032866
:1061700038BF24260AD3A4F10C00032838BF2526F3
:1061800004D3A4F10F00032838BF2626B24509D056
:1061900061483109B2460068C16106F00F017F20F5
:1061A000FAF752F90025B8F1000F1EDD5B484FEAFF
:1061B000161980FB0410A0EBE070A0EB800007191B
:1061C000B9F1010F0EBF05EB4710C5F11F0000EB41
:1061D000471080B2FAF751F9DBF80C106D1C4545F9
:1061E00001F8010BCBF80C10EADB0098641C844228
:1061F000ADDBDBF80C00BDE8F88F4648C08870477F
:106200002DE9F043002787B0B946FAF7E9FE414986
:106210004FF400608880FAF790FD0020FAF77DFDCA
:1062200000254FF05A082846FEF7DFFFFAF7DBFF9C
:1062300003F065F86846FBF7A6FA28B3684603F052
:106240008EFC002420262046FBF7C8F8002130F9F8
:10625000022BA2F26662B2F54D7F88BF641C491C16
:10626000B1EB460FF3D3ACB1454515D2FAF7B8FE02
:10627000A8B26D1CFEF7B9FFFAF7B5FF06F0C0FC37
:10628000002808BFFBF7B0FD002FD1D0B9F1000FF7
:106290000BD104E00127F9E7FAF7A2FE05E0002F91
:1062A0001EBF002007B0BDE8F083012007B0BDE8A5
:1062B000F08370471748816800291BBF017811F0EF
:1062C000020F0020C068704715481249006890F816
:1062D00025218878401CC0B28870824228BF704750
:1062E0000020887001210846FEF72CBC10B506F08E
:1062F00087FC074902284FF4107204D0BDE8104013
:10630000084811F009BBBDE81040074811F004BB74
:1063100034330020D40500206490110056555555A3
:10632000E8060020620C00201C6200201FB513F05C
:10633000070F069804D003F00702022A08D004E0F1
:10634000012202A90F2002F0B6FF04B0002010BD08
:10635000F84B5A79052A0DD1DA8982423CBF521C8A
:10636000DA8192B2824205D10020D88101200870E2
:106370000320587104B0012010BD1FB513F0070FA2
:1063800004D003F00700022808D004E0012202A98B
:106390000F2002F090FF04B0002010BD0120087013
:1063A00004B010BD1FB513F0070F04D003F00700B1
:1063B000022808D004E0012202A90F2002F07BFF8E
:1063C00004B0002010BD0120087004B010BD1FB53E
:1063D00013F0070F04D003F00700022808D004E0F0
:1063E000012202A90F2002F066FF04B0002010BDB8
:1063F0000120087004B010BD1FB513F0070F04D0C2
:1064000003F00700022808D004E0012202A90F20AF
:1064100002F051FF04B0002010BD0120087004B04C
:1064200010BD2DE9F00703F007050027C14EDDF888
:106430001CC0012D08BFF7810DD013F0070FBD4B15
:10644000DFF8F482DFF8F492DB8903F10104A4B2EF
:1064500005D0022D16D0BDE8F00700207047634537
:106460003CBFD9F80000C254F481644524D1D9F866
:106470000000D9F800104078097800EB0120A8F856
:106480000E0019E0B8F80E20D9F80050120A634542
:106490002A70D9F8005098F80E206A7004D2D9F802
:1064A0000020D25C0270F481F089604504D1F7814C
:1064B0000120087003207071BDE8F00701207047CB
:1064C0001FB513F0070F04D003F00700022808D00F
:1064D00004E0012202A90F2002F0EDFE04B000202A
:1064E00010BD0120087004B010BD1FB513F0070FD8
:1064F00004D003F00700022808D004E0012202A91A
:106500000F2002F0D8FE04B0002010BD012008705A
:1065100004B010BD1FB513F0070F04D003F007003F
:10652000022808D004E0012202A90F2002F0C3FED5
:1065300004B0002010BD0120087004B010BD1FB5CC
:1065400013F0070F069804D003F00702022A08D0C0
:1065500004E0012202A90F2002F0ADFE04B00020E9
:1065600010BD744B5A79052A0DD1DA8982423CBF9D
:10657000521CDA8192B2824205D10020D8810120DA
:1065800008700320587104B0012010BD002070472E
:1065900008B503F00700012806D18DF80000024677
:1065A00069460B2002F087FE002008BD08B503F005
:1065B0000700012807D100208DF80000012269465C
:1065C0000B2002F078FE002008BD10B503F0070094
:1065D000012808BFFEF7FBFA002010BD08B503F044
:1065E0000700012807D103208DF800000122694629
:1065F000002002F060FE002008BD08B503F007008F
:10660000012807D103208DF80000012269460020EF
:1066100002F051FE002008BD70B403F00702002410
:10662000444BDDF80CC0012A02D0022A08D004E055
:1066300005205871DC811C639C8270BC002070476F
:106640005A79052A11D1DA89624506D23C4DAD68E6
:10665000D600F5400570501CD881D889604504D11A
:10666000DC81012008700320587170BC0120704744
:106670001FB513F0070F08D19DF80800F02807D0C8
:10668000012202A9072002F016FE04B0002010BD6E
:10669000FEF7CEFBF9E71FB513F0070F04D1012277
:1066A00002A9104602F007FE04B0002010BD2DE93B
:1066B000F00103F007041F4E059D012C04BF0020CC
:1066C000F0811ED013F0070F1A4B1E4FDB8903F128
:1066D000010C1FFA8CFC02D0022C16D011E01749D5
:1066E000022B3CBF0868C254A6F80EC0AC4508D1C6
:1066F00008680278386880F8EB200968497880F8E3
:10670000EA10BDE8F001002070470E4A002B126825
:1067100004BF92F8EB10017006D0012B04D192F85F
:10672000EA20027001200870A6F80EC0BDE8F00152
:1067300001207047EC050020F80F00209090110018
:1067400014160020E806002030B403F0070CF84CC3
:10675000BCF1010F04BF0020E08118D013F0070F37
:10676000F34BDB8903D0BCF1020F13D00FE073B9F8
:10677000A271082A0BD2DFE802F004070704040420
:1067800004044FF4906001E04FF41070E06230BCFC
:1067900000207047E64A002BD26A04BF110A01703C
:1067A00004D0012B02D1027001200870581CE08136
:1067B00030BC01207047F8B5054603F007000026FD
:1067C000DB4C0F46012807D013F0070F2346DB8967
:1067D00006D0022828D025E005206071E68121E05E
:1067E00003BBA2714FF49060A0824010082A19D216
:1067F000DFE802F004060A0E10121416CD4810E06D
:10680000CD492163A0820DE0CC492163A08209E03B
:10681000CB4806E0CB4804E0CB4802E0CB4800E0A0
:10682000CB4820630020F8BD6079052847D1206B54
:10683000002844D0C749BE4A0968928A91F8EB10F3
:10684000012918BF032906D0694693422DD213F0BF
:10685000030F21D118E0934227D213F0010F07D084
:1068600094F82C002870E06A000AE062581C1BE0D3
:10687000AF49A079C989042821F0010214BFB648A4
:10688000B648805EE062EBE70422FBF719FC009853
:10689000E062206B001D206394F82C002870E06AF1
:1068A000000AE062E089401CE081E089A18A884218
:1068B00005D1E68101202663387003206071012034
:1068C000F8BD2DE9F84303F007020026984D089C17
:1068D0000F468046012A02D0022A06D002E0052097
:1068E0006871EE810020BDE8F883687905281CD125
:1068F000E889A04211D2FCF7EAFEAC208DF8000036
:106900007A208DF8010070208DF80200EA891DF8C8
:10691000020088F80000501CE88180B2A04204D137
:10692000EE8101203870032068710120BDE8F883F2
:106930002DE9F04182B003F0070200267C4D089C4F
:106940000F468046012A02D0022A07D002E0052025
:106950006871EE8102B00020BDE8F08168790528F9
:1069600021D1E889A04216D2FCF7B1FE53208DF860
:10697000000045208DF801007A208DF8020070207B
:106980008DF803008DF80460EA891DF8020088F88C
:106990000000501CE88180B2A04204D1EE810120A9
:1069A00038700320687102B00120BDE8F0812DE944
:1069B000F00388B003F007020027DFF87481DDF8E8
:1069C00038C0012A09D04446E489651CAEB2022AC7
:1069D0000DD013F0070F2FD004E0052088F8050034
:1069E000A8F80E7008B00020BDE8F003704798F8D2
:1069F0000520052A1BD164450ED2594D00226B4655
:106A000015F8029003F80290521CD2B2202AF7D354
:106A10001A5D0270A8F80E60B8F80E00604506D145
:106A2000A8F80E7001200870032088F8050008B04F
:106A30000120BDE8F0037047644538BFA8F80E6038
:106A4000B8F80E00604508BFA8F80E70CAE72DE937
:106A5000F007DFF800C183B003F0070ADCF800C0DC
:106A60000A9A0027BCF81640BCF81450DFF8C08022
:106A7000BAF1010F0ED0C4464FF00109BCF80EC0A8
:106A8000BAF1020F0CF10106B6B20DD013F0070FE8
:106A900040D004E0052088F80500A8F80E7003B087
:106AA0000020BDE8F007704798F80530052B2CD181
:106AB00094451FD2230A8DF800308DF804304FEA38
:106AC000152A12238DF808308DF801408DF8054005
:106AD00020238DF802A08DF806A08DF809308DF8DE
:106AE00003508DF807508DF80A701DF80C300370B4
:106AF000A8F80E60B8F80E00904206D1A8F80E7003
:106B000081F80090032088F8050003B00120BDE85B
:106B1000F00770471348944580F8009038BFA8F8F4
:106B20000E60B8F80E00904208BFA8F80E70B6E7E5
:106B3000EC05002054B0020054D8020054DC0200DE
:106B400054C8020054D0020054C0020054B80200DD
:106B500054EC0200E8060020006D002000750020C3
:106B6000F4370020440700202DE9F04383B080462D
:106B700003F007000026FF4D0A9C0F46012802D0B3
:106B8000022807D002E005206871EE8103B00020E2
:106B9000BDE8F083687905282DD1E8894FF0010917
:106BA000A04220D20021B220FBF75EF88DF8000051
:106BB000010A8DF80110010C8DF80210000E8DF8FD
:106BC00003007A208DF804001F208DF805000420B2
:106BD0008DF807008DF80690E8891DF8001088F8F8
:106BE0000010401CE88180B2A04204D1EE8187F8F9
:106BF00000900320687103B00120BDE8F0832DE907
:106C0000F84303F007020026DA4D089C0F46804641
:106C1000012A02D0022A06D002E005206871EE8126
:106C20000020BDE8F8836879052814D1E889A042DE
:106C300009D26846FBF72FFDEA891DF8020088F8A3
:106C40000000501CE88180B2A04204D1EE810120F6
:106C50003870032068710120BDE8F88310B403F098
:106C60000701DFF810C3012906D013F0070FC24B4C
:106C700008D0022910D00CE00020ACF80E00ACF8CF
:106C8000100006E0BCF80E0019680A54401CACF86D
:106C90000E0010BC00207047BCF810101A68525C3F
:106CA0000270481CACF8100010BC01207047F0B511
:106CB00083B003F0070201270025AF4CAD4EDDF88D
:106CC00020C0012A04D0022A00F0C68000F09DB83E
:106CD000FCF7FDFC012202A912200295FBF7F0F956
:106CE0000520707121687A2008702068477021683B
:106CF00021208870A14822680168897CD1700068D1
:106D00002268017C1171017E11F0040F0ED0C18A3E
:106D10002268090A51712268817D9171818A2268F5
:106D2000090AD1712168007D08720DE0818A22680C
:106D3000090A51712268017D9171C18A2268090A8C
:106D4000D1712168807D0872042269461046009541
:106D5000FBF7B6F92168009848722268010A91721F
:106D60002268010C000ED172216804220873694662
:106D700014200095FBF7A4F9216800984873226855
:106D8000010A91732268010C000ED1732168087406
:106D90000298009500283BD0042201A948200195C3
:106DA000FBF78EF9019804225030019069461C309F
:106DB000FBF786F92168009848742268010A9174EB
:106DC0002268010C000ED174216804220875009518
:106DD00001A948200195FBF773F90198042250306E
:106DE000019069462C30FBF76BF9216800984875D3
:106DF0002268010A91752268010C000ED175216884
:106E000008762168FF204876F58103B00020F0BDA8
:106E1000042269465A48FBF753F9216800984874E0
:106E20002268010A91742268010C000ED174216855
:106E300004220875694653480095FBF741F921681B
:106E4000009848752268010A91752268010C000EAD
:106E5000D17521680876D4E77279052A0ED1F289B6
:106E6000624504D223689B5C0370501CF081F0895A
:106E7000604503D1F5810F700320707103B00120CC
:106E8000F0BD30B403F007043B4B3A4D029A4FF08B
:106E9000000C012C02D0022C38D034E002206871A2
:106EA0003948A5F80EC00168880A444211EB8424D1
:106EB00018BF401C404201EB8000C01C20F00300C2
:106EC0003249B0F5003F014414D8CC78086864F327
:106ED0001F602F4CA0420DD10020002A13D901EBD6
:106EE000000C1C689CF804C004F800C0401C8242DE
:106EF000F5D808E00020002A05D9196801F800C07B
:106F0000401C8242F9D830BC002070476C79022CBA
:106F100010D1EC89944204D21B681B5D0370601C85
:106F2000E881E889904205D1A5F80EC001200870DB
:106F30000320687130BC0120704738B503F00702A8
:106F40000D4C00250B4BDDF810C0012A02D0022A9F
:106F50007ED086E0022058710E48DD8100680E491F
:106F6000884245D10D480168226811700168226885
:106F7000090A15E0EC05002090901100E8060020B9
:106F80005CC001006CC0010000FE1100E8FF0F00B2
:106F900034CD12ABF015002054464953FC150020A7
:106FA000517001682268090C917001682268090E0D
:106FB000D17041682268117141682268090A5171D3
:106FC00041682268090C917141682268090ED171EB
:106FD00081682268117281682268090A5172816889
:106FE0002268090C917280682168000EC87238E02E
:106FF0000422694620200095FBF762F8216800987A
:107000000422087000982168000A487000982168DE
:10701000000C887000982168000EC8706946242012
:10702000FBF74EF82168009808712268010A517137
:107030002268010C000E917121680422C871694612
:107040002820FBF73DF8216800980872010A00E04B
:1070500009E0226851722268010C000E91722168C9
:10706000C872002038BD5A79022A0FD1DA896245E8
:1070700004D22468A45C0470501CD881D88960456F
:1070800004D1DD810120087003205871012038BD32
:1070900070B503F007020025FA4CFB4BDDF810C079
:1070A000012A03D0022A0DD0002070BD02205871A1
:1070B000DD8103F0E5FE002814BF80204020216818
:1070C0000870F1E75A79022A0FD1DA89624504D2B1
:1070D0002468A45C0470501CD881D889604504D110
:1070E000DD810120087003205871012070BD70B54A
:1070F00003F007020025E34CE34BDDF810C0012A42
:1071000002D0022A10D00DE002205871DD8100204B
:10711000FBF729FE05460120FBF725FE216845EA1D
:1071200000100870002070BD5A79022A0FD1DA8948
:10713000624504D22468A45C0470501CD881D889AC
:10714000604504D1DD8101200870032058710120C1
:1071500070BD30B403F007020024CA4DCA4BDDF8FD
:1071600008C0012A02D0022A09D005E00220587185
:10717000DC8129685520087030BC002070475A799E
:10718000022A0FD1DA89624504D22D68AD5C057000
:10719000501CD881D889604504D1DC810120087059
:1071A0000320587130BC012070472DE9F84303F0EB
:1071B00007020026B34DDFF8D082089C4FF001098A
:1071C000012A02D0022A2CD028E003F09AFE876917
:1071D000022088F80500A8F80E6004226946002005
:1071E000FAF76EFFA948009981420FD1286880F80C
:1071F0000090296804204870286887702968380A38
:10720000C870286846712868867107E00020002C45
:1072100004D929680E54401C8442FAD80020BDE8E5
:10722000F88398F80520022A14D1B8F80E20A2425B
:1072300005D22B689B5C0370501CA8F80E00B8F8B0
:107240000E00A04206D1A8F80E6081F8009003203D
:1072500088F805000120BDE8F883F8B503F00702BF
:10726000884C0025884EDDF818C0012A02D0022A79
:1072700070D06CE003F045FE00282ED084480168F1
:107280002268117001682268090A51700168226839
:10729000090C917001682268090ED170416822685A
:1072A000117141682268090A517141682268090C0C
:1072B000917141682268090ED1718168226811724A
:1072C00081682268090A517281682268090C9172EA
:1072D00080682168000EC87236E0042269466D4855
:1072E0000095FAF7EDFE21680098042208700098D6
:1072F0002168000A487000982168000C8870009886
:107300002168000EC87069466348FAF7D9FE216803
:10731000009808712268010A51712268010C000E60
:10732000917121680422C87169465C48FAF7C8FE69
:107330002168009808722268010A51722268010CC3
:107340009172010E2068C17202207071F5810020D7
:10735000F8BDFFE77279022A0FD1F289624504D2A3
:1073600023689B5C0370501CF081F089604504D158
:10737000F58101200870032070710120F8BD38B537
:1073800003F007023F4C00253F4BDDF810C0012AF7
:1073900002D0022A4FD04CE0022058714048DD81D3
:1073A00001683A4A91421ED14168226811704168D1
:1073B0002268090A517041680A0C21688A70416884
:1073C0002268090ED1708168226811718168226873
:1073D000090A517181682268090C917180682168DD
:1073E000000EC87125E00422694610460095FAF7A0
:1073F00067FE216800980422087000982168000A3E
:10740000487000982168000C887000982168000E70
:10741000C87069460820FAF753FE21680098087181
:107420002268010A51712268010C000E91712168D5
:10743000C871002038BD5A79022A0FD1DA89624515
:1074400004D22468A45C0470501CD881D88960459B
:1074500004D1DD810120087003205871012038BD5E
:107460002DE9F04F85B0934603F00702DFF818903E
:10747000DDF838C0012A15D013F0070F19D0022A01
:1074800076D070E090901100EC05002054464953EE
:107490000816002068C001006CC0010070C0010027
:1074A000F0150020022089F805000020A9F80E0040
:1074B00059E0002440274FF001081BF0010F28D0AD
:1074C000BA46042203A95046FAF7FAFD042201A99C
:1074D0004820FAF7F5FDFB490398884240D101980E
:1074E0000025B5EB900F10D20AEB85000422694607
:1074F000FAF7E6FD0098032D044408BF06466D1C0C
:107500000198B5EB900FEFD304B93446B8F1000FF2
:1075100026D01BF0020F1DD00020042202A9FBF789
:107520001DF9E949029888421AD10025B5EB970F59
:107530000DD2A80004226946FBF710F90098062D29
:10754000044408BF06466D1CB5EB970FF1D3002C21
:1075500008BF3446B8F1000F18BFC9F82C4002D15B
:107560000020C9F82C0005B00020BDE8F08FFFE72F
:1075700099F80520022A1AD1B9F80E2062450AD2DC
:10758000C2F10303D9F82C40DB0024FA03F30370A3
:10759000501CA9F80E00B9F80E00604507D1002074
:1075A000A9F80E0001200870032089F8050005B035
:1075B0000120BDE8F08F10B503F00700012804D1C9
:1075C000002211461C2001F076FE002010BD70B58F
:1075D000044603F00700BD4D0E46012804BF0020FD
:1075E000E88119D013F0070F02D0022816D013E05B
:1075F000E889B74B03283CBF19680A54401C80B285
:10760000E881032808D1186890F9022090F9011048
:1076100090F90000FCF77AFD002070BDFCF7BFFC7C
:107620000246E88930B101280AD002280ED003288A
:1076300012D018E014211046FCF7BAFC207012E0BA
:1076400015211046FCF7B4FC20700CE01621104602
:10765000FCF7AEFC207006E017211046FCF7A8FCF2
:10766000207001203070E889401CE881012070BD45
:1076700013F0070F04D003F00702022A05D002E03E
:1076800092490020C88100207047924A1268027017
:1076900001200870704730B403F007030024DFF8BE
:1076A0002CC2029A012B02D0022B0BD007E005203E
:1076B0008CF80500ACF80E4020208CF8060030BC99
:1076C000002070479CF80530052B14D1BCF80E3013
:1076D000934205D29CF806500570581CACF80E0079
:1076E000BCF80E00904206D1ACF80E4001200870A4
:1076F00003208CF8050030BC012070472DE9F043D1
:1077000083B003F00705724E704FDDF828C04FF0CC
:107710000008012D0AD013F0070F3B46DB8903F167
:107720000104A4B211D0022D22D01DE001A96846A7
:1077300001F098FF05207871316801980870316870
:1077400000984870A7F80E800EE0634502D23068BA
:10775000C254FC81F889604506D1A7F80E803068D4
:107760000178407801F075FF03B00020BDE8F08398
:107770007A79052A0ED1634503D23268D25C027051
:10778000FC81F889604505D1A7F80E8001200870BA
:107790000320787103B00120BDE8F08370B503F0D9
:1077A00007000024494D4A4EDDF810C0012803D0DF
:1077B00013F0070F06D043E0EC81306804703068A6
:1077C00044703DE0E889604503D233681A54401C98
:1077D000E88180B2604533D13FA001220068EC818E
:1077E0000A703168C2B20978914229D13168C0F378
:1077F00007204978814223D11C2600244FF48015AC
:1078000005EB0430FAF7DAFD022808BF70BD601CF2
:10781000C4B2B442F4D3032600244FF48E1505EB12
:107820000430FAF7CBFD022808BF70BD601CC4B25B
:10783000B442F4D32948FAF7C1FD022808BF70BD4D
:10784000002070BD10B503F00700012808BF02F04A
:10785000DBF9002010BD70B503F007041B4D012CAF
:1078600009D013F0070F2B46D3F82CC0DB8908D0C2
:10787000022C17D014E00020E88104F0C6FDE86275
:107880000EE0002B04BF1002E86206D0012B04D1E9
:107890004CEA0200E86204F0B1FDE889401CE8818E
:1078A000002070BD002B04BF4FEA1C21017005D0E1
:1078B000012B03D180F800C001200870581CE8811A
:1078C000012070BD5446435354464953EC050020F3
:1078D000909011007005002055AC000000FE1100D2
:1078E00070B5064603F00700F84C0D46012808BFA6
:1078F00000200DD013F0070F02D002280BD008E0B3
:10790000E089002804BF104607F0B4FAE089401C63
:10791000E081002070BD07F0AAFA307001202870C5
:1079200070BD70B503F0070CE84D0E460446BCF17F
:10793000010F06D013F0070F07D0BCF1020F1CD0C7
:1079400019E00020E881288215E0E889002804BFBA
:107950001002E8620CD001280AD1E86A1043E862FC
:10796000F9F73EFBA88D80B2FDF73FFCF9F73BFC31
:10797000E889401CE881002070BD288A02280CD2CA
:10798000FEF73BFC2A8A002A04BF000A207004D0BC
:10799000012A02D1207001203070288A401C2882E0
:1079A000012070BD10B513F0070F04D003F00702DB
:1079B000022A08D005E0002A14BF0120002006F0AA
:1079C00070F9002010BDC24A92F85420D20802700B
:1079D0000120087010BD0020704770B503F0070249
:1079E0000026BC4CB94DDDF810C0012A02D0022A95
:1079F00015D012E005F02DF921680870FDF790F818
:107A00002168487003F0FCF821688870FDF78BF856
:107A10002168C87005206871EE81002070BD6A7908
:107A2000052A0FD1EA89624504D223689B5C037062
:107A3000501CE881E889604504D1EE81012008707E
:107A400003206871012070BD70B5064603F0070081
:107A50000D4602281CBF002070BD01F046FC002826
:107A600014BF0124002401F043FC002814BF0222AB
:107A70000022224332700120287070BD30B403F020
:107A80000703944A0024914DDDF808C0012B02D071
:107A9000022B4AD046E090490868904B98422FD17B
:107AA0004868B0F5887F2BD8C868FF282EBFFF2014
:107AB000C868C0B2136818700869FF283ABF08691F
:107AC000C0B2FF20136858704869FF283ABF486960
:107AD000C0B2FF201368987088681368000AD870D5
:107AE00088691368187188691368000A5871886971
:107AF000030C1068837188691168000EC87110E06A
:107B00001068047010684470106884701168FF2059
:107B1000C87011680871116848711168887111681E
:107B2000C871EC8130BC00207047EB89634504D2FA
:107B30001268D25C0270581CE881E889604502D165
:107B4000EC810120087030BC012070472DE9F04124
:107B500003F0070100255D4C0646012904BFE561DD
:107B6000E58101D0022902D00020BDE8F081207F0C
:107B7000584F00F00701E1812078084304D13868AC
:107B800002F0C0F801202070E189052928BF257086
:107B90003868405C3070E069401CE0610120BDE85D
:107BA000F08170B503F0070200254A4B474CDDF821
:107BB00010C0012A02D0022A08D005E0186802F09D
:107BC000A1F805206071E581002070BD6279052A69
:107BD0000FD1E289624504D21B689B5C0370501C84
:107BE000E081E089604504D1E5810120087003202F
:107BF0006071012070BD70B503F007020025334CA1
:107C0000012A02D0022A11D00EE005206071002165
:107C1000E581084601F026FD4FF6FF7101EA4000BC
:107C2000608201F02BFDA061002070BD6279052A01
:107C300016D1E289B4F812C0624507D212F0010FE2
:107C40001CBFA37903700DD0501CE081E089604512
:107C500006D1E581012008700320607101F01CFD50
:107C6000012070BDA66922F00103F35A1E0A0670B6
:107C7000A371E9E77FB51C460E46054613F0070FD2
:107C800008D103F0FDF828B1012202A91D2001F05E
:107C900012FB03E004F00700022802D004B0002029
:107CA00070BD01F0B8FD28700120307004B070BDC7
:107CB0002DE9F04103F007020027044E88460546EF
:107CC000012A0DD0022A16D012E00000EC05002097
:107CD000F80F0020909011001416002054435246D3
:107CE00005207071F7810A20708201F0C7FCB06135
:107CF0000020BDE8F0817079052818D1F289708ADA
:107D0000824208D212F0010F1CBFB079287011D046
:107D1000F089401CF081F089718A884207D1F7818F
:107D2000012088F800000320707101F0B5FC0120EB
:107D3000BDE8F081002401F06EFD012804D1F08936
:107D4000B16920F001000C5A200A2870B471DFE7F5
:107D50007FB50D46044613F0070F04D003F007006B
:107D6000022808D004E0012202A90A2001F0A3FAA7
:107D700004B0002070BD04F06CFF2070012028705A
:107D800004B070BDF8B503F007020025FF4C0E46A5
:107D90000746012A02D0022A0ED00BE005206071AE
:107DA00003F07BFA206300281ABF44F26440A082EB
:107DB000A582E5810020F8BD6079052822D1E289FD
:107DC000A08A6946824214D212F0030F08D104221D
:107DD000206BFAF775F90098E062206B001D2063B4
:107DE00094F82C003870E06A000AE062E089401CD8
:107DF000E081E089A18A884204D1E58101203070C8
:107E0000032060710120F8BD10B513F0070F04D0F6
:107E100003F00702022A0DD00AE0012A05D0002A49
:107E200004BF0120FAF775FF02E00120FAF766FFB0
:107E3000002010BDD64A1268126802F002020270D9
:107E40000120087010BD70B50D46044613F0070FF1
:107E500004D003F00700022808D005E0002A14BF70
:107E60000120002001F0C2FE002070BD01F0C5FE1F
:107E7000002814BF0122002222700120287070BD4A
:107E800070B503F00700C14D1446012808BF00205B
:107E900016D013F0070F14D1E889002808BFAA7183
:107EA0000CD001280AD1A879FAF765FFA8792040FB
:107EB000FAF724FFA879A043FAF72BFFE889401CC2
:107EC000E881002070BD2DE9F00103F00704AF4EFA
:107ED000059F012C04BF0020F08135D013F0070F5F
:107EE000AA4BAC4DDB8903F1010C1FFA8CFC02D0CC
:107EF000022C2DD028E0A8490868C254781E83427D
:107F000020D10868007830B101280AD002280ED0AC
:107F1000032812D016E008682968407881F88001AB
:107F200010E008682968407881F881010AE0086853
:107F30002968407881F8820104E00868296840785F
:107F400081F88301A6F80EC0BDE8F001002070475B
:107F5000904A126813B1012B0AD014E092F88011F4
:107F600001F00F0392F8811163F31F1101700AE011
:107F700092F8823192F8832103F00F0363F31F120A
:107F8000027001200870A6F80EC0BDE8F0010120C3
:107F9000704710B4DFF804C213F0070F04D003F0E9
:107FA0000702022A18D014E0012A01D04AB110E0D9
:107FB000DCF80000806ADCF8001020F00300886222
:107FC00007E0DCF80000806ADCF8001040F00300F5
:107FD000886210BC00207047DCF80020926A0270B2
:107FE0000120087010BC704770B503F00700002531
:107FF000664C0E46012806D013F0070F04BF6079C7
:10800000022805D019E002206071E581E56214E0E4
:10801000E089A18A884207D2614811460068FBF7CF
:10802000E8FAE089401CE081A18A80B2884204D14C
:10803000E5810120307003206071002070BD2DE9C2
:10804000F04103F007020025504C0E460746012A76
:1080500002D0022A06D002E002206071E5810020F1
:10806000BDE8F0816079022814D1E189A08A8142BB
:1080700007D24B480068FBF7EAFA3870E089401CE9
:10808000E081E089A18A884204D1E5810120307035
:10809000032060710120BDE8F08110B503F00702F4
:1080A0003A4C012A02D0022A27D024E003F0F8F843
:1080B0000023002804BF2363A3821BD000F15401D6
:1080C00021634168B1F5887F90F820100CD390F8B7
:1080D000212001EB020C01FB02C190F8222090F854
:1080E00023001044084404E090F822000A1801FB21
:1080F0000020A082E381002010BDE289A38A9A4279
:1081000007D2D4F830C01CF802C080F800C0501C60
:10811000E081E089984204BF01200870012010BD71
:1081200010B513F0070F04D003F00702022A05D0A0
:1081300002E0104601F0BDFA002010BD194A127885
:1081400002700120087010BD1FB513F0070F04D195
:10815000012202A9092001F0AEF804B0002010BDF0
:1081600070B503F007000949012804BF0020C88149
:1081700030D013F0070F2DD1C889074C03283CBF1E
:1081800023681A54401C80B2C8810DE0EC05002021
:1081900058901100E80600209090110060901100A6
:1081A0007C90110031060020032813D1F8F72AFF34
:1081B0002068B0F8010045BAF8F742FD040018BF86
:1081C000F9F75CF829460020F8F791FC002C18BF5D
:1081D000F9F756F8002070BD70B503F00700F949B3
:1081E000012804BF0020C88124D013F0070F21D13B
:1081F000C889F54D02283CBF2B681A54401C80B238
:10820000C881022816D1F8F7FDFEF8F719FD040021
:1082100018BFF9F733F82868007818B12868407853
:10822000F8F769FC28684078F8F765FC002C18BF5F
:10823000F9F726F8002070BD13F0070F04BFE148DE
:10824000C270002070477FB50D46044613F0070F3B
:1082500004D003F00700022808D004E0012202A99C
:108260000E2001F028F804B0002070BD04F0B8FC26
:10827000002814BF0122002222700120287004B0BF
:1082800070BD7FB50D46044613F0070F04D003F010
:108290000700022808D004E0012202A90F2001F003
:1082A0000AF804B0002070BD04F08BFC207001209F
:1082B000287004B070BD10B503F00700DFF804C3E8
:1082C0000299012804BF0020ACF80E001AD013F068
:1082D000070F17D1BCF80E00BB4B03283CBF1C682E
:1082E0002254401C80B2ACF80E0088420AD11868B3
:1082F0001968B0F80100097840BA00B2002908BF37
:10830000FCF770FF002010BD10B503F00700DFF888
:10831000B4C20299012804BF0020ACF80E0017D0A7
:1083200013F0070F14D1BCF80E00A74B03283CBF75
:108330001C682254401C80B2ACF80E00884207D161
:108340001868B0F8010041BA18680078F9F725FB01
:10835000002010BD70B503F007029A4CDDF810C084
:10836000012A02D0022A07D004E00020E081FAF7B7
:1083700093FFE062002070BDE289624506D2C2F13F
:108380000303E56ADB0025FA03F30370501C80B297
:10839000E081604504BF01200870012070BD70B508
:1083A000044603F0070C0020864DBCF1010F06D0F7
:1083B00013F0070F07D0BCF1020F13D010E0E881D3
:1083C0002882A8710CE0E889002808BFAA7104D0AF
:1083D00001227E49102000F06EFFE889401CE881F0
:1083E000002070BD2A8A3AB1207001200870288AC6
:1083F000401C2882012070BD04F077FC2070F6E755
:1084000070B50D46044613F0070F04D003F00700C3
:10841000022805D002E0104606F0DAF8002070BD10
:1084200006F0D9F820700120287070BD10B513F047
:10843000070F1FD1500048F6B801B1FBF0F46449B2
:1084400003200968C86101217F20F7F7FDFFE1B231
:108450004FF48470F7F7F8FF20460FF0B0FF5D4A45
:108460005D4B10F013F80FF07DFFC1B24FF4857033
:10847000F7F7EAFF002010BD10B513F0070F4ED13B
:10848000122A4CD2DFE802F0090E132B2B2B2B30D3
:108490003336393C4B4B4B3F42475049002009682B
:1084A00008773CE04D4901200968087737E04849E2
:1084B00003200968C86101217F20F7F7C5FF152156
:1084C0004FF48770F7F7C0FF75214FF48470F7F70A
:1084D000BBFF4D214FF48570F7F7B6FF1FE0002179
:1084E000D01E04F0FEFC1AE0F9F729FD17E0F8F7BA
:1084F0007AFE14E0F8F774FD11E004F0F6FA0EE0ED
:1085000004F006FB0BE0FDF715FE08E033490220FE
:108510000968088603E031490020096808860020C0
:1085200010BD10B5144613F0070F16D1072C14D840
:10853000274903200968C86102217F20F7F784FFDB
:10854000052040EA041140F20220F7F77DFF04F114
:1085500088014FF40170F7F777FF002010BD7FB559
:108560000C46054613F0070F04D003F0070002285D
:1085700008D004E0012202A9062000F09CFE04B00D
:10858000002070BDFCF7CCFA022808BF00200BD0F9
:10859000032808BF022007D0042808BF032003D007
:1085A000052814BFFF20012028700120207004B08E
:1085B00070BD10B5104613F0070F08BF04F02BFB79
:1085C000002010BDEC05002090901100F205002065
:1085D000649011001F85EB51B81EE53FE8060020AE
:1085E00010B5104613F0070F08BF04F020FB002061
:1085F00010BD70B5044603F007000D4602281CBFED
:10860000002070BD04F020FB20700120287070BD98
:1086100070B403F007020024FE4BDDF80CC0012A01
:1086200005D0022A04BF5A79022A0AD01BE0022090
:108630005871F948DC816FF07F410068081AD862F0
:1086400011E0DA89624506D2DE6AD50026FA05F520
:108650000570501CD881D889604504D1DC81012087
:1086600008700320587170BC0120704713F0070F89
:1086700004BFEA4802700020704710B5944603F02A
:108680000700E449029A012804BF0020C88112D0E3
:1086900013F0070F0FD1C889E14B90423CBF1C6813
:1086A00004F800C0401C80B2C881904203D10D2064
:1086B000196800F000FE002010BD70B503F007043B
:1086C000D44D012C0AD0AC4613F0070FBCF8123081
:1086D000DCF830C006D0022C21D01EE00020E8815A
:1086E00028821AE0E889002808BF2A6312D00128EE
:1086F00004BF501C68820DD0022816BFC11EAA827A
:10870000994207D2297D0844C01EC1B20CF0FF0077
:10871000F9F7F7FAE889401CE881002070BDFF22D4
:10872000027093B12A8A9444521CBCF5807F0BD20C
:108730000CF5801C0CF5F83C9CF800C080F800C0DB
:108740009A4204BF012008702A82012070BD2DE9E1
:10875000F04103F007050026AE4C9446012D04BFFE
:10876000E681268224D013F0070FAA4B5A8A1B6B8E
:1087700002D0022D28D01BE0E089002808BFC4F8F1
:1087800030C012D0012816D0A549801E90423CBFAF
:108790000D6805F800C0401C904206D103F580101A
:1087A000096800F5F830FAF787F8E089401CE081A5
:1087B0000020BDE8F0810CF1010060821844B0F5A2
:1087C000807F88BF6682F0E74FF0FF0C80F800C022
:1087D0009AB1258A03EB050C6B1CBCF5807F0BD28C
:1087E0000CF5801C0CF5F83C9CF800C080F800C02B
:1087F000934204BF0120087023820120BDE8F0816C
:1088000010B5944603F007008249029A012804BF7C
:108810000020C88112D013F0070F0FD1C889804BF8
:1088200090423CBF1C6804F800C0401C80B2C88164
:10883000904203D10220196800F03DFD002010BDD8
:1088400010B5944603F007007249029A012804BF4C
:108850000020C88112D013F0070F0FD1C889704BC8
:1088600090423CBF1C6804F800C0401C80B2C88124
:10887000904203D10320196800F01DFD002010BDB7
:1088800013F0070F05D003F00700022804BF0120F2
:108890007047002070471FB513F0070F04D1012265
:1088A00002A9112000F007FD04B0002010BD03F064
:1088B0000701DFF860C10098012907D013F0070F06
:1088C00004BF9CF80510012909D01FE001208CF895
:1088D00005000020ACF80E00CCF8280014E0BCF82D
:1088E0000E10814208D2DCF82830491C42EA0322EB
:1088F000CCF82820ACF80E1089B2814206D10320B2
:108900008CF80500DCF82800CCF830000020704717
:1089100003F007003F494FF0010C012806D013F087
:10892000070F04BF4879012807D014E081F805C07B
:108930000020C881087148620DE0C889002804BF82
:108940000A71A1F80EC006D0012806D00323022820
:1089500018BF4B7106D000207047100248620220F9
:10896000C881F8E7486A104348624B71F3E770B575
:10897000154613F0070F0FD12A49264C09682079B4
:10898000C861A08CC0F307217F20F7F75DFD94F844
:1089900024002946F7F758FD002070BD70B5044645
:1089A00003F007000D4602281CBF002070BD1948C7
:1089B000818C007989B2F7F7FBFC207001202870C8
:1089C00070BD03F007011348012904BF0021C181D4
:1089D00003D013F0070F08BF827200207047F8B56C
:1089E00003F0070200230E4E0A4F012A02D0022A8A
:1089F0002FD02CE00024022000937871FB81B87AFC
:108A00004FF44835834222DA042269462846F9F7B2
:108A100057FB09E0EC050020A005002032050020EE
:108A200090901100649011003168009808553168E9
:108A300000982144000A48700098000C8870009843
:108A4000000EC870B87A241D2D1D8442DCDB002086
:108A5000F8BD7A79022A15D1FA8997F80AC06245D9
:108A600007D2D6F800C01CF802C080F800C0501C25
:108A7000F881F889BA7A904204D1FB81012008700C
:108A8000032078710120F8BD10B503F00700FC4900
:108A9000012804BF0020C88118D013F0070F15D19A
:108AA000C88991F80AC0F74B604505D2D3F800C0D9
:108AB0000CF80020401CC8818A7A80B2904205D10F
:108AC0008A7A4FF448301968F9F7F6FE002010BD95
:108AD00070B54FF444324FF4407101FB0024012083
:108AE000F8F7C1F8FDF726FBFCF778F90546F8F72B
:108AF0007AFBE34B4FF4107220461C639A8229469E
:108B0000BDE87040F9F7D8BE70B513F0070F18D163
:108B10004FF444314FF4407000FB02140120F8F789
:108B2000A2F8FDF707FBFCF759F90546F8F75BFBE0
:108B3000D34B4FF4107220461C639A822946F9F7F2
:108B4000BBFE002070BD13F0070F04BFCC4842727B
:108B500000207047F8B503F007020027C94EDFF880
:108B600020C3012A02D0022A2DD02AE09CF8090055
:108B7000002400EB40004FF4443101EB00250220BB
:108B800000978CF80500ACF80E704FF41070ACF83C
:108B90001400042269462846F9F792FA31680098D1
:108BA0002D1D0855316800982144000A487000982E
:108BB000241D000C88700098000EC870B4F5107F5A
:108BC000E7DB0020F8BD9CF80520022A16D1BCF88E
:108BD0000E20BCF814309A4205D23468A45C0470AC
:108BE000501CACF80E00BCF80E00984206D1ACF850
:108BF0000E700120087003208CF805000120F8BDDC
:108C000003F00701DFF878C20098012907D013F0BC
:108C1000070F04BF9CF80510022909D01FE00220AD
:108C20008CF805000020ACF80E00CCF82C0016E003
:108C3000BCF80E10814208D2DCF82C30491C42EA04
:108C40000322CCF82C20ACF80E1089B2814206D158
:108C5000BCF82C00ACF8140003208CF805000020B0
:108C6000704770B503F007000025854C0E460128BB
:108C700006D013F0070F04BF6079022805D023E067
:108C800002206071E581E5621EE0E089A18A8842E8
:108C900011D2E16A090A41EA0261401CE162E08105
:108CA00010F0030F07D104227749206BF9F704FE77
:108CB000206B001D2063E089A18A884204D1E581F0
:108CC0000120307003206071002070BDF8B503F002
:108CD000070200256A4C0E460746012A02D0022AE6
:108CE00005D002E002206071E5810020F8BD6079C6
:108CF000022822D1E289A08A824215D212F0030F03
:108D000009D104226946206BF9F7DAF90098E0628C
:108D1000206B001D206394F82C003870E06A000A74
:108D2000E062E089401CE081E089A18A884204D1A8
:108D3000E58101203070032060710120F8BD70B41E
:108D400003F0070200254E4C012A02D0022A06D069
:108D500002E002206071E58170BC002070476279FA
:108D6000022A1CD1E289B4F814C062450FD212F075
:108D7000030F04D1236B53F8046BC4E90B6394F81D
:108D80002C300370E06A000AE062501CE081E08948
:108D9000604504D1E581012008700320607170BC3A
:108DA0000120704730B403F007000024DFF8D0C082
:108DB000012807D013F0070F04BF9CF80500022814
:108DC00008D025E002208CF80500ACF80E40CCF865
:108DD0002C401DE0BCF80E00BCF8143098420CD2B8
:108DE000DCF82C502D0A45EA0262401CCCF82C20FD
:108DF000ACF80E0010F0030F0DD0BCF80E00984236
:108E000006D1ACF80E400120087003208CF8050054
:108E100030BC00207047DCF83000B0F5002F28BFD0
:108E20000260001DCCF83000E7E730B403F007041F
:108E30000025DFF84CC0012C08BFACF80E503ED026
:108E400013F0070F02D0022C3CD038E0042A08BFF0
:108E50004FF42C3031D01DDC002A08BF4FF48010B5
:108E60002BD0012A08BF094827D0022A08BF4FF497
:108E70008E1022D0032A08BF05481ED01AE0000039
:108E8000EC050020909011001806002000FE110053
:108E900000F81100052A08BFF8480ED0F848102A3B
:108EA00000680AD0112A08BFF64806D0202A08BF59
:108EB000B43002D0CCF8285001E0CCF8280030BC07
:108EC00000207047BCF80E20042A07D2C2F1030329
:108ED000DCF82840DB0024FA03F30370501C80B256
:108EE000ACF80E00042824BF01200870012030BC1B
:108EF000704710B503F00700012804D10022114685
:108F00000C2000F0D8F9002010BD2DE9F04103F04D
:108F1000070CDD4E069D0F460446BCF1010F04BF51
:108F20000020F08117D0D84913F0070FCB8903D068
:108F3000BCF1020F12D00EE0D449022B3CBF0868EE
:108F4000C254581C80B2F081A84204D102220968A0
:108F5000052000F0B0F90020BDE8F08113B1012B2D
:108F600004D008E0FBF7DCFD207004E0FBF7DBFD3C
:108F7000207001203870F089401CF0810120BDE88C
:108F8000F08170B503F00700BF4D012803D013F046
:108F9000070F05D024E00020A862E862A8711EE057
:108FA000B949EC8991F806C0886A0CEB0201CBB292
:108FB000022C03D242EA0020A86206E0B249042C47
:108FC000C96A04D242EA0120E862AB7105E0052CCF
:108FD00003D2624508BF00F057FFE889401CE881D2
:108FE000002070BD10B503F007011046012905D01F
:108FF00013F0070F08BF00F01BF904E0A24900209E
:1090000088628871C881002010BD10B5104613F029
:10901000070F08BF00F00CF9002010BD70B5032643
:1090200000244FF48E1505EB0430F9F7C7F9022838
:1090300008BF70BD601CC4B2B442F4D3012070BD3F
:1090400030B403F007030024DFF83CC2029A012B7E
:1090500002D0022B0CD008E005208CF80500ACF8FB
:109060000E409CF808008CF8060030BC00207047C9
:109070009CF80530052B14D1BCF80E30934205D274
:109080009CF806500570581CACF80E00BCF80E0099
:10909000904206D1ACF80E400120087003208CF8F5
:1090A000050030BC012070472DE9F04778A0DDF8BD
:1090B00020C0006803F007050027734E734C012D94
:1090C00003D013F0070F06D034E0F7812068077053
:1090D000206847702EE0F389634503D22568EA547F
:1090E0005A1CF281F289624524D1F7814FF00108C0
:1090F00081F800802168C2B2097891421AD12168B2
:10910000C0F307204978814214D1032500244FF48D
:109110008E1909EB0430F9F751F9022804D0601CCC
:10912000C4B2AC42F5D34046012806BF86F8088099
:10913000F77137720020BDE8F0872DE9F0414FF05C
:10914000000C03F00700534E4F4C6546012803D036
:1091500013F0070F0CD068E06570A5812562A5703B
:10916000002046F82050401CC0B24028F9D35CE0F3
:10917000607805283CBF401C6070C0B2012808BF61
:10918000100222D040490228CB8A08BF98181CD070
:1091900024BFA1898B4248D93F4F01F0030001F160
:1091A00001083A54A7F134004FF48E12006A984532
:1091B00002EB002008BF002109D1491CC9B20429D3
:1091C000FBD33449F9F79BF926E0E0822DE0032236
:1091D00032EA010120D17A5CCB009A40491CC9B225
:1091E00042EA0C0C0429F6D3A17801F03F02491C95
:1091F000C9B246F822C0A17040290DD12549F9F71E
:109200007EF9A570206A401C2062002046F820509C
:10921000401CC0B24028F9D3A089401C80B2A08174
:10922000E18A884204BF0120E0710020BDE8F0819E
:1092300010B5154C2146E2898B6A8979022A05D23C
:1092400040EA03220844A262A07112E0B2F5817FD5
:1092500008D20E490968114401F8020CA1790844AA
:10926000A07106E008BF884203D10A49184600F001
:1092700025FEE089401CE08110BD000000F01100D7
:10928000E8060020F80F0020EC0500209090110067
:1092900055AC00001438002020060020DC480021D6
:1092A00001704170C1700171DA4A08461154401CC6
:1092B0000428FBD3704710B4D54C6378002B1EBF35
:1092C000002010BC7047E07022710020002A88BF87
:1092D000D04B06D911F800C003F800C0401C8242F0
:1092E000F8D80120607010BC7047C94840787047BA
:1092F000C74880787047C64900208870704770B5AD
:109300000024FAF786FAC24D6878012806D100F0E9
:1093100012F804461E20E87000206870FBF700FC7D
:10932000022802D101F068FD18B9002C04BF00200A
:1093300070BD012070BD2DE9F05FB5480024C078F4
:109340001E2880F06281DFE800F0121E2C350F41EC
:10935000FD4597A0A6ABE4FCB9C7CCD197979797EA
:10936000979797979797FBFAFBF739FC16E0FBF76F
:10937000D7FBA74C6071A01D01780120FBF7E2FB31
:109380000120A0700AE0A348007801F083FF0121CA
:109390000320FBF7D7FB9E4901208870012400F0D1
:1093A00034B99C484178007841EA002003F0CCFAB7
:1093B00000F02BB99748007803F0CBFA0421032082
:1093C000FBF7C0FB924901208870E7E7914841789C
:1093D00000789BE0DFF8388200264FF0010A08F1A0
:1093E000060BB146012788F802A088F8019098F88A
:1093F0000000D0BB9BF8005088F800A015F0100FBB
:1094000011D00120F7F72FFCFBF78DFBA8B3F8F77D
:10941000AFF8FF210F20FBF70CFF074645F00105D1
:109420000020F7F77AFC15F0010F1CD0FAF72CFB9F
:109430000020FAF798FD0120F7F715FCFAF783FCF6
:1094400001460220FBF776FD0220FBF751FDF7F7FE
:10945000CAFEFAF778FCFAF770FDFAF774FC4FF4DD
:1094600090610EF0D8FA88F8009088F80290002FEA
:109470001CBF761C032EB5DBC7E0FFE7F8F778F8D2
:10948000FF210F20FBF771FFC7E762480078401EFD
:1094900001F018FC82E75F48007803F0DFFB7DE70E
:1094A0005C480078002804BF0021032003D003F0AB
:1094B000ACFB01460220FBF745FBA6E0554D2878A2
:1094C000002818BF012003F081FB2878002818BF6E
:1094D000012000F011FD98E04E48007803F067FB92
:1094E0005CE74C48007803F0CCFB8EE049480078FC
:1094F00020B1012856D0022804D086E04648F8F76B
:10950000E5FE82E001F0F9FC00210420FBF71AFBE4
:1095100044E73F484FF0000880F801804646454642
:1095200072B6F9F775FF48B1FAF730F80646FAF760
:109530000DF8FAF731F80546FAF718F803E060E09D
:1095400055E043E02FE0F7F75DFDF7F779FB814643
:10955000F7F717FFF9F792FE070018BFF9F78DFE2E
:109560004FF41870F9F765FE62B62C48C0F8008019
:10957000F8F76AFB72B6B9F1000F03D0F7F742FDB6
:10958000F7F731FEF9F744FF38B1002E18BFF9F7AD
:1095900041FF002D18BFF9F77CFF002F18BFF9F726
:1095A0006AFE62B631E01B480078012804BF022140
:1095B0000520ABD0022804BF00210320A6D0032839
:1095C00019BF02210846002104209FE711480178B5
:1095D000427841EA02218278C078120442EA0060AF
:1095E00041EA00026221072002F015FF0DE0F8F7C2
:1095F000C0FC0120F7F737FBFAF7C3FDF7F7F3FDDF
:10960000CCE60448007800F0F2F82046BDE8F09F70
:10961000240600202A06002000FE11006405002018
:1096200002460020022928BF704752B1012A18BF04
:10963000704701EB810000EBC100FE4901EB001017
:10964000704701EB410000EBC100FB4901EBC0108A
:10965000704700FB01F2B2F5307F9CBFF74AC2E9C8
:10966000020170470028F54A926818BF0260F3486B
:109670000029C06818BF086050437047EF480121B7
:109680000171007880F0010000EB400101EBC000A7
:10969000E94901EBC0107047E8488278002132B1F7
:1096A000C27822B9027882F00102027081700171E1
:1096B0007047E24910B54C7848701E2808BF00205A
:1096C00008D01F2808BF012004D00E2808BF812021
:1096D00002D000E00870012003F0D3FA204610BD4C
:1096E000F0B4D64E96F800C0B5680CEB4C0404EB11
:1096F000CC0CD14C8D4204EBCC1C03FB05F40CEBE1
:10970000440C34BF2C460C46F768FE1A964228BF1C
:1097100016461A44974224BF0023002E9CBFF0BC7B
:1097200070470022002C06D930F812702CF8127005
:10973000521C9442F8D85B1C0CEB450C00EB41002A
:10974000B342EED3F0BC70472DE9F041BB4F144655
:109750008C4601467A7806981D468A4218BFBDE8B5
:10976000F0810121F970012802D0022825D02AE0D9
:109770003878BE6800EB400101EBC000AE49A6425C
:1097800001EBC01134BF32462246F868A84238BF08
:1097900005460023002D16D90020002A06D91CF802
:1097A000007021F81070401C8242F8D85B1C01EB5D
:1097B0004601A444AB42EFD305E000232A462146EC
:1097C0006046FFF78DFFBDE8F04100F0EBB910B542
:1097D000002808BF10BD01229849CA7049780023AB
:1097E0000821FFF77DFFBDE8104000F0DBB9934A88
:1097F00001281146D071497808D000280CBF2429CF
:10980000704730205070012003F03BBA2420507084
:10981000012003F036BA8948C079704770B4DFF888
:1098200020C2DCF800C0DCF818C01CF0040F1ABF1E
:10983000012424EA0C060CF0010605680C68002ED1
:109840001CBF1B1B5C1E1CF0020F1CBF521B551EB5
:109850001CF0040F19BF04600D6005600C6070BC43
:10986000704710B5002808BF10BD01227349CA70A7
:109870004A787449DFF8D0C102220B789CF80010B6
:10988000FFF72EFFBDE8104000F08CB92DE9F04342
:109890006A498BB00122CA706C4A49781578694AC6
:1098A0002529147824BF0BB0BDE8F083DFE801F070
:1098B000134D4D4D134D4D4D4D4D4D4D4D4D4DFD9C
:1098C0004D555555FDFDFDFDFDFDFDFDFD4DFDFD20
:1098D000FD7D7DFD8500002800F002810646002701
:1098E000F7F75EFD5FEA000C16D0544908788F68E0
:1098F00000EB400202EBC0004F4ABD4202EBC01039
:1099000094BF2B463B46C968A14238BF0C46002194
:10991000002C06D800F0E4B83B46224629463046E3
:1099200048E00022002B08D91CF9028036F8188084
:1099300020F81280521C9342F6D8491C00EB4700D5
:1099400006EB4506A142ECD3CAE0002870D0002304
:1099500022462946FFF7C4FEC2E03D4800780128B0
:1099600084BF3C480478F7F7CDFB10F0020F18BF16
:10997000641CFBF733FA002205FB04F3002BC4BF81
:10998000DFF8B8C02C4C53DD10F8015B9CF80010D8
:1099900001EB410606EBC10104EBC11121F81250A5
:1099A000511C8AB29342EFDC9AE0002840D0002399
:1099B000A21C2946FFF794FE92E0002838D0064604
:1099C0001F480068007E10F0040F0EBFA946A14694
:1099D0002C464FEA9902A1080591A9EB990006913E
:1099E00000924FEA5901401ECDE90101610807913B
:1099F000A4EB9401491E08910991CDE90320234667
:109A00004A4605A96846FFF709FF23464A4605AFBF
:109A100006A9E84601A8FFF701FF23464A4607F1D9
:109A2000080108F10800FFF7F9FE23464A4613E053
:109A300056E0000014470020143C002030060020AF
:109A4000E8060020BF050020C5050020BE05002057
:109A5000C0050020C205002007F10C0108F10C0030
:109A6000FFF7DCFE23464A4607F1100108F110001B
:109A7000FFF7D4FE58480078002200EB400101EBCC
:109A8000C0005649914601EBC01020F8129058F8DA
:109A90002210A1F1010C491C61451ED357F8221078
:109AA0004B1E491C994211D300E01EE003FB05C187
:109AB00036F9114030F912108C42C8BF20F812401C
:109AC00057F822105B1C491C9942EDD258F822101D
:109AD0000CF1010C491C6145E0D2521C052AD4D37B
:109AE0000BB0BDE8F04300F05DB80BB0BDE8F0830B
:109AF00039491E288A79887108BF002003D01F28A1
:109B000008BF012000D148711046704770B50D465E
:109B100031490122CA70324A49781678314A2129DE
:109B200014781EBF2229232970BD002818BF002DDC
:109B300011D0002322463146FFF7D2FD631C0122DB
:109B400021462846FFF7CCFD05EB4400A31C01226B
:109B50003146FFF7C5FDBDE8704000F023B810B5F1
:109B60001D4C6178002904BF4068FFF78FFE6078C4
:109B7000112804BF0020FFF789FE6078122804BF77
:109B80000020FFF783FE6078132803D1FCF792FBD7
:109B9000FFF77CFE60781D2818BF10BD1248BDE895
:109BA000104073E670B5F9F740FB00F00806082096
:109BB000F9F736FB084C20790025002801BF2078F2
:109BC00080F001002070A5701CBF0120A0703046FD
:109BD000F9F722FBE57070BD30060020143C002030
:109BE000BE050020BF05002080680020A349002892
:109BF00014BF0020012008707047A048007800289A
:109C00000CBF01200020704710B59C4C2078002824
:109C10001CBF0120F9F772F800206060A060E060CE
:109C20002061606110BD10B5944C207800281CBFE5
:109C30000120F9F763F800206060A060E060206117
:109C4000606110BD70B50446F9F7EFFA00F0080541
:109C50000820F9F7E5FA894A89490023106901EBE0
:109C6000C001401C1061B0F5807F28BF13612078CF
:109C7000087060784870A0788870E078C8702079A3
:109C8000087160794871A0798871E079C87150696C
:109C9000B0F5807F3CBF401C506116D31D2008707A
:109CA00001204870207888706078C870A0780871AA
:109CB000E0784871207988716079C871D068401C5B
:109CC000D060B0F5807F28BFD360506840F00100BD
:109CD0005060107800281CBF0120F9F71AF82846B8
:109CE000F9F79AFA012070BD10B50178022211F03F
:109CF00003011CBF0129022902D1FFF7A3FF02467D
:109D0000104610BD2DE9F0415C4E044630467268A5
:109D100003780025002A1CBF00204FF0010C54D00E
:109D2000B1680CFA01F7174207D1491CB1600D293F
:109D300028BFB560401C0D28F2D3B16809B3514863
:109D400000EBC1000CFA01F122EA01010838716050
:109D5000317D02782270427862708278A270C27877
:109D6000E27002792271427962718279A271C079BE
:109D700001F03F0100F0C0000843E0717068D8B9FD
:109D800015E0716909B33E48D6F80CC000EBCC0071
:109D90000CF1010CC6F80CC0BCF5807F28BFF56043
:109DA000491E716104BF22F001017160D0E7002BF0
:109DB0001CBF0120F8F7A2FFB068401CB0600D285E
:109DC00028BFB5600120BDE8F081002B1CBF012039
:109DD000F8F794FF25706570A570E57025716571C1
:109DE000A571E5710220BDE8F081244910B44A68EC
:109DF00000204C69002A19BF01210B4610BC704796
:109E000003FA01FC1CEA020F18BF401C491C0D2973
:109E1000F6D312F0010F18BF204410BC704700B5F4
:109E20000178427883B0890102F0070241EA820199
:109E30008DF80010418809098DF801108188090901
:109E40008DF80210817801F00F02017962F31F1181
:109E50008DF80310017A8DF80410417A8DF8051001
:109E6000807900F03F008DF8060000208DF8070093
:109E70006846FFF7E7FE03B000BD00004006002083
:109E800014490020B448002070B50E4680280CD23A
:109E90008119491E802908D205030024002E04D907
:109EA0002846F8F78BFA012801D0002070BD641C09
:109EB00005F58055B442F3D3012070BDB0F5006FB5
:109EC00024BF0020704710B50002F8F718FB0128E6
:109ED00018BF002010BD10B5064CFFF710FA01287E
:109EE00008BF10BD206801F0D3F8002818BFFAF7AA
:109EF00051FEF2E7E8060020FC4A0028516814BF32
:109F000041F0010021F0010050607047F74B5968A3
:109F10000A0E120721F07F4142EA006008435860B0
:109F20007047F2484068C0F30360704770B5EF4D6A
:109F3000AA68521CAA604FF0000C0028C8BFC5F8E0
:109F40000CC00ED06A6812F0010F40D0E84BC2F38B
:109F5000036214001B6808D0022A18BF002413D023
:109F600028E0EA68521CEA60ECE70028C8BF022437
:109F700022DC93F81601A96888421BD8022401202C
:109F8000C5F808C0286117E0002918BF0A2402D0CC
:109F900004F06BFF10E068B9B3F81201E968884279
:109FA00038BF0024F4D32869012804BF0024C5F871
:109FB00010C001D094420AD06868010E090720F051
:109FC0007F4041EA046108436860012070BD0020C1
:109FD00070BD2DE9F041C54D04460026E8693746BD
:109FE000012806D16068F9F7B2FE286A032808BF85
:109FF000EF616068B0B103F005FA0028C8BF012620
:10A000000FDC2888401C2880B9480068017F11F0C7
:10A01000010F07D0807F2988814203D96068F9F752
:10A0200096FE2F803046BDE8F04100217EE72DE905
:10A03000F04F06468DB00020AC4F059000247868A4
:10A04000A046C0F303654FF0FF308246049070686D
:10A050000DF11809A346D8B1CDE902BACDF800B088
:10A0600000234A4604A9CDF804B000F0C3FB8046A3
:10A0700000F0BAFB04469F480078012804BF204640
:10A08000FFF704FC04980028C8BFA7F800B002DC62
:10A090003888401C388096480068017F11F0010F15
:10A0A00015D0B0F814013988814202D838690128E6
:10A0B0000DD15B46A7F800B0CDE900B4CDF808B0EB
:10A0C00042465146CDF80CB00498FAF7FDFC84B135
:10A0D000022D04D0042D04BF0498012809D1306852
:10A0E000CDE90004CDF80C906846049904F0C5FE53
:10A0F00005900498012818BF00200599FFF716FF66
:10A100000DB0BDE8F08F7C4801680969006841F036
:10A1100001010161794801684969026841F40071EF
:10A12000516101680969026841F004011161016827
:10A130000969006841F0100101617148016809680E
:10A14000006841F0010101606E4800780022674913
:10A1500000281CBF4A8070474888B0F57A7F87BFC7
:10A160004A8030BF401C488070472DE9F04F87B0CF
:10A1700004460025052700F0D3FE002804BF07B0E1
:10A18000BDE8F08FFAF7CCFC8146FAF7CCFC8046AC
:10A190000F212046FAF790FD002804BF07B0BDE864
:10A1A000F08F0420DFF860A1DAF800108860DAF898
:10A1B0000010486002212020F7F716F90020F6F77A
:10A1C000ACFD524C2068406C216840F4006048644B
:10A1D000012002F0C8FB2068406C216820F4006078
:10A1E0004864F7F700F8DAF800000068DAF80010C1
:10A1F00040F00100086030BF3C4C01200026266280
:10A20000E061DFF8ECB0FFF77AF8012844D0FAF704
:10A2100087FC484540D1FAF786FC40453CD168466A
:10A22000F7F7B1FA002833D0206A401C2062684654
:10A23000FFF795FCE0690025012806D10198F9F7A0
:10A2400086FD206A032808BFE6610198B0B103F0DB
:10A25000D9F80028C8BF01250FDC2088401C2080C9
:10A26000DBF80000017F11F0010F07D0807F21880B
:10A27000814203D90198F9F76AFD2680002128461A
:10A28000FFF754FE0546F7F7A9FAFAF799FC01E043
:10A29000FAF775FC002DB6D0DAF800000068DAF89D
:10A2A000001020F0010008600020F7F70FF8F6F723
:10A2B000F3F9FAF735FC052805D0FAF731FC074623
:10A2C0000520FAF73CFCFAF77AFD052F1CBF38464B
:10A2D000FAF735FCFBF7A3FE0D4801780D4800782E
:10A2E000F7F782F807B0BDE8F08F000058060020AD
:10A2F000E806002031060020609011004C9011000B
:10A3000080901100340600206890110064901100C4
:10A31000BF050020BE0500202DE9F04F87B0F6F7FD
:10A320005FFEF9F705F85C4D0124A86910B9F7F74D
:10A3300086FDAC61DFF864A1DAF80000B0F90E1117
:10A34000B0F90C0100F002FA04F08BFD6C61FAF731
:10A35000E7FB052804BF4FF0000B514F26D1DAF878
:10A3600000006A68C2F30361D0F8F8008B00D8409F
:10A3700000F00F00C5F808B0C5F80CB0002970D087
:10A38000022918D004296DD00A2922F07F404FEA13
:10A39000017118BF41F0007108436860FEF7AFFF1C
:10A3A000012803D0FAF7BCFB0528D8D007B0BDE8D8
:10A3B000F04F04F058BD064600244FF00508FAF7A8
:10A3C000B2FB81460F213046FAF776FC0028E5D033
:10A3D00000F0F7FB39687020886039680220486017
:10A3E000304E3068406C316840F4006048640120B1
:10A3F00002F0B9FA3068406C316820F400604864BB
:10A40000F6F7F1FE38680068396840F0010008602E
:10A4100030BFFEF774FF012806D06868C0F3036000
:10A42000484508BF002C1ED000F0CBFBFAF778FBA4
:10A43000052805D0FAF774FB80460520FAF77FFB64
:10A44000FAF7BDFCB8F1050F1CBF4046FAF777FBE1
:10A4500038680068396820F001000860FBF7A8FD43
:10A460009CE713E015E06846F7F78DF958B16846A8
:10A47000FFF775FB6846FFF7DAFD0446F7F7AEF91C
:10A48000FAF79EFBC5E7FAF77AFBC2E7FFF76DFE26
:10A4900084E702F066FF81E758060020E806002006
:10A4A0006890110064901100F0B4FF4EDDE905C41E
:10A4B0003668049DB66916F0010F04D01F464B1B89
:10A4C000CD1BDBB2EDB216F0020F06D06746A2EB51
:10A4D000040CD21B0CF0FF0CD4B216F0040F08D001
:10A4E00080F800C04A1B84704270C91AC170F0BC69
:10A4F00070470370857080F801C0C470F0BC70476D
:10A500002DE9F043164601FB06F90D46014685B0DC
:10A510001F464A46E5480DF0FFF9E44C02F00BFCFB
:10A520004FF0000818B104F056F801281AD002F0D4
:10A5300002FC18B104F04FF8082842D0B7F5805F4C
:10A540001CBF0020B9F1000FDCBF05B0BDE8F083EF
:10A550002156794309132154401C8145F8DC05B08C
:10A56000BDE8F08300210B46002ECEBFDFF838C3D4
:10A5700005B0BDE8F0830020002D1CDDDCF80020D4
:10A5800092F83E919945DCBF92F83F914B450CDC27
:10A5900092F83C918145DCBF92F83D21904204DC69
:10A5A00062567A431213625401E004F80180401CA1
:10A5B000491CA842E2DB5B1CB342DCDB05B0BDE812
:10A5C000F083AE428CBF701E681EC2B2B54234BF6B
:10A5D000681E701EC1B20420CDE90002002303A84A
:10A5E0000292FFF761FF00210A46002EDCBF05B092
:10A5F000BDE8F0830020002D19DD9DF80D30934259
:10A60000DCBF9DF80F309A4209DC9DF80C30834284
:10A61000DEBF9DF80E30984204F8018003DD6356DA
:10A620007B431B136354401C491CA842E5DB521CAE
:10A63000B242DFDB05B0BDE8F0832DE9F0411C46F6
:10A6400015460E460746F8F7E5FB21462846F8F77B
:10A6500000FC0623954A31463846F8F710FDBDE860
:10A66000F041F8F7D8BB924A5060916070472DE9ED
:10A67000F00F0024DDE90875B7F5805F08BF642D91
:10A680002AD00026002B87BFA5F16409C5F1640814
:10A69000BDE8F00F70470020002A17D9B0FBF2FA8E
:10A6A00031F914C0642D0CFB07FC4FEA2C3C27BF8A
:10A6B0000AFB09FA0CFB0ACC0AFB08FA0CFB1ACCC1
:10A6C00021F814C0401C641C9042E7D3761C9E42C3
:10A6D000E1D3BDE8F00F7047884204BFBDE8F00F3A
:10A6E00070475A43BDE8F00F52000DF015B92DE93F
:10A6F000F04180466C4882B00F4600681D46164601
:10A7000090F84C10ADF8001090F84D10ADF8021014
:10A71000B0F84A10ADF80410B0F848000024ADF8C5
:10A720000600F8F777FB6846F8F768FC29463046DC
:10A73000F8F786FB39464046F8F772FCF8F76BFBF2
:10A740005B48C46002B02046BDE8F08158490880EB
:10A7500070472DE9F041574E8AB005465448CDE97F
:10A760000056A6F148080C46CDF80880B0F9001054
:10A7700003913F29C8BF3F2005DC11F1400FB8BF4E
:10A780006FF03F0000DA039000200490F8F742FBDE
:10A7900049484A4F01783878F8F752FB6846F8F78D
:10A7A000E6FB0890F8F737FBC4E90068BDF8140031
:10A7B0002081BDF816006081BDF81800A081BDF8A9
:10A7C0001A00E081BDF81C002082BDF81E006082E6
:10A7D000BDF81C00BDF81E103A7801FB020035F9E7
:10A7E00010000AB0BDE8F081314800697047304878
:10A7F000406970472DE9FF4FADF2A44D00208A4615
:10A80000CDF89C04ADF88C048346471E9146DDF8D4
:10A81000E0844FF4906102A80DF01FF9B8F1000F29
:10A8200018BF98F800B02548254E057822480478CE
:10A830001D480068008ECDF8940406F59060CDF8B0
:10A840009804DDF8A404CDF89004FAF769F9022819
:10A850001ED1FAF768F902281AD1F9F780F90190A8
:10A86000B0B1DDF8A4242B46009410460199F9F705
:10A8700051F914480078022804BF0198FFF706F840
:10A8800010480078092804BFDDF8A404FEF7FEFF95
:10A89000DDF89004CDF8880405480661F9F753FA0D
:10A8A000CDE900402B460FE0E806002014510020BF
:10A8B0007C0600209C530020BF050020BE05002020
:10A8C0001C54002031060020024602A8DDF888143E
:10A8D000F9F720F9BC480078032804BF0198FEF777
:10A8E000D5FFB9480078052804BF02A8FEF7CEFFBF
:10A8F000B5480078062804BF02A8FEF7C7FF02A8E3
:10A90000CDF88804B0480078222803D1002102A89D
:10A91000FFF7FCF8DDF8940410F0010F15D0DDF816
:10A9200088040090F8F776FA21462846F8F791FA5D
:10A930000623A64A30460099F8F7A1FBF8F76BFA10
:10A94000A1480078082810D012E064214FF480500C
:10A95000CDE9000123462A463046DDF88814FFF78A
:10A9600086FE99480078082802D13046FEF78EFF0F
:10A97000DDF8940410F0060F31D002F0A9F870BB96
:10A980000020CDF894049248006890F84C10ADF87F
:10A99000001090F84D10ADF80210B0F84A10ADF864
:10A9A0000410B0F84800ADF80600F8F733FA68462E
:10A9B000F8F724FB21462846F8F742FA31460846C4
:10A9C000F8F72EFBF8F727FA8249DDF89404C860FF
:10A9D0007D4800780A2804BF3046FEF757FFBAF1D9
:10A9E000000F1FD0B9F1000F25D0DDF89C040090B6
:10A9F0000DF28C433046DDF88824DDF89814F9F721
:10AA000017FD0746680000FB04F23046DDF88814A5
:10AA10000CF082FFB7F1FF3F12BF002F0020ADF80E
:10AA20008C0402E0B9F1000F05D049463046FFF72B
:10AA300090FEA9F8140064480078072804BF304647
:10AA4000FEF724FFBAF1000F18BFCAF80070DDF856
:10AA5000D80400281CBFBDF88C140180B8F1000F89
:10AA600018BF88F800B0DDF890040DF2B44DBDE8D1
:10AA7000F08F594870472DE9F05F814657481746D7
:10AA800088460078544C4600F9F765FADFF838B18B
:10AA9000824600259BF80000042804BF4846FEF7C4
:10AAA000E0FE9BF80000052804BF4846FEF7D9FEEB
:10AAB0009BF80000032804BF5046FEF7D2FE9BF827
:10AAC0000000232804BF4846FEF7CBFE0020002EDE
:10AAD00009D939F810103AF81020891A24F8101002
:10AAE000401C8642F5D89BF80000062804BF20468B
:10AAF000FEF7B7FE9BF80000222804BF2046FEF7B1
:10AB0000B0FE0020711E18BF0A4612D004EB4001AF
:10AB100034F810304988C91A09B224F810100029F5
:10AB2000B8BF494209B2A942C8BF0D46401C904275
:10AB3000ECD304EB460020F8025C9BF800000A28E6
:10AB400004BF2046FEF78DFE9BF80000082804BFD6
:10AB50002046FEF786FE9BF80000072804BF20462B
:10AB6000FEF77FFE9BF80000012804BF2046FEF799
:10AB700078FE9BF800000E2804BF2046FEF771FE09
:10AB80009BF80000212804BF2046FEF76AFEB8F1BA
:10AB9000000F10D00E494FF0FF300968B1F9722054
:10ABA000AA42B8BF012004DBB1F970108D42B8BFD2
:10ABB0000020C8F80000002F18BF3D804846BDE8BF
:10ABC000F09F7047704700003106002014510020AC
:10ABD000E80600207C0600201C5D0020C505002042
:10ABE00008283CBF9C490870704700209A49C860FB
:10ABF0009A48006890F88100082838BF08707047AC
:10AC000095480078704710B50446F6F7E9F9944A7C
:10AC100003211268D161052C4ED2DFE804F0031243
:10AC200021303F0001217F20F5F70EFC8C214FF4ED
:10AC30008470F5F709FC5C214FF48570F5F704FC8E
:10AC40003AE001217F20F5F7FFFB87214FF4847064
:10AC5000F5F7FAFB59214FF48570F5F7F5FB2BE07A
:10AC600001217F20F5F7F0FB75214FF48470F5F793
:10AC7000EBFB4D214FF48570F5F7E6FB1CE001215D
:10AC80007F20F5F7E1FB67214FF48470F5F7DCFBDB
:10AC900043214FF48570F5F7D7FB0DE001217F20AC
:10ACA000F5F7D2FB58214FF48470F5F7CDFB3A212C
:10ACB0004FF48570F5F7C8FBF9F710F8F6F793FA3B
:10ACC000012010BD01207047644863490068B0F856
:10ACD00076004242C8688242BCBF401EC8607047CE
:10ACE0002DE9F04FA1B09346884604464FF0000985
:10ACF00001F0AFFF594E8246574D3068B0F96E00F3
:10AD0000A0420DDAA868401EA86009D26420A8609D
:10AD1000686803280CBF0020401C6860FFF773FFC1
:10AD2000504F3878072829D14F485946007882007B
:10AD300068460CF0F1FDADF80040ADF80280ADF8CA
:10AD400004A0A889ADF80600A888ADF8080030680E
:10AD5000B0F87210ADF80A10B0F87410ADF80C101D
:10AD6000B0F86E10ADF80E10B0F87600ADF8100027
:10AD70003878072804BF6846FEF773FD484621B0BF
:10AD8000BDE8F08F34488078002818BF0120704754
:10AD90000020DFF8C4C09CF80210002914BF012273
:10ADA00000229CF80110002918BF01218A4208BF27
:10ADB00070470A1C18BF012210B48CF80220274AE1
:10ADC0001368D3F8A42012F0040F0FD021B1C2F3FE
:10ADD0000310082809D206E00020CCF80C0093F8F4
:10ADE0008100082801D28CF80000012012F0020F27
:10ADF00018BF012010BC70472DE9F041174F002605
:10AE00003868D0F8A40010F4807F21D0124D697802
:10AE10000C1C18BF0124C0F30330012101FA00F01B
:10AE2000F7F7A1FF3968B1F8A41011F4007F01D041
:10AE300028B103E0002818BF002000D1012084427F
:10AE400006D0002818BF01206870FFF7A1FF064652
:10AE50003046BDE8F081000094060020E80600209E
:10AE60006490110031060020C5050020714800687B
:10AE700000F5407070476F48006800F580707047BB
:10AE800070B56C4C6C4922681068884204BF5068E9
:10AE9000B0F5087F24D1D2F808C0BCF5405F1FD8B8
:10AEA0006649D06888420DD0002311461846B3EB9E
:10AEB0009C0F07D251F8045B401C6B40B0EB9C0F19
:10AEC000F8D36BB902F5807000F0E2F840B1206869
:10AED00000F5407000F0EBF800281CBF012070BDA9
:10AEE000002070BD534910B54FF48E100860FFF775
:10AEF000C7FF002818BF012010BD4FF48E10F7F7D0
:10AF0000E5B94C484C4A00680168914206BF416867
:10AF1000B1F5087F00207047464800680069704717
:10AF2000444909680A6982429CBF00207047C0EB0F
:10AF3000C00001EBC00000F5806070473D4A126818
:10AF400002EB80035B6A1A443D4B53F82000FF304C
:10AF500020F0FF0000FB012070472DE9F0010022E6
:10AF6000344D17462E1D831893F92840002CB8BF86
:10AF700041F8227010DBD5F800C0D3B20CEB830887
:10AF800056F82330D8F82480FF33C44423F0FF035D
:10AF900003FB04C341F82230521C102AE3D3BDE85E
:10AFA000F00170472DE9F0410025174604460029BD
:10AFB000B8BFBDE8F081042C02D0052C10D014E0FD
:10AFC000F9F7AEFD052810D1FEF7ABFF022808BF48
:10AFD00003250AD0FEF7A5FF002808BF022504E0DC
:10AFE000F9F79EFD052808BF01251248144E006898
:10AFF00056F8241000EB8400FF31406A21F0FF0175
:10B0000000F5E030503005FB0105F9F789FD022815
:10B0100008D101F0F5FD28B956F82400FF3020F0E2
:10B02000FF00054456F8242039462846BDE8F04183
:10B03000F7F742BCA406002054465053EFBEADDEE5
:10B04000A806002010B51F4CFFF74CFFA0B1FFF77A
:10B050000DFF0146AC221C480CF0A3FCFFF70BFFD0
:10B0600001464FF4C47220680CF09BFC2068406DD0
:10B07000BDE8104001F025BD4FF4C47120680CF00C
:10B08000ECFC00210420F9F75DFDFEF724FFDBE76F
:10B0900058B10E4A0168914207D1406820F00F0074
:10B0A000B0F5087F04BF012070470020704738B119
:10B0B000006820F00F00B0F5907F04BF01207047BA
:10B0C00000207047E8060020F80F0020415053523E
:10B0D000002808BF7047401E00BF00BF00BF00BF70
:10B0E00000BF0028F7D1704770B5614D82B00024D1
:10B0F000286804665F480168D1F82C13006841F0A5
:10B100000801C0F82C13F8F7FFF8286800692968CF
:10B1100040F001000861601EF8F782F8564880236D
:10B120004FF48012002152F821C040F821C0491C80
:10B13000B1EB930FF7D3F8F785F8F8F723FBF8F79F
:10B140004DFB0020F8F71FFB2320F8F710FBF7F763
:10B150003CFEF8F7C3FAF8F73BF9F7F75DFEF6F7B0
:10B160001BFEF5F7B9FDF8F702F8F7F7BDFF434E00
:10B17000009401940423002207213068F8F71CFA98
:10B180003068F8F794FA0420CDE900043C4C0346FB
:10B19000002207212068F8F70FFA2068F8F787FAED
:10B1A000F6F7CDFEF6F798FF364800683649884234
:10B1B00018BFF6F791FFF8F701FCFEF76FF8FEF7FE
:10B1C00032FD62B6FFF73EFF304803F0BCFC304C66
:10B1D0002068B0F90C0103F042FEF8F755FCF9F7CE
:10B1E0007FFE2068418A008AFEF733FA2068806E6D
:10B1F000C0F34E0161F35F0001F000F9FFF7E2FCDC
:10B2000000221146022001F006F9002264210720E5
:10B2100001F001F929680120086602B0002070BD24
:10B2200001F0F3FC01460220F9F78CFCF9F778FCF9
:10B2300006281AD2DFE800F019090313160602F0F7
:10B2400094FAF3E7FFF768F8F0E7FAF7D3FAF9F7BB
:10B2500067FC012804BF0220F9F771FCE6E701F062
:10B26000FCFAE3E7FEF737FEE0E7F9F7B0FCDDE7CD
:10B270006090110064901100006800207C90110023
:10B2800078901100F015002054464953F80F002023
:10B29000E8060020FE49087070474FF42C307047D4
:10B2A00070B54FF42C3044F264422146F6F708FFA3
:10B2B000F84A2168204691421BD16168B1F5007FB0
:10B2C00017D3D4F808C0002344F264418C4588BFEA
:10B2D00044F2644C0022B2EB9C0F28BF70BD54F8BE
:10B2E0002250521C2B44B2EB9C0FF8D3002B08BF0A
:10B2F00070BD002070BDE74901604FF400714160EE
:10B3000044F2644181600021C16080F8201080F81F
:10B31000211080F8221080F8231040F2FF72C0E95B
:10B3200004218161C161016500F580404FF6FF7124
:10B33000A0F85414A0F85614A0F85814A0F85A1401
:10B34000A0F85C14A0F85E14A0F86014A0F86214D1
:10B350000120704770B50021C1600B46D0F808C0CD
:10B3600044F2644104468C4588BF44F2644C002298
:10B37000B2EB9C0F06D254F82250521C2B44B2EB75
:10B380009C0FF8D35942C1604FF42C3044F2644210
:10B390002146F7F791FA012818BF002070BD2DE96A
:10B3A000F04F05468FB00E460020F6F717F80C90C8
:10B3B000F9F714FD8046B848DFF8E4B2032490F8AA
:10B3C00000A0B6480778DBF80000C46102217F20A6
:10B3D000F5F73AF840F20220F5F74FF8C0F30219FA
:10B3E000012E7DD000200690AE480390AE48089014
:10B3F000AE480490AE48002601960090DBF80000AD
:10B40000C46101217F20F5F71FF84FF48770F5F72D
:10B4100034F8C0B20D9002217F20F5F715F840F204
:10B420000720F5F72AF8C4B24FF40270F5F725F8B3
:10B430000DF0C8FB07909F4814F0100F50F829003A
:10B4400002909D4850F82900059018BF974E14F0BF
:10B45000200F04D0304604990DF062FA064614F02D
:10B46000400F04D0304600990DF05AFA0646E00924
:10B4700004D0304600990DF053FA064614F0010F3F
:10B480001CBF8A48019014F0020F04D0049901985F
:10B490000DF046FA019014F0040F04D0DDE900101D
:10B4A0000DF03EFA019014F0080F04D0DDE9001011
:10B4B0000DF036FA019016F1FF4F2CBF86F00040D8
:10B4C00030467E4CA042D8BF2646314601980DF04A
:10B4D0009BFA01904FF0FF3103980DF09CFD00E0C6
:10B4E00018E0814608990DF0B9FB83465946484655
:10B4F0000DF016FA0B90594648460DF0B7FC0A902D
:10B500000AFB07F04FF00009049000281ED80FB086
:10B51000BDE8F08F00240AFB07F6002E8EBF684FAF
:10B520000FB0BDE8F08FB5F900000DF04BFB57F8F8
:10B5300029100DF093FB0DF029FB25F8020B601C80
:10B5400084B2A642EFD80FB0BDE8F08F0020009083
:10B550000C98B0F9000009900C98801C0C9018F819
:10B5600001BB1BF0800F1CBF4FF07E5006900024E3
:10B570002BFA04F010F0010F13D00120A0400CF0C2
:10B580001EFF504A504B0CF081FF07468A46009838
:10B590000DF09AF93A4653460CF028FE0CF0F4FDF3
:10B5A0000090601CC4B2072CE2D3059902980DF0FC
:10B5B0005DFC0446DDE90A100DF058FC089009987E
:10B5C0000DF000FB6FF00A010DF025FD4FF07E51EC
:10B5D0000DF04CFC8346DDE902100DF0A1F906994F
:10B5E0000DF03CFB07464FF07E5006990DF03EFCF7
:10B5F0008246059903980DF093F951460DF02EFB04
:10B6000039460DF033FC82460D98401E0DF0DAFAF3
:10B61000074610F1FF4F28BF87F0004027498842B6
:10B62000D8BF264F4FF0804107980DF079F9099067
:10B63000394608980DF0E8F909990DF00FFB5946C5
:10B640000DF00CFB03990DF006FC834614F1FF4F3F
:10B650002CBF84F00040204618498842D8BF0C46D1
:10B6600016F1FF4F2CBF86F0004030468842D8BF0D
:10B670000E46DDE901010DF0F1FA0DF025F9CDE9F5
:10B680000801314600980DF0BFF951461EE0000058
:10B69000F006002053454C46BE050020BF050020A3
:10B6A000649011000000B040CDCC4C3FC3F5A040E9
:10B6B00048E1DA406C9411008C9411000AD7233CC5
:10B6C000AC9411009A9999999999A93F0DF0C6FAED
:10B6D0000DF0FAF807468A4658460DF0F5F84FF097
:10B6E000FF320DF06AFC3A4653460CF07FFDDDE96F
:10B6F00008230CF07BFD07468A4621464FF07E501A
:10B700000DF082F90DF0E0F83A4653460CF0BEFE1B
:10B710000022FE4B0CF0EEFF04460F4630460DF0C3
:10B72000D3F822463B460CF0B1FE0CF02DFDF84953
:10B730000DF094FAF7490DF0F3F80DF027FA25F81B
:10B74000020B09F101001FFA80F9049848453FF601
:10B75000FDAE0FB0BDE8F08F2DE9F043ADF2844DA2
:10B760000C4681464FF000084FF4906168460CF09B
:10B7700074F9E94FF5F7E9FA0020F5F7D9FA002056
:10B78000F5F7CBFAF5F7BDFA6846F8F7D6FBE348CC
:10B790000578E3480678002E18BF002D47D02068B2
:10B7A000002119F0030F80F8205080F8216080F804
:10B7B000221080F8231038D0F5F715FD0020F8F797
:10B7C000D2FB0120F5F74FFA2046F5F706FCFAF711
:10B7D000B1FC24680020F5F701FE0146754343F2F1
:10B7E00054006A0020440CF097F8F9F7F7FA014684
:10B7F00043F654002A4620440CF08EF8C94880785D
:10B8000010F0010F11D0F6F7B4FB002104F1540041
:10B81000FFF7C5FD386890F8EB00012805D1C2029A
:10B8200004F15401C0480CF077F84FF00108F5F727
:10B8300061FC0DF2844D4046BDE8F0832DE9F04FE8
:10B84000ADF5117D0E46044617464FF4107168465B
:10B850000CF003F9B3484FF000084FF0FF3980783F
:10B8600010F0020F43F2540007EB000504FB06F052
:10B8700090904ED06946AC46C246002E88BFA4F1D7
:10B88000010B2ED90020002C25D9584508BF81F87E
:10B8900000801CD03CF91020002AD8BF81F800900D
:10B8A00015DD0CEB4003B3F90230934207DCD31AE9
:10B8B0004FF0640E03FB0EF393FBF2F206E09A1ACC
:10B8C0004FF0640E02FB0EF292FBF3F20A70401C82
:10B8D000491CA042D9D30AF1010A0CEB440CB24531
:10B8E000D0D342F65400384469468246909A0CF010
:10B8F00058F88948006890F8EB00012804D1C2028A
:10B90000514689480CF008F84FF4107168460CF065
:10B91000A4F88448807810F0040F04BF0DF5117D61
:10B92000BDE8F08F68464FF0000A002C88BF06FB88
:10B9300004FB36D900221146BBF1000F05D829E0DF
:10B94000112A08BF80F800801FD00AEB010C35F9DE
:10B950001C30002BD8BF80F8009016DDA44435F9C8
:10B960001CC09C4508DCA3EB0C0C4FF0640E0CFBD8
:10B970000EFC9CFBF3F307E0ACEB03034FF0640E0B
:10B9800003FB0EF393FBFCF303702144521C204491
:10B990008B45D5D804FB1600401C0AF1010A54451A
:10B9A000C8D842F65440384469460446909A0BF091
:10B9B000F8FF5948006890F8EB00012804D1C20252
:10B9C000214659480BF0A8FF0DF5117DBDE8F08F19
:10B9D0002DE9F041504D0646144628680F4690F870
:10B9E000E8205248028000F0EAFD002306FB07F140
:10B9F000002984BFDFF838C14E4A12D9DCF80000B4
:10BA000041F6540730F8136004EB43003E521668C9
:10BA100000F5005036F813605B1CA0F854609942A2
:10BA2000ECD8286890F8EB0001280ED1C20241F64C
:10BA3000540021183C480BF06FFF42F254002118CB
:10BA40004FF400623C480BF067FF36490120486024
:10BA5000BDE8F08130B5054691B000240120F5F72E
:10BA600002F92046FFF75CFA6946FFF776FA00997B
:10BA70000798F4F79BFF314901200968C1F81403C6
:10BA80002846FAF74DF9FF20F9F7AFFBF5F75DF916
:10BA90000020F5F74DF90020F5F73FF9F5F731F9FA
:10BAA0000020F8F799F90020FAF703FC0120F8F7D5
:10BAB0005AFA11B030BDF0B5ADF2C44D0D46064690
:10BAC000144600274FF4906168460BF0C6FF202013
:10BAD000F9F78BFB0120F5F7C6F83846FFF720FA97
:10BAE000070008BFF9F756F80DF590613846FFF7E3
:10BAF00034FADDF88014DDF89C04F4F757FF0F49A1
:10BB000001200968C1F814031AE000000000F03FAA
:10BB100000007A440080CE43E8060020BE050020E5
:10BB2000BF050020F0060020006D00200407002063
:10BB30000C07002008070020007500206490110009
:10BB4000FAF7EEF8F5F701F90020F5F7F1F8002023
:10BB5000F5F7E3F8F5F7D5F80120F8F704FA6846A9
:10BB6000F8F7EBF90020FAF7A4FB0020F5F736FC14
:10BB700006FB05F14A00014641F254002044044608
:10BB80000BF0CAFEFE48006890F8EB0001281CBFCD
:10BB90000DF2C44DF0BD4FF400622146F9480BF0A0
:10BBA000BBFE0DF2C44DF0BD70B515460E46044601
:10BBB000F8F7C9F804FB06F14C0021460BF02BFF07
:10BBC0000220FFF747FFFAF7F3F90320FFF742FFE0
:10BBD000FAF7FBF9F8F7B7F80146224605F65400E4
:10BBE0000BF09AFEE648006890F8EB00012805D1BA
:10BBF000C20205F65401E3480BF08EFEF8F7A3F8F5
:10BC00002146BDE870400BF006BF2DE9F14FADF5C0
:10BC1000065D4FF00109C8464FF410610DF6D8508B
:10BC20000BF01BFF14204FF0000A14901390129099
:10BC300011905446CDF840A00120F5F714F82046A5
:10BC4000FFF76EF96946FFF788F900990798F4F74E
:10BC5000ADFEDFF834B30120DBF80010C1F81403A7
:10BC6000122720247D010020F5F757F8F5F7B6FDDF
:10BC7000DBF800100320C86101217F20F4F7E4FB0A
:10BC800011210E20F4F7E0FB5A210820F4F7DCFB29
:10BC900036210A20F4F7D8FB02217620F4F7D4FBF2
:10BCA00002217F20F4F7D0FB6A210220F4F7CCFBBD
:10BCB0008E210420F4F7C8FBF1210720F4F7C4FB20
:10BCC00007210820F4F7C0FB00211620F4F7BCFB85
:10BCD00003217F20F4F7B8FB89210520F4F7B4FB9A
:10BCE00067210620F4F7B0FB45210720F4F7ACFBF1
:10BCF00023210820F4F7A8FBF1210920F4F7A4FB85
:10BD000068004FEA570B04FB07F6009002E0B8F119
:10BD1000000F50D00120F4F7A6FFF5F729FC002012
:10BD2000F9F763FAF5F75FFA0120F4F79CFFF5F7EE
:10BD30001FFC1198F9F759FAF5F755FAB9F1000F08
:10BD400034D042F260106844F5F71DFD58B300206E
:10BD5000F4F7E3FFF5F742FDB8F1000F26D00AF142
:10BD600001001FFA80FABAF1010F4FF000000BD06A
:10BD7000F5F734FB014641F658306844009A0BF061
:10BD8000CBFD4FF0000811E0F5F728FB014641F22A
:10BD9000D8606844009A0BF0BFFD149911980844CC
:10BDA00080B2119002E0B9F1000FCAD14FF0010941
:10BDB000B8F1000FAED10020002D18D941F2D863A0
:10BDC0006B4403F590620DF59B6C32F9101033F95A
:10BDD0001080A1EB08014FF0640801FB08F101EBB2
:10BDE000D17149104CF82010401CA842EDD34FF0FF
:10BDF00000084346002C25D941F6D87A0DF59B69F9
:10BE0000EA4409F5DC5E00210A464046B8EB560FCD
:10BE10000BD259F820C0624400EB560C204459F86C
:10BE20002CC0B0EB560F6144F3D3B2FBFBF04AF8E1
:10BE30002300B1FBFBF04EF823005B1C08F1010866
:10BE4000A342E0D30020002D1FD941F6D8730DF591
:10BE50009B626B4402F5DC5C0DF15808B0FBF4F119
:10BE600004FB1101B0EB550F34BF53F821105CF8FF
:10BE7000211052F82090A1EB09010029B8BF4942D6
:10BE800028F81010401CA842E8D34FF00008002FFB
:10BE900082BF42F22019E944A9F1480A23D916A821
:10BEA00000EB8811402248460BF036FD0020002FA1
:10BEB00015D90021002C09D939F811305AF8202061
:10BEC000491C1A444AF820208C42F5D85AF8201010
:10BED00091FBF4F14AF82010401CB842E9D308F174
:10BEE0000108B845DBD30020002D82BF42F2D808FC
:10BEF000E8440DF1580C0CD941093CF8103058F8C1
:10BF00002120D11A48BF991A2CF81010401CA842C1
:10BF1000F2D30020002D84BF16AA0DF6D85109D9FE
:10BF200051F8203032F810C0634441F82030401CF2
:10BF30008542F5D810981399401CC0B21090129801
:10BF4000119010984FF001084FF0000AC14681424D
:10BF50003FF6DDAE0024002D21D9DFF8308016AE8B
:10BF60000DF6D857109857F82410B1FBF0F00CF0EC
:10BF70003DFA4FF0663243460CF088FA08E00000C4
:10BF8000E8060020006D0020649011006666E63F20
:10BF90000CF0E8F926F81400641CAC42E2D30DF56D
:10BFA000005316A9D3F8800143F654431844009A6D
:10BFB00004460BF0F6FCFE48006890F8EB00012800
:10BFC0001EBF61B00DF5005DBDE8F08F4FF400625B
:10BFD0002146F8480BF0A0FC61B00DF5005DBDE80E
:10BFE000F08F2DE9F05FADF5924D44F270476F444C
:10BFF0004FF4906138460BF030FD03ADFF2244F260
:10C00000644128460BF0FFFCDFF8AC834FF0FF30B3
:10C010000290D8F804000DF1080A4FF0FF0928B982
:10C02000FF224FF40061E5480BF0EDFC2846029535
:10C03000FFF761F9DE4E346894F8EA00A8F80200D0
:10C04000B4F9D8000CF0BEFD019094F8EB00032881
:10C0500004D1012088F80000A8F802900120F4F72C
:10C0600002FE514698F80000FFF776FB3846F7F7D6
:10C0700064FF9DF82C409DF82D70002C12BF002FFE
:10C080000DF5924DBDE8F09F4FF0000B2A46394662
:10C090002046CDF81CB0FFF7D1FB98F8020010F055
:10C0A000080F04D02A4639462046FFF791FC98F83D
:10C0B000000010F0010F39D098F8020010F0200FA6
:10C0C00004D02A4639462046FFF7F5FC98F80200CE
:10C0D00010F0400F2AD0F7F736FE04FB07F14FEAC5
:10C0E000410949460BF097FC0220FFF7B3FCF9F732
:10C0F0005FFF0320FFF7AEFCF9F767FFF7F723FEBA
:10C1000001464A4605F654000BF006FC306890F8EC
:10C11000EB00012805D1C20205F65401A5480BF039
:10C12000FBFBF7F710FE49460BF075FC98F8020090
:10C1300010F0800F1CBF2846FFF767FD98F800003D
:10C1400010F0400F40F025810898401C0890079897
:10C15000002814BF0A98099800F1010014BF0A9042
:10C16000099004FB07F0441E58BFDFF854A27CD4AA
:10C1700098F8020010F0010F2FD0924901980CF0AE
:10C1800043FC4FF07E5100900CF065FE51460CF0E0
:10C1900065FD05EB44078146B7F954000CF012FD2C
:10C1A00049460CF027FD10D34FF07E5100980CF05B
:10C1B000B7FB51460CF052FD8146B7F954000CF024
:10C1C00001FD49460CF016FE07D217980DF5804187
:10C1D00040F001001790A1F86844B8F8020010F090
:10C1E000020F15D02919326801F5005191F9541840
:10C1F000B2F9C8308B4203DCB2F9CA208A4207DAAE
:10C2000017990DF5804241F002011791A2F86044A0
:10C2100010F0040F15D02919326801F5005191F979
:10C22000541CB2F9CC308B4203DCB2F9CE208A42E6
:10C2300007DA17990DF5804241F004011791A2F831
:10C24000624410F0080F18D005EB4401326801F584
:10C250008051B1F95418B2F9D0308B4203DCB2F9F5
:10C26000D2208A4209DA179900E06EE041F0080115
:10C270000DF580421791A2F8644410F0100F16D00B
:10C2800005EB4401326801F50051B1F95410B2F9DF
:10C29000D4308B4203DCB2F9D6208A4207DA1799F0
:10C2A0000DF5804241F010011791A2F8664410F09C
:10C2B000200F16D005EB4401326801F58051B1F929
:10C2C0005410B2F9DC308B4203DCB2F9DE208A4232
:10C2D00007DA17990DF5804241F020011791A2F875
:10C2E0006A4410F0400F14D0326805EB4401B1F9F4
:10C2F0005418B2F9E0308B4203DCB2F9E2208A42F2
:10C3000007DA17990DF5804241F040011791A2F824
:10C310006C4410F0800F15D005EB440043F65441F7
:10C32000415E3068B0F9E4208A4203DCB0F9E600EF
:10C33000884207DA17980DF5804140F08000179089
:10C34000A1F86E44641E7FF513AF306890F8EB00DF
:10C35000F8B90598002144F264422B46CDF818B094
:10C36000904294BF024644F264420020B0EB920F28
:10C3700006D255F820C0401C6144B0EB920FF8D3B0
:10C380004842D8604FF42C3044F264422946F6F714
:10C3900093FA306890F8EB00032802D1054917980A
:10C3A00008801D208DF8000041208DF801000BE071
:10C3B000E8060020006D0020F00600200075002037
:10C3C00000803B450000C8429DF85C008DF80200EB
:10C3D0009DF85D008DF803009DF85E008DF8040067
:10C3E0009DF85F008DF8050006226946072000F0E1
:10C3F0003BF80DF5924DBDE8F09F00005149C2B2E7
:10C40000C0F307200A80488070474E484188008862
:10C4100061F31F20704710B54A4C012303FA00FC5A
:10C42000248882B01CEA040F04BF02B010BD00F0E3
:10C430000F0043EA80008DF800008DF801108DF8A0
:10C440000220100A8DF80300100C8DF80400100E65
:10C450008DF8050000208DF806008DF8070068466D
:10C46000FDF742FC02B010BD012303FA00F000B555
:10C47000344B83B01B88184204BF03B000BD072AA9
:10C4800088BF072200206B46002A08D911F800C097
:10C4900003F800C0401C9042F8D3082804D20021C1
:10C4A0001954401C0828FBD31846FDF71DFC03B0A7
:10C4B00000BDDFF890C001238340BCF802C013EA3E
:10C4C0000C0F08BF704710B582B000F03F0040F07D
:10C4D00080008DF80000072A88BF072200206B46E5
:10C4E000002A09D911F800C01C18401C84F801C0AA
:10C4F0009042F7D3072805D200211A18401C51702A
:10C500000728FAD31846FDF7EFFB02B010BD10B4B0
:10C510000C4C40EA01230228A288944602D0052848
:10C5200005D009E0002918BF022905D103E0002940
:10C5300018BF022900D11A46944518BFA28010BC2A
:10C5400070470000F8060020F74908707047F64869
:10C5500000B5C07848F6B80183B0484301218DF892
:10C56000011000214A1E8DF807108DF80010ADF85B
:10C5700004208DF80810ADF802208DF806108DF813
:10C580000910F7F7B4F8FCF7BAFE01280DD0012026
:10C59000F6F7B4FBF7F7C2F80028F4D06846FDF7C9
:10C5A0003EFC0020F7F7B7F8EDE7F7F7AFF803B078
:10C5B00000BDDD4948707047DB48407870472DE981
:10C5C000F04FADF2F44D4FF4906104A80BF045FA32
:10C5D000DFF854830221002088F80110FEF7A0FC48
:10C5E000040008BFF8F7D6FAF4F7FAFC0DF59261EB
:10C5F0002046FEF7B2FCDDF89014DDF8AC04F4F749
:10C60000D5F9CA4901200968C1F81403F4F79DFB64
:10C610000020F4F78DFB0020F4F77FFBF4F771FBAB
:10C6200004A8F7F78AFCF4F76DFDCDF8EC0498F850
:10C63000020010F0100F18BFF5F700FABC4890F890
:10C640000090BC480778BC48002F0578BB480678A6
:10C6500018BFB9F1000F0ED0FEF7B3FA0020F7F7BC
:10C66000BBFB98F8020010F0100F0AD00120F7F77A
:10C670007AFC012009E0002E18BF002DECD100F05B
:10C68000E6B80020F7F76FFC0020F7F76CFC0120FC
:10C69000F4F727FAF4F7A7FD1E20FDF70AF80021AA
:10C6A0000846FCF7BDFFC8F8080001210020FCF790
:10C6B000B7FFC8F80C00002009FB07F4DFF880A2E0
:10C6C000002C88BF47F6FF710AD9D8F8082022F855
:10C6D00010A0D8F80C2022F81010401C8442F4D886
:10C6E0001E20FDF705FA00210120FCF799FF834683
:10C6F00001210846FCF794FF01460020AB1918BF42
:10C7000047F6FF7206D02BF810A021F81020401C2D
:10C710008342F8D8B8F804000026864238BF4FF0AC
:10C72000000B6FD2FCF7EBFD01286BD00DF59A6082
:10C73000F5F729F800285FD0DDF8D404002857D099
:10C7400098F8020010F0100F0BD0DDF8D454F7F772
:10C75000FAFA2A4601464B4610460097F7F7DAF9EF
:10C7600022E00023CDF800B0CDF804B0CDF808B039
:10C77000CDF80CB01A461946DDF8D404FEF73AF8A5
:10C78000054698F8020010F0200F03D0FEF72CF8B1
:10C79000054608E0F7F7D7FA2A4601464B46104609
:10C7A0000097F7F7B7F91DB30021002C88BF534657
:10C7B0001ED935F91100B0F5004FA8BF47F6FF703C
:10C7C00003DA10F5004FB8BF1846D8F8082032F940
:10C7D00011C08445B8BF22F81100D8F80C2032F9F6
:10C7E00011C08445C8BF22F81100491C8C42E0D812
:10C7F000F4F7F4FF761C01E0F8F7CCF9B8F8040080
:10C8000086428FD30120F4F72EFAFEF7DAF9B8F852
:10C810000400B0421BD8DDF8EC0410F0020F16D073
:10C8200000234FF6FF721846002C88BFD8E902C5D6
:10C830000DD93CF9101035F91060891B9942C8BF19
:10C840000B469142B8BF0A46401C8442F1D8F4F727
:10C8500051FC0DF2F44DBDE8F08F2DE9F041324D61
:10C86000002484B06C70374F4FF00108661EFCF74F
:10C8700046FD012806D1F8F753F903281CBF04B080
:10C88000BDE8F081287810F0010F05D0FFF7A9FB73
:10C890003C702C70FCF72FFD287810F0020F07D0A9
:10C8A000FFF78DFE287820F002002870FCF723FDAA
:10C8B000287810F0040F2FD0E8788DF801808DF8DB
:10C8C000074048F6B8018DF80040ADF804608DF8D7
:10C8D00008404843ADF802608DF806408DF80940E5
:10C8E000F6F705FFFCF70BFD01280DD00120F6F748
:10C8F00005FAF6F713FF0028F4D06846FDF78FFA23
:10C900000020F6F708FFEDE7F6F700FF287820F0A3
:10C9100002002870FCF7EFFCF8F702F90328A6D014
:10C9200004B0BDE8F0810000000700206490110011
:10C93000BE050020BF050020C3050020C40500205F
:10C940000080FFFF1607002003490968A1F8E800EE
:10C9500070470249C8707047E806002000070020B1
:10C96000F748C079704700220028D8BF70470021DF
:10C9700000BF491C0829FBDB521C8242F7DB7047D1
:10C980002DE9F04F002283B0EE490092019291F818
:10C9900004904F8AB1F810804E79B7FBF9FEB8FBCE
:10C9A000F6FBB1F90E5094461446B9F1000F18DDAC
:10C9B0000021002E11DD01EB421330F91330AB42A0
:10C9C00007DD0CEB441A30F91AA05345C4BF1446D6
:10C9D0008C46491C09B28E42EDDC511C0AB29145CD
:10C9E000E6DC5CEA04004FF0010355D0611CD54A37
:10C9F0000CF1010000FB0BF0948A00B201FB0EF178
:10CA0000D58A09B204FB00FC9CFBF8F005FB01F29F
:10CA100092FBF7F100B209B28045DCBFA8F101003A
:10CA200000B2B942A4BF791E09B2C74A126892691E
:10CA300012F0040F14BF23EA020C02F0010CBCF147
:10CA4000000F02D0691A491E09B212F0020F02D07B
:10CA5000201A401E00B212F0040F12BF0A4602460E
:10CA6000084641218DF800108DF8013011098DF82C
:10CA7000021001098DF8031002F00F0161F31F107D
:10CA80008DF804000A208DF805006846FDF72CF9A2
:10CA900003B00120BDE8F08F43208DF80000002096
:10CAA0008DF801308DF802008DF804008DF8030038
:10CAB0008DF805006846FDF717F903B00020BDE8C2
:10CAC000F08F9F4982B26FF30F00C1E904027047F3
:10CAD0009B48407870479A4A0028516914BF41F03A
:10CAE000020021F002005061704710B55A20F5F79E
:10CAF000BCF980220021B620F5F703F900220121BC
:10CB0000B620F5F7FEF8BDE81040A520F5F7ADB961
:10CB100010B55A20F5F7A9F911220021B620F5F732
:10CB2000F0F806220121B620F5F7EBF8BDE8104039
:10CB3000A520F5F79AB9854810B50068C068804906
:10CB400010F0040F087A16D0022808BF10BD02208A
:10CB500008725A20F5F789F980220021B620F5F7EE
:10CB6000D0F800220121B620F5F7CBF8BDE810403F
:10CB7000A520F5F77AB9022818BF10BD0120087268
:10CB80005A20F5F772F911220021B620F5F7B9F80D
:10CB900006220121B620F5F7B4F8BDE81040A52023
:10CBA000F5F763B96648007DC0F340007047644AFA
:10CBB000F02303EA0010516921F0F00108435061AD
:10CBC00070475F48007DC0F3031070475C4A00283F
:10CBD000516914BF41F0010021F00100506170471C
:10CBE0005748007D00F001007047554B19690A0E47
:10CBF000120721F07F4142EA006008431861704744
:10CC00004F480069C0F3036070474F480068406DAB
:10CC1000C0F303607047012101FA00F04FF47F0177
:10CC200001EA004146480269114301617047012150
:10CC300001FA00F04FF47F0101EA00414048026927
:10CC400022EA0101016170473D480069C0F30740D5
:10CC500070473B48008AC0F303307047384A4FF4AE
:10CC6000704C0CEA00301169C1F3033321F47041B8
:10CC700008431061184670473148808AC0F380200D
:10CC8000704770B52E4E0446C0F380007569C5F339
:10CC90000021884218BFF7F751F814F0040F14BFB1
:10CCA00045F4807025F4807014F0080F14BF40F430
:10CCB000007020F4007014F0200F14BF40F4806066
:10CCC00020F4806014F0100F14BF40F4006020F4D2
:10CCD000006014F0800F14BF40F0800020F080004E
:10CCE0007061BDE87040FEF753B8154841690020F7
:10CCF00011F0400F18BF012011F4807F18BF40F0E1
:10CD0000040011F4007F18BF40F0080011F4806F98
:10CD100018BF40F0200011F4006F18BF40F0100061
:10CD200011F0800F18BF40F0800070470448007D6C
:10CD3000C0F3401070470248808AC0F3002070475B
:10CD400010070020F80F0020E80600206090110076
:10CD5000FB48808AC0F300307047F9484069C0F34F
:10CD6000003129B1C0F34010002804BF01207047F2
:10CD700000207047F2498A691043886170472DE9A5
:10CD8000F047EF4F0D46396A491C39624FF00008F1
:10CD90000028C8BFC7F8248015D0002DC8BFC7F829
:10CDA000288014D0397D11F0010F7DD03969DFF86A
:10CDB0009493C1F303642646062C56D2DFE804F0B0
:10CDC0000B2A3A556464796A491C7962E5E7B96AC5
:10CDD000491CB962E6E7002805DD022000F083FE69
:10CDE00008B1022444E0002D05DD012000F07BFEA7
:10CDF00008B101243CE0D9F80000396A90F8290014
:10CE000000EB8000884231D802240120C7F820803E
:10CE1000F8622DE0002804DD022000F064FE002806
:10CE2000DFD11DBBD9F80000B96AB0F85E008842B6
:10CE30001CD216E0002818BFC7F82C8016D101209C
:10CE400000F051FE0028D4D1D9F80000796AB0F87A
:10CE50005C00884205D3F86A012808BFC7F82C8017
:10CE600004D1002000F03FFE00B10024B44235D0D0
:10CE70003869010E090720F07F4041EA0461084348
:10CE800038610120BDE8F087002806DD022000F0AF
:10CE90002AFE002818BF0224E8D1002D08DD012059
:10CEA00000F021FE002800E018E018BF0124DDD1C9
:10CEB000042E0DD17869C0F3003149B1C0F34010A0
:10CEC00030B9052000F00FFE002818BF0524CFD18F
:10CED000002000F008FE0028C8D0C6E70020BDE80A
:10CEE000F0872DE9F04188460446F5F728F8F4F775
:10CEF00077F8954A03211268D1611F26934D4A277E
:10CF00001CB1012C12D0022C26D001217F20F3F776
:10CF10009BFA1F210E20F3F797FA4A210820F3F716
:10CF200093FA85F8EE6685F8E87615E001217F2012
:10CF3000F3F78AFA15210E20F3F786FA75210820F7
:10CF4000F3F782FA152085F8EE0675207C4985F8FE
:10CF5000E80601208870C870B8F1010F04BF0020F6
:10CF6000F7F701F8F4F73FF9BDE8F041F4F7CABF6D
:10CF70002DE9F04FA3B000254FF0FF3BCDF818B0DE
:10CF8000ADF864508DF86850CDF828B0CDF81CB0DD
:10CF9000CDF814B0CDF810B01595446807461B9530
:10CFA00009950020D7F80890149018900890DFF8A1
:10CFB00090A11CA82E46A8460B90B9F1000F08D0EE
:10CFC00016AA05A94846FDF756FD1790FDF751FD35
:10CFD00014909CB15E4A1AA919A80A9B8DE80F000B
:10CFE0009AF9003007A920460B9AFDF703FC099037
:10CFF000FDF7FAFB1B90FDF7FAFB8046DAF81410F8
:10D00000C1F34000002800F0D980524801968068A2
:10D0100038680D901B98CDE90E080B981096CDE955
:10D02000126014981190BDF88400ADF83000DAF861
:10D03000180011F0400F40F40070CAF818601CBFCF
:10D0400011F0040F40F0010011F4807F18BF40F090
:10D05000040011F4007F18BF40F0080011F4806F45
:10D0600018BF40F0200011F4006F18BF40F010000E
:10D0700011F4805F18BF40F0400011F0800F18BF1E
:10D0800040F08000BAF81010C1F3033140EA0140CB
:10D09000002918BF40F48060002C08BF20F0010078
:10D0A0000799B1F1FF3F08BF01259AF80C10032939
:10D0B00038BF01259AF803100127012904BF042174
:10D0C000ADF8641006D0BDF86410072908BF8AF8CF
:10D0D000057003D09AF80510012902D10721ADF897
:10D0E00064100095BDF8643001AA0CA901F047FE58
:10D0F00005460198806820F0080110F0080FCAF872
:10D100001C1014BF8AF801708AF8016010F0100F2B
:10D110002AD09AF8020020B19AF8030001281BD007
:10D1200022E09AF804009AF8031008431CD1002169
:10D130000120FFF7D6FE8AF802708AF8037013E028
:10D1400010070020E8060020649011009C5D00207C
:10D150001D0700201416002000210846FFF7C1FE1D
:10D160008AF802608AF804700198007A10F0200FA3
:10D170009AF80A0008D080B98AF80A70012264215E
:10D180000720FFF748F908E0012806D18AF80A606D
:10D19000002264210720FFF73EF901980168002969
:10D1A000CCBF8AF800708AF80060002D06BF416885
:10D1B00000298AF8096032D0D0F800B0079800281A
:10D1C000C4BFAAF80E608AF80B6008DCB0F1FF3F1C
:10D1D000BAF80E000CBF801C401CAAF80E009AF88A
:10D1E0000C00032807D29AF80C00401C8AF80C00A7
:10D1F0004FF0FF300790FA4D2868017F11F0010FC2
:10D200007AD0407FBAF80E10814222D8DAF82C107A
:10D2100001291CBF0799B1F1FF3F6DD119E0017AD7
:10D220004FF0C80211F0400F03D007968AF809208A
:10D23000C2E79AF8091031B1491CC9B28AF809103D
:10D24000C829F2D2B8E70799012908BF8AF80970FE
:10D25000B2E7AAF80E608AF803608AF804608AF8D8
:10D260000560BAF80E10884204D2012299210720E5
:10D27000FFF7D1F8DAF82C00012804D10222992115
:10D280000720FFF7C8F80798B0F1FF3F04D1032249
:10D2900099210720FFF7BFF86CB115981899CDE9CF
:10D2A00002B0CDE90018DDE90703DDE90921F7F750
:10D2B0000BFC8AF80960179828B1DAF82420014697
:10D2C0000598F7F7E8FB9AF80B00401CC0B28AF803
:10D2D0000B00042810D905208AF80B009AF80200E8
:10D2E000012809D101210020FFF7FBFD8AF8036026
:10D2F0008AF802608AF80460BA4C2078242804BFB7
:10D300001B98FCF7C3FA2078012804BF1B98FCF790
:10D31000BDFA20780E2804BF1B98FCF7B7FAB9F1C4
:10D32000000F1CBF9AF80D00022811D0286890F851
:10D330006C0010F0010F0BD0BDF95800149A05993C
:10D34000FDF7CEFC00281EBF012023B0BDE8F08F02
:10D35000DDE90610DDE90432FFF711FD23B0BDE879
:10D36000F08FF0B587B00746F7F7DAFB0546F7F719
:10D37000DAFB9D490646052D0CBF9C4CAFF20F44CD
:10D380004869C0F3031118BF052E08D1C0F300325D
:10D390002AB1C0F34010002808BF41F0020138460E
:10D3A000F7F78AFC002804BF07B0F0BDF6F796FC3B
:10D3B00007460020F3F795FBF3F715FFFBF79FFFF8
:10D3C000012809D0F7F7ACFBA84205D1F7F7ABFB72
:10D3D000B04208BF002F05D0F3F702FEF7F7EFFCCD
:10D3E00007B0F0BD6846F4F7CEF940B16846FCF7E7
:10D3F000B6FB6846A0470746F4F7F0F9DEE7F7F713
:10D40000BEFBDBE72DE9F04F002485B0784904949A
:10D4100023460E78009401940294224604A90394B2
:10D42000FDF7E8F9FDF7E0F90546002700940194BF
:10D43000F7F776FB6A490528096851D0888FB1F85B
:10D440003EA0C0F30B09000BB9FBF0F80020711EE1
:10D4500004468446EE46029100210CFB06F3002EA2
:10D460002ED935F913203EF91CB0934505DA0DF19C
:10D47000040B2EF81C202BF81C104A451BDD3A44E7
:10D4800031B105EB430737F9027C3A44474500DDEB
:10D490000120029FB94206D205EB4307B7F902709B
:10D4A0003A44474500DD012401280CBF012C5245B8
:10D4B000A4BF012204920027491C5B1CB142D0D3B7
:10D4C0000CF1010CBCF1020FC6D3464800780128CC
:10D4D00004BF2846FCF7DAF9049805B0BDE8F08FE0
:10D4E000B1F80001B1F802A1C0F30B09000BB9FBC0
:10D4F000F0F8ABE72DE9F04F87B00646002402278D
:10D50000FDF70EFD002804BF07B0BDE8F08F364DD3
:10D51000287DC0F3031AF7F703FB8146F7F703FBF7
:10D52000804651463046F7F7C7FB002804BF07B0D6
:10D53000BDE8F08FE8792F4E4FF0010B4FF0000A55
:10D54000012838D0F8F7F6FDF8F7D0FE0120F6F7FD
:10D550000AFDF6F7F8FB01464FF4906226480AF000
:10D56000DBF985F807B002212020F3F73DFF00200A
:10D57000F3F7D3FB3068406C316840F400604864D6
:10D5800001220021002000BF401C0828FBDB491CB1
:10D590009142F7DB3068406C316820F400604864E9
:10D5A000F4F7B0FCF3F71FFEC5F830B0002C08BF4D
:10D5B000124E7CD124E03068D0F82C03316820F082
:10D5C0000400C1F82C033068C0F810A30120F3F761
:10D5D0004AFB0948F6F7BBFBF4F73BFAC3E7000048
:10D5E000E80600203106002010070020DF9F100011
:10D5F000BE05002064901100E2070020AA0500206B
:10D60000FBF77DFE012807D0F7F78AFA484503D1DA
:10D61000F7F789FA404504D0F4F791FCF3F7E0FC02
:10D620008BE0F74800789C2810D0F4F788FCF54888
:10D630000168D1F82C13006841F00401C0F82C13E4
:10D640000020F2F7DBFF86F800A005E0307818B97B
:10D65000F4F758FCF3F7C7FDEB4800684069C0F3E6
:10D660000720022808BFF6F7DAF96846F4F78BF8C6
:10D6700000285FD06846FCF772FAE4480068C0688A
:10D6800010F0040F287A16D0022828D00220287221
:10D690005A20F4F7EAFB80220021B620F4F731FB90
:10D6A00000220121B620F4F72CFBA52000E044E085
:10D6B000F4F7DBFB13E0022811D1012028725A2075
:10D6C000F4F7D3FB11220021B620F4F71AFB06224F
:10D6D0000121B620F4F715FBA520F4F7C6FB4FF0A7
:10D6E000FF340198A346C0B1FFF78CFE0028C8BFE5
:10D6F000012410DCE8890024401CE881C44800684B
:10D70000017F11F0010F08D0807FE989814204D99F
:10D710000198F6F71CFBA5F80EA0FDF7D5FA00233B
:10D720001A4659462046FFF72AFB0446F4F756F8F6
:10D73000F4F71FFC002C3FF463AFF2F7ADFFF7F7EF
:10D74000EFF9022805D0F7F7EBF907460220F7F7C3
:10D75000F6F9F7F734FB022F1CBF3846F7F7EFF95D
:10D76000F8F75DFC07B0BDE8F08F2DE9F04FADF2A2
:10D770001C5DF5F7C9FDFDF738FAA54C2068B0F936
:10D780003610B0F93400FCF7E1FFA2484FF0010B6E
:10D7900080F8C0B6A04880F8C0B62068B0F858003D
:10D7A000C0F303200F2818BFF6F7B2FA9B4D686943
:10D7B00040F001006861F7F7B3F9022808BF4FF0A5
:10D7C000000A40F079812869C0F303649048A10001
:10D7D0000068806DC5F820A0C84000F00F00C5F8B3
:10D7E00024A0C5F828A0062C80F05D81DFE804F0B5
:10D7F000FC030303FBFB8046686900274FF0020926
:10D80000C0F30316022C0BD1C0F3003131B1C0F3C9
:10D810004010002808BF46F0020601D026F002069C
:10D82000A879012843D031464046F7F745FA002849
:10D8300000F03981F8F77EFCF8F758FD0020F6F784
:10D8400092FB85F806B0FDF7BCF9686940F002006C
:10D850006861A86940F00100A8610020F3F75DFA53
:10D86000F4F750FB684E30688068316840F0020081
:10D870008860F3F7B8FC85F800A001F04DF9DFF8F7
:10D88000A0813068C06810F0100F07D03068806841
:10D89000316840F010008860F4F779FBFBF72FFD4A
:10D8A000012812D0F7F73CF9022807D00DE0F7F76E
:10D8B000ADF931464046F7F7C3F9C4E72869C0F32C
:10D8C0000360A04208BF002F1AD0F4F738FBF3F72B
:10D8D00087FBFDF776F9F8F76BFBF7F721F90228DC
:10D8E00005D0F7F71DF981460220F7F728F9F7F779
:10D8F00066FAB9F1020F1CBF4846F7F720F9D2E0EB
:10D900003F4800789C2810D0F4F719FB3D48016887
:10D91000D1F82C13006841F00401C0F82C1300204A
:10D92000F2F76CFE88F800A006E098F8000018B93D
:10D93000F4F7E8FAF3F757FC30684069C0F30720C2
:10D94000022808BFF6F76BF80DF5A060F3F71BFF90
:10D95000002896D00DF5A060FCF701F93148007859
:10D9600001280FD14FF4A06168460AF076F8002133
:10D970006846FDF714FD2C4800780B2804BF684664
:10D98000FBF784FF21480068C06810F0040F287A74
:10D9900014D0022826D0022028725A20F4F765FA03
:10D9A00080220021B620F4F7ACF900220121B62034
:10D9B000F4F7A7F9A520F4F758FA13E0022811D1DB
:10D9C00085F808B05A20F4F750FA11220021B62049
:10D9D000F4F797F906220121B620F4F792F9A52071
:10D9E000F4F743FA01E024E020E00DF5A060FFF732
:10D9F000BFFA0746F3F7F2FEF4F7BBFA41E700007F
:10DA0000AE0500206490110080901100609011001C
:10DA1000E80600209C5D0020E2070020100700209F
:10DA2000AA050020EF05002031060020FFF762FD67
:10DA300039E08046F7F774F80646F7F774F80746BA
:10DA4000052E0CBF354CAFF6D7246869C0F303111F
:10DA500018BF052F08D1C0F300322AB1C0F340101F
:10DA6000002808BF41F002014046F7F725F9D0B180
:10DA7000F6F734F980460020F3F733F8F3F7B3FBF9
:10DA8000FBF73DFC01280AD0F7F74AF8B04206D16F
:10DA9000F7F749F8B84208BFB8F1000F12D0F3F712
:10DAA0009FFAF7F78CF9FBF72AFC012804D0F7F767
:10DAB00037F802283FF487AE0DF21C5DBDE8F04F49
:10DAC000FDF793B86846F3F75EFE40B16846FCF791
:10DAD00046F86846A0478046F3F780FED0E7F7F7A0
:10DAE0004EF8CDE770470E4A0228117D1269C1F346
:10DAF0000311C2F3074205D0012808BF11F0020F3D
:10DB00000AD002E011F0040F06D0012101FA00F062
:10DB1000104018BF0120704700207047DF9F1000A1
:10DB200010070020FE487047FE487047FE48007806
:10DB30007047FD48407870470346002002460029A0
:10DB4000D8BF704753F822C0521C60449142F9DCA0
:10DB500070472DE9F05F0E46054600F0D9FC0446FB
:10DB600000F0D2FC310291FBF0FC290291FBF4F3AE
:10DB7000DFF8B4E3EB4D5E12BEF80490BEF8068009
:10DB800000214FEA6C2705F5907A002C0BDD01FB94
:10DB900003F206EB222245F821204AF82120491CF5
:10DBA00009B28C42F3DCDE4E002106F5907B0028A2
:10DBB0000BDD01FB0CF207EB222246F821204BF88B
:10DBC0002120491C09B28842F3DC0CFB09FC03FB51
:10DBD00008F34FEA6C315A135F13CEF80C102B6820
:10DBE0004FEA6C3C9B1A2B6005EB840353F8045CF2
:10DBF000154443F8045C33685B1A336006EB80031A
:10DC000053F8045C0D4443F8045C9EF80330002B89
:10DC1000DAF8003017D09B1ACAF800300AEB8403F8
:10DC20000BEB800053F804CC624443F8042CDBF87F
:10DC30000020521ACBF8002050F8042C114440F870
:10DC4000041CBDE8F09F9A1ACAF800200AEB84026F
:10DC50000BEB800052F8043C3B4442F8043CDBF8F8
:10DC60000020511ACBF8001050F8041C6144E6E77C
:10DC7000AE4930B40968AC4A4FF00A0C4C8A098AA4
:10DC80001423A2F804C0D380A0201081400050814A
:10DC9000204630BC5DE7A448C078012818BF0020AA
:10DCA00070475FEA000C30B4A0489F4B0268508A6E
:10DCB000118A14D092F854C0528B4FEADC0404FB52
:10DCC00000FCBCFBF2F21A705A700A229A801422ED
:10DCD000DA80A0221A8152005A8130BC39E7002232
:10DCE0001A705A70F1E79148026892F85430508ADD
:10DCF000B2F81AC0DB084343B3FBFCF3118A8A4A2B
:10DD0000137053700A2393801423D380A0231381AC
:10DD10005B005381C0EB0013B3FBFCF39370002353
:10DD2000D37016E72DE9F04FB3B00D460446CC2270
:10DD30007F49684609F035FE7C48B5F90220006845
:10DD4000012A90F805C090F80480478A068A68780E
:10DD500000FB0CF109B2D8BF01222B78DFF8D4E127
:10DD6000EB4683B1ACF101094B45194417D104EBE3
:10DD7000410131F9021C0129D8BF0121C9024942E0
:10DD800091FBF2F140E004EB4101B1F902100129ED
:10DD9000D8BF0121C90291FBF2F109B235E004EBD1
:10DDA000410939F9021C0129D8BF0121B9F90290B2
:10DDB000B9F1010FD8BF4FF001094FF0640A01FB20
:10DDC0000AF109FB0AF901EB620109EB620991FB17
:10DDD000F2F199FBF2F93BF911103BF91990494521
:10DDE00008BF002111D001EB090A1AF5004FB8BF96
:10DDF000F24604DBBAF5004FA8BF47F6FF7AA1EB65
:10DE00000901C90291FBFAF109B2A0B1A8F1010917
:10DE10004845A0F1010909FB0CF90FFA89F9994469
:10DE200015D134F91940012CD8BF0124E402644211
:10DE300094FBF2F246E003EB0C0934F91940012C93
:10DE4000D8BF0124E40294FBF2F212B23BE034F9B1
:10DE50001990B9F1010FD8BF4FF0010900F1010A83
:10DE60000AFB0CFA0FFA8AFA9A4434F91AA0BAF1AA
:10DE7000010FD8BF4FF0010A642409FB04F404EB3E
:10DE8000620494FBF2F44FF064090AFB09F909EB10
:10DE9000620999FBF2F23BF914403BF912209442DB
:10DEA00008BF00220FD004EB020919F5004F05DB73
:10DEB000B9F5004FB4BFCE4647F6FF7EA21AD20294
:10DEC00092FBFEF212B21B04000403EB011100EB03
:10DED000021201F5004002F5004190FBFCF091FBBD
:10DEE000F8F1704301FB07F100144FEA21414CBFE8
:10DEF00000220246B242C8BF304602DC0028B8BF4A
:10DF000000200029B4BF00220A46BA42C8BF3946E1
:10DF100002DC0029B8BF0021A5F8B4000CE0000025
:10DF2000007D0020907D0020480700206007002031
:10DF3000CC9411000080FFFFA5F8B61033B0BDE807
:10DF4000F08F70B5A4B00D46044616469021684681
:10DF500009F083FD0023002CC8BF684609DD55F891
:10DF6000231056F82320514340F823105B1C9C4299
:10DF7000F5DC002368461A46002C05DD50F8221017
:10DF8000521C0B449442F9DC4FF0000C6246002C0A
:10DF900005DD55F82200521C84449442F9DC93FBC1
:10DFA000FCF024B070BD2DE9FF4FADF54F7D0D465F
:10DFB000064690469021684609F04FFD902124A81E
:10DFC00009F04BFD902186A809F047FD9021AAA8F1
:10DFD00009F043FD00F06CFA00F07EFA00F09CFAC4
:10DFE000074600F091FA044600F092FA7190FA4860
:10DFF0000068418A8591008ACE9098F8012098F8AF
:10E000000000F649729102FB040090394891285CA7
:10E0100000F03F0A98F80C00499098F80D3098F8F5
:10E020000FB098F80E105B459CBFE8460DF1900EBE
:10E0300023D8499A03FB04F01FFA80F98A4218D8C2
:10E0400009EB020036F910C0285C00F03F00504593
:10E050000BD1BC4509DB58F82200604448F8220087
:10E060005EF8230060444EF82300501C82B28A42BE
:10E07000E6D9581C83B25B45DBD900216A460846C5
:10E08000002C7CDD52F82030401C1944A042F9DB02
:10E09000002974DD0021719A24AB0846002A6EDD48
:10E0A00053F820C0401C61448242F9DC002966DD3F
:10E0B00069462046489AFFF744FFDFF82493054657
:10E0C00099F80300D8BB489EA04606EB8804EB46AF
:10E0D00054F804ACA422C34948A8376809F061FC8D
:10E0E00048A9CB2D0ADC7B2D01DC282015E0C5F1E9
:10E0F000CB0000EBD07040101ED40EE042F2347022
:10E10000A84219DC42F284708542EEDAA5F51C5073
:10E11000343800EBD07040100ED451F82000324655
:10E12000391A316054F8041C084444F8040C594668
:10E130004046FFF706FF0546376044F804AC24A9C3
:10E14000729A7198FFF7FDFE99F80310E9BBDDF8AC
:10E15000C491729E044606EB89070DF1900B57F8A7
:10E1600004ACF422A04948A8D6F8008009F019FCB4
:10E1700048A9642C08DC282C02DC3C2010E037E0A5
:10E18000D4F164001CD40BE041F21460A04217DC0F
:10E1900041F250608442F0DAA4F5B05014380FD444
:10E1A00051F820003246A8EB0001316057F8041CFA
:10E1B000084447F8040C59464846FFF7C2FE044697
:10E1C000C6F8008047F804AC2046002DB8BF0025F3
:10E1D0000028B8BF0020CE99491E8D42C4BFCE99F9
:10E1E0004D1E8599491E8842C4BF8598401E01E096
:10E1F00000252846D2990D80DC9908800DF5537DC5
:10E20000BDE8F08F10B4794992B0B1E81C108DE8E8
:10E210001C10B1E81C10CDE90423CDE9064C51F8DF
:10E22000042B0892B1E81C10CDE90923CDE90B4C71
:10E23000B1E81C10CDE90D23CDE90F4C096811910F
:10E240000479B0F8B42041786B460DF1240C012C10
:10E2500005D0B0F93640B4F5E17F18DD07E0B0F93C
:10E260003440B4F52F7F02DC0478142C07D833F83F
:10E2700011101144A0F8B41012B010BC70473CF853
:10E2800011101144A0F8B41012B010BC70470478FB
:10E29000142CF4D8EBE72DE9F04F83464E488A461C
:10E2A00083B00168144691F8560091F8551000F0BB
:10E2B0007F0901F07F08C709CE0900F0F9F800F0E6
:10E2C0000BF900F015F9014694F85B00C0EB401023
:10E2D00001EBC00500F01CF902A8009001AB22463A
:10E2E00051465846FFF75FFE09EB890008EB8801AD
:10E2F000C0B2C9B2002F1CBF4042C0B2002E1CBF2A
:10E300004942C9B2BDF80420104480B2A4F8B40058
:10E31000BDF808201144A4F8B61095F8E0100129C2
:10E3200004BF94F8E11001290BD1B5F8B410401ADC
:10E33000FA2802DD2A78032A1DD3642801DD287813
:10E34000C8B194F8F30001210222022820D003284A
:10E350001CBF03B0BDE8F08F84F8F51095F8F50008
:10E3600001282DD0022812BF0328032084F8F500CD
:10E3700003B0BDE8F08FA1F1C80000B20028B8BF1B
:10E380000020A4F8B400B5F8B600A4F8B600D8E7A9
:10E3900084F8F51094F8E00000281CBF03B0BDE835
:10E3A000F08F94F8EA0000281FBF94F8ED000028D1
:10E3B00003B0BDE8F08F84F8F52003B0BDE8F08F1E
:10E3C00094F8EA00002804BF94F8E0000028F2D096
:10E3D00003B0BDE8F08F000060070020B07E002091
:10E3E00048070020989511003C96110030971100C5
:10E3F00010B5044600F05CF800F07AF8014694F895
:10E400005B000222C0EB401001EBC001012084F848
:10E41000F40094F8F50002280FD0032818BF10BDAF
:10E4200091F8F400022811BF0328032084F8F400B7
:10E4300010BD94F8E20028B110BD94F8E200002865
:10E4400018BF10BD84F8F42010BD10B51446FFF7B6
:10E4500022FF00F02DF800F04BF894F85B10022238
:10E46000C1EB411100EBC101012084F8F40094F8E4
:10E47000F50002280FD0032818BF10BD91F8F40052
:10E48000022811BF0328032084F8F40010BD94F87B
:10E49000E20028B110BD94F8E200002818BF10BDBA
:10E4A00084F8F42010BD0000FE487047FE48704715
:10E4B000FE48FF49007800EB001000EBC00001EBC4
:10E4C00080007047F948FB494078C0EB401000EBF2
:10E4D000800001EB00107047F448F549007880F0A7
:10E4E000010000EB001000EBC00001EB8000704762
:10E4F000EE48F049407880F00100C0EB401000EB9E
:10E50000800001EB00107047E84880684079704750
:10E51000E648806800797047E4488068B0F90C00EC
:10E52000704710B4E44991B0B1E81C108DE81C109C
:10E53000B1E81C10CDE90423CDE9064CB1E81C106C
:10E54000CDE90823CDE90A4C91E80E100CAC84E823
:10E550000E103DF9100011B010BC7047D34800797F
:10E56000C0F3C0007047D1480179C1F3C001002950
:10E5700012BF19208068B0F90E007047CB480178AF
:10E5800081F0010101707047C848417881F00101B4
:10E59000417070474FF41B6109F05FBA4FF4197175
:10E5A00009F039BA2A2109F036BAC04910B5886095
:10E5B000FFF799FBBDE8104001F09DBBBB48017817
:10E5C00081F001010170417881F0010141707047D3
:10E5D000B64988707047B54880787047B349C870AD
:10E5E0007047B248C0787047B04948607047AF483C
:10E5F00040687047AD488168497A11F0010F12BF39
:10E6000000204068C0F300707047A8480079C0F34C
:10E6100080007047A5484068C0F380607047A348F9
:10E620000079C0F3C0107047A0480079C0F3001013
:10E6300070479E4900200A7912F0040F08BF704706
:10E640008978092914BF0A290120704700209749B9
:10E65000974A097801EB011101EBC10102EB81013D
:10E66000897A022908BF012204D00022032908BFA9
:10E67000012300D000231A4305290CBF01210021EA
:10E68000114318BF012070472DE9F0410546874826
:10E690004FF41071806806794479824809F0DDF9F9
:10E6A0000027002E8CBFDFF8FC81BDE8F08101213E
:10E6B000012C1ED907FB041082B205EB420035F98C
:10E6C00012C030F9020CB0EB0C0348BFACEB0003F6
:10E6D0001BB2C82BC8BFC823DBB208F8023001291F
:10E6E00004BF08EB020000F8013C481CC1B2A14283
:10E6F000E0D3781CC7B2B742D9D3BDE8F0812DE989
:10E70000F04FADF24C5D05460020684ECDF8300567
:10E71000CDF81C05CDF82805B06890214479007922
:10E72000CDF834050DF5906009F097F90020CDF88B
:10E730001805CDF82405CDF82C054FF490616846F6
:10E7400009F08BF930785A4900EB001000EBC0005B
:10E7500001EB8000CDF83C05DDF83405671E4FF075
:10E76000000C002840F3758100200CFB04F1CDF86B
:10E770002005CDF8380535F9119005EB4101064625
:10E78000CDF88094B246B1F90290D04602460346D5
:10E79000C646B9F1000FB8BFC9F10009B1F90410BC
:10E7A0000029B8BF494289441921B1EB690FC4BFA0
:10E7B0000121CDF838150121012C2CDD0CFB0419A9
:10E7C0000DF5906B35F9199001FB01AA09FB01EEDB
:10E7D0004BF821900E44C84419F13C0F06DADDF8DD
:10E7E0001CB50BF1010BCDF81CB508E0B9F13C0FDD
:10E7F00005DDDDF830B50BF1010BCDF830B5B9F121
:10E800000A0F05DDDDF82C9509F10109CDF82C95ED
:10E81000491CA142D2DB07FB0EF106FB1811CDF813
:10E82000141507FB0AF106FB1611CDF8101500218F
:10E83000002C7CDDDDF8149507FB09F9CDF8449533
:10E84000DDF8109509FB07F9CDF84095DDF8449502
:10E850000CFB041A09FB01FBDDF8109509FB08BB52
:10E86000DDF8149509FB16B9DDF840B599FBFBF905
:10E8700035F81AB0ABEB09090FFA89F92DF81A909F
:10E8800035F91AA0BAF1000F1DDA002956DD19F189
:10E89000320F3CDA0DF5906E6FF01D0B4EF821B083
:10E8A0000CE0000094970020407F002058070020D3
:10E8B0006A7F002034840020789711004FF0010B0C
:10E8C000CDF820B523E00029C8BFB9F1320F0ADD29
:10E8D0000DF5906E4FF01E0B4EF821B04FF0010B6E
:10E8E000CDF820B513E0DDF838B5BBF1000F18BF47
:10E8F000BAF1640F09DD0DF5906E4FF01E0B4EF866
:10E9000021B04FF0010BCDF820B5002916DDB9F18B
:10E91000000FB4BFC9F1000BCB46BAF1000FB4BF72
:10E92000CAF1000ED646F34508DD521C00E00CE0AB
:10E93000B9EB0A0B48BFAAEB090B584419F1280F91
:10E94000B8BF5B1C491CA14280DBDDF82015012902
:10E9500069D100231E46B246D0461A461846C14623
:10E96000012C0CDD0DF5906B01FB01AA5BF821B0C9
:10E970000E440BFB0199491CD8448C42F2DC07FB86
:10E9800009F106FB1811CDF8141507FB0AF106FB77
:10E9900016114FF00009CDF81015002C43DDDDF8FD
:10E9A00014157943CDF83815DDF810157943CDF8F5
:10E9B0002015DDF838150CFB049A01FB09FBDDF886
:10E9C0001015B9F1000F01FB08BBDDF8141501FBB0
:10E9D00016B1DDF820B591FBFBF135F81AB0ABEBC1
:10E9E000010109B22DF81A1015DD0029B4BFC1F1DB
:10E9F000000B8B4635F91AA0BAF1000FB4BFCAF16B
:10EA0000000ED646F34506DD521CB1EB0A0B48BF9B
:10EA1000AAEB010B584411F1280FB8BF5B1C09F198
:10EA20000109A145C5DBDDF818150CF1010C1144F5
:10EA3000CDF81815DDF824150844CDF82405DDF8C7
:10EA400028051844CDF82805DDF834058445FFF67F
:10EA50008BAEDDF83C05B0F902002438402807D21F
:10EA6000DDF82C05FA28BCBF0DF24C5DBDE8F08F37
:10EA7000DDF81C0514280AD9DDF81C15DDF8280579
:10EA8000B0EB910F15D8DDF83005002811D0DDF876
:10EA90001805142807DDDDF81815DDF8240590FBAE
:10EAA000F1F0322805DC4FF490626946284608F000
:10EAB00033FF0DF24C5DBDE8F08F70B5044614488D
:10EAC0000D4614494078C0EB401000EB800001EB8C
:10EAD00000104FF41B6108F0C0FF2046FFF70FFE47
:10EAE0002046FFF7D1FD2946204602F0E4FD06F05E
:10EAF0007CF8204604F05DFF2946204603F049FCDF
:10EB00000146204600F044FFBDE8704004F09DB887
:10EB1000580700203484002070B5FFF7C9FC044674
:10EB2000FFF7DAFC0546FFF7C1FC064602F0EAFDF6
:10EB30002046FFF733FD2846FFF730FD3046BDE89D
:10EB40007040FFF72FBD2DE9F0410446FFF7B0FC00
:10EB50000546FFF7C1FC0646FFF7A8FC074620461E
:10EB6000FFF723FD02F0CEFD2846FFF717FD3046E4
:10EB7000FFF714FD3846BDE8F041FFF713BD70B54F
:10EB8000FFF796FC0446FFF7A7FC0546FFF78EFC4F
:10EB900006462046FFF702FD2846FFF7FFFC3046F9
:10EBA000FFF700FDBDE8704002F0ACBD70B5044653
:10EBB000FFF7AEFC0646FFF7A7FC0546FFF778FC1B
:10EBC000237AA27A217B94F80EC00024934298BF46
:10EBD000614507D98471691E0172C471711E417249
:10EBE000C47406E083710272C17180F809C001210A
:10EBF000C1748472C4730474447470BD10B5044647
:10EC0000FFF782FC14234FF0000C002C1CBF0021E6
:10EC100000280ED934F91120002AB8BF524292B20E
:10EC20009A4202DD4FF0020C03E0491CC9B2814256
:10EC3000F0D3604610BD2DE9F04700261746884600
:10EC400081463546FFF734FC0446FFF745FC034692
:10EC500009F0FF00022818BF012807D0042818BFB8
:10EC6000072803D0987A022815D021E00221A1724A
:10EC70000121E172042808BFA173012808BF84F8AC
:10EC80005812072808BF84F861120126187B2073E8
:10EC90003046BDE8F087587C48B9187B012806D07B
:10ECA00077484068B84203D2D87A012800D10225BB
:10ECB000A572002D0CBF0020D87AE07218BF012683
:10ECC00084F85882E2E770B50546FFF7F1FB044689
:10ECD000FFF702FC29886180E969097C2170E969F4
:10ECE000897C617090F85A1284F85A12017D21755E
:10ECF00090F85D1284F85D12407D28B16049097872
:10ED00003C293CBF607570BD0020607570BD2DE969
:10ED1000F04115460E460746FFF7CAFB0446FFF7CB
:10ED2000C5FB0023002F04BF84F85A3280F8283036
:10ED3000207C534A002818BF93600FD0A07D012883
:10ED400004BF1370BDE8F0811078401CC0B2107091
:10ED50003C2824BF3C201070BDE8F0819068401C26
:10ED60009060A842EAD99560237584F85D32012E3F
:10ED7000E4D1A372E37284F858322373DEE72DE9FD
:10ED8000F05F00259B4691460E4680462C464FF08C
:10ED9000140AFFF78DFB07464046FFF725FC38466F
:10EDA000FFF7FCFB18F0010FA84648D0F069FFF709
:10EDB000FDFE524658460A99FFF73DFF8346FFF78E
:10EDC00077FB0546FFF788FB31886980F169097C8C
:10EDD0002970F169897C697090F85A1285F85A1285
:10EDE000017D297590F85D1285F85D12407D28B18E
:10EDF000234909783C2938BF687501D385F8158007
:10EE0000D6E90201FFF759FE054652465946FFF77B
:10EE10007EFF787D002818BF0824B87A022808BF32
:10EE200044F02004787B012808BF44F0100497F8D0
:10EE30006002012808BF44F04004FFF7BFFB1148FF
:10EE40000560B7F902105A29C6BF397C4160C0F885
:10EE500004808460C9F800002846BDE8F09F0120C6
:10EE60007047012070470120704701207047044817
:10EE70004078704702494870704700207047000092
:10EE800064070020D49900204FF6FF71A0F8B41059
:10EE9000A0F8B610A0F8B810A0F8BA10A0F8BC10EE
:10EEA000A0F8BE10A0F8C010A0F8C21070472DE95D
:10EEB000F04F85B0FFF706FB0490FFF7F9FA002545
:10EEC0002C460090FFF720FB0098007D01280CBF26
:10EED0004FF4DE71DE210098F84A4FF00008407CC4
:10EEE000012888BF82F800801CBF05B0BDE8F08F04
:10EEF0004FF000070098007C00289CBF05B0BDE8DB
:10EF0000F08FC7EB4712049800EBC20090F8F4C0F2
:10EF1000BCF1020F18BFBCF1030F40F07E81E74E39
:10EF20003278039252B3E64BF278029233F822B071
:10EF3000B0F8B630BBEB030954BF4A46A3EB0B0253
:10EF40008A42B8BF0124DFF87CA3DC4A127901921F
:10EF50003AF822A0B0F8B420BAEB02064CBFA2EBFC
:10EF60000A0EB6468E45B8BF0125BCF1020F1ED071
:10EF7000BCF1030F00F0F38000F0DFB8BCF1020F2A
:10EF800040F04B810122CE4B3270B0F8B6C0A3F8EE
:10EF900000C05A80B0F8B430CA4803804280727012
:10EFA000B27086F8038086F8048000F036B954EA1F
:10EFB000050C04D0002C71D0002D6ED0BDE0BF4EEA
:10EFC0004FF0000AD44696F80190B9F1000F88BFBF
:10EFD000DFF8ECE228D93EF82CB0BBEB030648BFC3
:10EFE000A3EB0B068E4216DAB44E86F803C0019AE4
:10EFF000521CD2B23271B3785B1CDBB2B3700F2BF0
:10F0000028BF86F8008080F00881AE4B03EB8202B7
:10F01000A2F8028091E00CF1010C0CF0FF0CCC4541
:10F02000D9D3BAF1000F51D1DFF890C200239CF878
:10F0300002B0BBF1000F88BFDFF888E228D93EF8A4
:10F040002360B6EB020C48BFA2EB060C8C4518DA25
:10F05000DFF868C28CF80430029A09F10103521CEF
:10F06000D2B2DBB28CF803208CF801300A2B02D329
:10F070008CF80080D1E0924B03EB8202A2F8028070
:10F080005BE05B1CDBB25B45D9D3BAF1000F54D116
:10F090008A4880F80080C0E000E02EE0DFF81CE243
:10F0A0004FF0000A52469EF80190B9F1000F88BF58
:10F0B000DFF80CB212D93BF82260B6EB030C48BF64
:10F0C000A3EB060C8C4502DA8EF8032035E0521CC7
:10F0D000D2B24A45EFD3BAF1000F2ED1029A09F10C
:10F0E0000103521CD2B2DBB28EF803208EF801303D
:10F0F0000A2BC0D38EF800808FE0DFF8C0E14FF01C
:10F10000000A53469EF80290B9F1000F88BFDFF85D
:10F11000B4B117D93BF82360B6EB020C48BFA2EBA1
:10F12000060C8C4502DA8EF8043006E05B1CDBB27C
:10F130004B45EFD3BAF1000F04D0039A5F4E012A7A
:10F140001FD06AE0019A09F10103521CD2B2DBB26E
:10F150008EF804208EF802300F2BCBD255E7DFF863
:10F160005CC1B9F1000F48BFA3EB0B098945BFF69D
:10F170007FAF002E48BFA2EB0A068E42BFF678AFE3
:10F18000DBE7DFF83C91F27809EB820CBCF8023047
:10F19000F3B342F2107A53450DD2B0F8B6A039F865
:10F1A00022B00BFB03AA5B1C9BB2ACF80230BAFB8B
:10F1B000F3F329F8223039F82230B0F8B6209B1A40
:10F1C00003EBD37302EB6302A0F8B620DFF8F490F0
:10F1D000327909EB820CBCF8023083B342F210762C
:10F1E000B3420DD2B0F8B46039F822A00AFB03662E
:10F1F0005B1C9BB2ACF80230B6FBF3F329F822306B
:10F2000039F82230B0F8B4209B1A03EBD37300E036
:10F210000DE002EB6302A0F8B420781CC7B200989E
:10F22000007CB8423FF66DAE05B0BDE8F08FB0F897
:10F23000B63029F822300122ACF80220C6E7FFE7F9
:10F24000B0F8B40029F822000120ACF80200E4E78D
:10F250002DE9F047FFF736F90446FFF729F9024692
:10F26000007D01280CBF4FF4DE707820517C164DD4
:10F270000026A5F10C07012907D098BFBDE8F0874B
:10F280003E722E806E80BDE8F08792F810C04FF07D
:10F290000001BCF1000F98BFBDE8F087C1EB41123F
:10F2A00004EBC20292F8F430022B18BF032B0DD0EE
:10F2B000491CC9B28C45F1D8BDE8F0877007002021
:10F2C000E0990020089A00207C0700203B7A012B5F
:10F2D00012D0002BF0D1C1EB411004EBC00090F82C
:10F2E000F4000228E8D101203872B2F8B400288076
:10F2F000B2F8B6006880DFE7C1EB411304EBC3034B
:10F30000B5F80090B3F8B430B5F80280A9EB030368
:10F310000FFA83FCB2F8B630BCF1000FA8EB030380
:10F320001BB2B4BFCCF1000AE246504538DB002BDB
:10F33000B4BFC3F1000A9A46824531DC92F8F4006A
:10F34000022815D042F6AB200CFB00F00114A1EB13
:10F35000E07142F6AB2058430314A3EBE070A9EB35
:10F360000101A2F8B410A8EB0000A2F8B600A3E7D0
:10F3700046F267600CFB00F04114A1EBE07146F22D
:10F38000676058434314A3EBE073A9EB0100A2F8B4
:10F39000B400A8EB0301A2F8B610288069808BE7BF
:10F3A0003E722E806E8096E72DE9F04F83B0FFF716
:10F3B00089F80446FFF77CF80746FFF7A5F80190A7
:10F3C000FFF7A6F80090787CFE4E01254FF0000A6A
:10F3D00001280DD09CBF03B0BDE8F08F757186F891
:10F3E00007A003B04FF00100BDE8F04FFEF740BCAE
:10F3F0007079A8B1397C002000299CBF03B0BDE81A
:10F40000F08FC0EB401204EBC20292F8F420022A03
:10F4100072D0401CC0B28142F3D803B0BDE8F08F77
:10F4200097F810B00023BBF1000F9CBF03B0BDE8FC
:10F43000F08F4FF0020EDFF8908308F10609C3EB5E
:10F44000431004EBC00191F8F320022A05D0032AEF
:10F4500004BFB079022830D076E0C3EB431214F831
:10F460003220012A16D9019B9B1E9A4212DA04EB24
:10F47000C0025278012A0DD9009B9B1E9A4209DADC
:10F48000757186F807A00120FEF7F2FBB57103B095
:10F49000BDE8F08F04EBC00086F806E0B0F8B400D9
:10F4A000A9F80000B1F8B600A9F8020088F800A099
:10F4B00088F801A003B0BDE8F08FB9F80000B1F8FA
:10F4C000B470B1F8B6C0C21BB9F80200A0EB0C01D1
:10F4D0004CBF50421046F02818DD98F8000020B1CB
:10F4E00001280AD002280CD00EE0002AB4BF88F808
:10F4F000005088F800E007E02EE0002A3FF76EAFEA
:10F5000002E0002AFFF66AAFA9F800700029B4BF34
:10F5100048420846F02817DD98F8010020B101287C
:10F5200009D002280BD00DE00029B4BF88F80150A3
:10F5300088F801E006E000293FF750AF02E000291B
:10F54000FFF64CAFA9F802C0581CC3B29B453FF66A
:10F5500076AF03B0BDE8F08F86F807A003B0BDE832
:10F56000F08F2DE9F041044698480068C68A858AE4
:10F57000FEF7BEFF034694F8F4004FF0000C02289B
:10F5800023D0032818BFBDE8F081207903281CBFD1
:10F59000B4F8C0000A2898BFBDE8F081A6F10B01BD
:10F5A0008842A8BFBDE8F081B4F8C2200A2A98BFFB
:10F5B000BDE8F081A5F10B008242A8BFBDE8F08153
:10F5C00094F8E720012A46D066E07E490122487976
:10F5D0000028B4F8C0001BD00A280DD9A6F10B03EF
:10F5E000984209DAB4F8C2000A2805D9A5F10B033C
:10F5F0009842B8BFBDE8F08181F808C084F8E720E0
:10F600004A7181F807C0BDE8F0410120FEF730BB28
:10F610000A280DD3A6F10B03984209DCB4F8C20006
:10F620000A2805D3A5F10B039842D8BFBDE8F081A5
:10F6300081F808C084F8E7202079032808BFBDE8D6
:10F64000F08184F8E8204A7181F807C0BDE8F041F4
:10F650000120FEF70DBB94F85B200B27C2EB421292
:10F6600003EBC202B2F8C0300A2B98BFA4F8C070F6
:10F6700005D98B42A4BFA6F10C01A4F8C010B2F8C2
:10F68000C2100A2998BFA4F8C27005D98142A4BF4C
:10F69000A5F10C00A4F8C20084F8E7C0BDE8F08131
:10F6A0002DE9F04FADF5197DFEF70CFF9390FEF7B5
:10F6B000FFFE0646FEF710FF0446FEF719FF929084
:10F6C00006F1170004F117059090FEF71DFF0027C3
:10F6D0009190307C3C463B4600287DD99398C3EB03
:10F6E000431100EBC10191F85B00C0EB401292980E
:10F6F00000EBC20991F8E30001286ED191F8F30004
:10F70000022818BF032868D1601CC4B291F85920A0
:10F710002F4800EB820C3CF8048CA8F57F40FF38A2
:10F720001FBF3CF8022CA2F57F40B0F1FF0040461D
:10F7300004BFB9F80600B9F80820B1F80690CDF872
:10F74000549209F1050ADFF88C90A9FB0ABACAF3B2
:10F75000CF0ECDF860E2B1F808E0CDF850E20EF13E
:10F76000050AA9FB0ABACAF3CF0ACDF85CA200F1D8
:10F77000050AA9FB0ABACAF3CF0B02F1050AA9FBD5
:10F780000AA9C9F3CF0ADDF854924CF6CD4E09FB15
:10F790000EF94FEAD949CDF85892DDF850E24CF60F
:10F7A000CD490EFB09F94FEAD949CDF854924CF6F0
:10F7B000CD4900FB09F94CF6CD4E4FEAD94902FB81
:10F7C0000EFE0BE0700700207A0700206007002083
:10F7D000449A0020CDCCCCCC30E027E04FEADE4E7E
:10F7E000CDF850E2DDF860E2DE4504BFDDF85CB242
:10F7F000D34507D0DDF858A2CA4504BFDDE9949A85
:10F80000CA4513D17F1CDFF8F0924FF6FF7AFFB2A2
:10F81000D04504BF3CF8028CD04507D12CF8040C2D
:10F8200091F8590009EB800020F8022C581CC3B253
:10F83000307C98423FF652AFA7427DD1707C0228BF
:10F840007AD3AE49487A401CC0B248721E283CBFE9
:10F850000DF5197DBDE8F08F1E2048724FF410722F
:10F860006846909908F058F8307C4FF0000B00285B
:10F8700070D99398CBEB4B1100EBC10191F85B0071
:10F88000C0EB4012929800EBC20291F8E30001280D
:10F8900059D191F8F300022818BF032853D10B78EF
:10F8A00091F801C091980CFB00339098C05C0B7BE1
:10F8B00000F03F0A107B984238BF0873507B4B7BA7
:10F8C000984238BF4873907B8B7B984288BF88737F
:10F8D000D07BCB7B984288BFC873087B95904C7BCC
:10F8E0009494137892F801C0919A91F80F800CFBD0
:10F8F0000232887BAA5C444502F03F091AD8919AEB
:10F90000624397B2959A824210D8BB1815F803C08B
:10F910000CF03F0ECE4505D12CF03F0C4CEA0A0C02
:10F920000DF803C0521C92B28242EED9621C94B20E
:10F930004445E4D9959A00E016E00A73949A4A7314
:10F94000887381F80F800BF1010000F0FF0B307C11
:10F9500058458ED84FF410726946909807F0DCFF36
:10F960000DF5197DBDE8F08F64480021624A4172AF
:10F9700008464FF6FF7122F8201002EB8003401C6E
:10F98000C0B259800A28F6D30DF5197DBDE8F08F75
:10F990002DE9F05F8B468246FEF794FD0746FEF7A1
:10F9A000A7FD8046FEF784FD0546BBF1000F72D12E
:10F9B000287C05F1170900287BD0FFF771FE287C11
:10F9C0000024002888BF4FF6FF7620D9C4EB4410EE
:10F9D00007EBC00292F8E300012813D1A2F8B4604B
:10F9E000A2F8B660A2F8B860A2F8BA60A2F8BC604B
:10F9F000A2F8BE60A2F8C060A2F8C26049465046B4
:10FA0000FEF723FD601CC4B2287CA042DED800268D
:10FA100010F0FF0F1CBF4FF000094FF0020A48D052
:10FA2000C6EB461007EBC00494F8F400022818BF98
:10FA3000032806D094F8F500022818BF03282BD01D
:10FA400032E0204600F017FF94F89D0001282BD1EA
:10FA500094F85B00C0EB401008EBC00090F8F41085
:10FA6000022918BF03291FD1B430B434B0E80E10F6
:10FA7000A4E80E10B0E80E10A4E80E1070E83512DD
:10FA8000D0F8DC0044F8D419C4E9362084F884A006
:10FA900084F8649008E00CE0B4F8B400A4F8B8006E
:10FAA000B4F8B600A4F8BA00701CC6B2287CB04204
:10FAB000B6D8287C0024002898BFBDE8F09FC4EB8E
:10FAC000441007EBC00090F8E31001290CD190F826
:10FAD000F310022918BF032906D190F8EC10002971
:10FAE00004BF594601F0AFF9601CC4B2287CA042A3
:10FAF000E5D8BDE8F09F0000449A00207007002080
:10FB0000F7484078002818BF01207047F548006882
:10FB100090F8580000F001007047F24909688A6DBA
:10FB200060F300028A657047EE4B10B4D3F800C052
:10FB3000BCF8123003FB00F4BCF81A005943B4FBC4
:10FB4000F0FCB1FBF0F10CFB0CF4DFF89CC3494373
:10FB5000CCE9084103FB02F1B1FBF0F04043CCF8E3
:10FB6000280010BC70474FF6FF7202EA0023DE48FF
:10FB700002EA0121C38501864FF4A0514186491054
:10FB8000818670472022D84906280ED2DFE800F08F
:10FB90000D030D05080A102000E0402088857047FD
:10FBA0008020FBE74FF48070F8E78A85704700B546
:10FBB00002220A210C20FFF7B7FFDFF828C30A232F
:10FBC0001422DCF8000090F85C00C0F3031100F090
:10FBD0000F00FFF7C8FFDCF80000B0F85C005DF82C
:10FBE00004EBC0F30330CDE72DE9F04190460D461C
:10FBF0000446FEF75DFCBD48BA4E47190A38054475
:10FC0000BCB1012C3AD0022C4DD0032C18BFBDE85A
:10FC1000F08104220E210F20FFF786FF30680A23AF
:10FC20001422B0F85C00C0F303200146FFF79BFFED
:10FC30001CE002220A210C20FFF776FF15F8010CC8
:10FC4000002801BF17F8010C002898F8F3000328DA
:10FC500030684FF00A034FF0140290F85C00C0F3D4
:10FC6000031100F00F00E1D1FFF77DFF3068B0F81D
:10FC70005C00BDE8F041C0F3033083E702220E21AF
:10FC80000F20FFF751FF30680A231422B0F85C0000
:10FC9000C0F3032100F00F00491CFFF764FFBDE82B
:10FCA000F04104206EE715F8010C012804BF17F895
:10FCB000010C01284FF0040219BF112112200C2160
:10FCC0000D20FFF731FF15F8010C02283068C06DD8
:10FCD00018BFC0F30351C0F303404FF00A034FF0C5
:10FCE000140208BF0321FFF73EFF3068C06DBDE876
:10FCF000F041000F46E730B57A4C794D022220687A
:10FD0000418A408B8900B1FBF0F04043A8600A2192
:10FD10000C20FFF709FF20680A23142290F85C00EA
:10FD2000C0F3031100F00F00FFF71DFF2068B0F8CB
:10FD30005C00C0F30330FFF725FF05F110014FF61B
:10FD4000FF700880488005F10C004FF0FF31018002
:10FD500041800020287030BD634B03EB40000389D5
:10FD60008B4288BF991A38BF991808BF7047018124
:10FD700070472DE9F04F83B09B460D460446FEF7D1
:10FD800097FB0190FEF7B4FB0246564894F859A041
:10FD9000DFF84CE10068544B418A408BC1EB011104
:10FDA000890091FBF0F000FB00F194F8F4000228C8
:10FDB00011D0A3F1500000EBCA0050E9026794F89B
:10FDC0005800B5F800800228B5F8029094F8DC00DD
:10FDD00014D028B332E0002003EB0A0C2E886F8881
:10FDE0000CF8010C03EB4A08B3F834C0A8F808C0BB
:10FDF000BAF1010F08BF8EF80100E0E7F0B194F806
:10FE00005B00C0EB401002EBC00090F8DC00A8B92A
:10FE100003EB4A001A8EB0F808C094450ED90CE0E6
:10FE20008B4524BF94F8F400032807D103EB4A0064
:10FE30001A8EB0F808C0944500D9028120790228B2
:10FE400018BF032806D094F8DC0018B98B4538BFDA
:10FE5000988E00D3588E588694F8DCC0BCF1000F01
:10FE600008D194F8F4008B4502D2032813D101E0A5
:10FE7000022810D060469A6A5A4588BF0220009036
:10FE80009EF801100122002904BFBAF1010FBCF154
:10FE9000030F0BD101E00220EDE713488EF801209B
:10FEA0004189188E814284BF0F4948810E4B0C99BD
:10FEB0000098D3F820C0DC4503D8022801D00129DE
:10FEC00008D0094B4FF0020E5A6A5A4510D9022841
:10FED0001ED10DE00448504400F8012C24E000003D
:10FEE0008407002060070020BC9A0020FE9A0020B2
:10FEF00071B15A4598BFE3450FD202280FD003EBEA
:10FF00000A0010F8011C032908BF00F801EC0BE0FF
:10FF100003EB0A0000F801EC06E0022804D103EB31
:10FF20000A00032100F8011CFEF7C2FAFE4B8646C8
:10FF300003EB0A02988D12F8012C198EB3F82EB03B
:10FF4000B3F832C0022A04D0012A1CD0032A6DD093
:10FF500032E003EB4A0201EB410CB2F808B0E34592
:10FF600006D99EF80AB0BBF1000F08BFA2F808C07E
:10FF7000B2F808C08C4588BFACEB000038BF6044C5
:10FF80001AD0108118E003EB4A0CBCF8082091420B
:10FF90000AD2501AA2EB6000000A4FF6FF7101EA84
:10FFA0000020ACF8080007E05A4588BF101A38BF97
:10FFB000104401D0ACF8080003EB4A000289002A83
:10FFC00004BF002001461FD01046B2F5807F36BF27
:10FFD0004FF4807101464FF48072D448009B022B8D
:10FFE0002ED094F859C000230CF80030A1F5807091
:10FFF000704300EB0820B0FBF1F0A2F5807179436B
:020000021000EC
:1000000001EB0921B1FBF2F194F85930C84A02EB37
:10001000C30343F8080C94F8593002EBC30242F8CA
:10002000041CA880E98003B0BDE8F08F03EB4A020E
:100030001189614588BF081A38BF0844A1D1BBE7C0
:1000400094F859C01CF80030FA2B3CBF5B1C0CF82C
:10005000003094F85930185C3C28C7D30198090A3D
:10006000120A407C0228B348006818D3B0F818A0E0
:10007000B0F81AC00AFB08F3B0F810800CFB09F9BD
:10008000408AB3FBF8F30AFB06FA0CFB07FCB9FB4A
:10009000F0F9BAFBF8F8BCFBF0FCB34617E0B0F897
:1000A00014A0B0F816C00AFB08F3B0F810800CFBDF
:1000B00009F9408AB3FBF8F30AFB06FA0CFB07FCCC
:1000C000B9FBF0F9BAFBF8F8BCFBF0FCB346A1F1C0
:1000D000010000FB0830B0FBF1F3A2F1010000FBCE
:1000E0000C90B0FBF2F293480168B1F8109009FB54
:1000F00003F009D3B1F81890B1F812A0B0FBF9F0F1
:100100000AFB02F9498B08E0B1F81490B1F812A08B
:10011000B0FBF9F0C98A0AFB02F9B9FBF1F14345DA
:1001200018BF62457FF470AF434508BF584662452B
:1001300008BF394668E72DE9F04F90F859C08FB0F5
:100140004FF4806300290CBF7B4C7C4C04EB4C14B7
:100150007B4D029205EB4C1705F5A5756544203CD7
:1001600015F8015C07EB051606EBC10858F8206C82
:10017000921B039290F8F40002287CD058F81C8C53
:1001800004EB051206EB0809CDF83090D2F8049084
:10019000D6689568106809EB0602DFF8A891284434
:1001A0001044D9F800A035445044D9F804A0524472
:1001B000D9F808A0D9F80C9055444E44DDF808A0B1
:1001C000DDF83090AAEB0909CDF82090DDF80C900D
:1001D000DFF874A1A9EB0809CDF82C90DAF80090AB
:1001E00009EB000ECDF828E0DAF80490DAF808B050
:1001F000DAF80CA09144B244AB440EFB0AFE09FBB2
:100200001BEE9EFBF3FEBEF1000F08BF4FF0010E88
:100210004FEA8A2A9AFBFEFA4FEA892999FBFEF9EE
:10022000CDF838A0C9F1000A4FEA8B29CDF834A0E7
:10023000DDF828A099FBFEF94FEA8A2A9AFBFEFB1B
:10024000DDF838A0C9F1000900FB0AFA02FB09AA8F
:100250009AFBF3FEDDF834A0CDF828E000FB0AFAA3
:1002600002FB0BAA9AFBF3FECDF824E0DDF838A0E0
:1002700005FB0AFA00E073E006FB09A999FBF3F914
:10028000DDF834A0CDF8389005FB0AF906FB0B9990
:1002900099FBF3FADDF828E0DDF820900EFB09FB6E
:1002A000DDF824E0DDF82C900EFB09BEDDF820B06F
:1002B000DDF838909EFBF3FE09FB0BFBDDF82C907C
:1002C0000AFB09B999FBF3F9C844DDF830B0DDF851
:1002D0003890F344CDE900B8DDF828E0C9F1000911
:1002E000CEF58068DDF824E0CAF5806ACEF1000B17
:1002F00008FB00FE0BFB05EE08FB02F809FB00F013
:100300000BFB06880AFB05009EFBF3FE98FBF3F847
:1003100090FBF3F0CDF810E0CDE9058009FB02F089
:100320000AFB060012E00000BC9A0020B19B0020EE
:100330006C9A002060070020BC9B0020FC9C0020E1
:100340003C9E0020C0070020D007002090FBF3F067
:100350000022E84604AE0790FE4800EB0C0315E0CF
:10036000FC4A00206244039012F8012C02AB07EB18
:10037000021202EBC10253F8204002EB8005401C40
:1003800000B245F8204C0228F5DB20E013F8015CB0
:1003900058F8220007EB051505EBC10505EB8205B2
:1003A00045F8200C002006EBC20513F801AC55F807
:1003B000209004EB0A1A0AEBC20A4AF82090401C6B
:1003C00000B20228F1DB501C02B2022ADEDBE14857
:1003D000604410F8010C07EB001000EBC10050F86E
:1003E000200C0FB0BDE8F08F70B4012803BF0224C9
:1003F00001204FF0000C04241CBF03204FF0010C1F
:100400000026D54D0029C8BF204609D00CEB8C0131
:1004100005EB810101EB420121F8026C70BC7047D1
:10042000CE480CEB8C0100EB4100104405EB810140
:1004300001EB420210F8010C32F8021C642924BFBF
:1004400070BC7047491C22F8021C0121197070BC55
:1004500070472DE9F0010128DDE9055614BF0120A0
:10046000002000EB8000DFF8F4C20CEB400C8C4461
:100470001CF801CCBCF1000F04BFBDE8F0017047CF
:10048000DFF8DC82002408F13C07944531D1A7F164
:10049000280202EB800202EB410232F8022C9A425F
:1004A00007D908EB4000084400F8014CBDE8F00112
:1004B000704708EB40020A4412F8013C642B24BF49
:1004C000BDE8F0017047002E1CBFBDE8F001704789
:1004D0005B1CDBB202F8013C0A2B3CBFBDE8F0011B
:1004E000704707EB4000084400F8014CBDE8F001FC
:1004F000704708EB40020A4407EB400012F8013C49
:100500000844052B36BF10F8011C00F8014C642983
:1005100004D20A2DA4BF491C00F8011C02F8014CAA
:10052000BDE8F00170472DE9F04F89B08246088898
:10053000ADF8100048888946ADF81400FDF7B8FF03
:1005400000909AF8F4009AF85940022804BF204617
:1005500000F0D0FC8348874A2044089010F8015CE2
:1005600081488349204402F1080C00F8015C7F486F
:1005700000EB040818F8010CD8B1681CC0B21428AC
:1005800021D304EB840001EBC00000EB450330F8FD
:1005900028EC33F828BCAEEB0B0B02EB840E4EF8C4
:1005A00004BC1B8D008DC01A0CEB840343F8040CB3
:1005B00020E002EB8403002043F8040C0CEB8403DE
:1005C00043F8040C16E004EB840301EBC30303EBD4
:1005D000400030F8283C30F82ABCA3EB0B0302EBB8
:1005E000840B4BF8043C038DC08C181A0CEB84036D
:1005F00043F8040C04EB840001EBC000079000EB0F
:100600004500BDF8103020F8283CBDF814B0A0F823
:1006100028B0132D04BF012008F8010C9AF8F4004B
:1006200003284FD1002D1CBF681EC0B25AD00799B5
:1006300001EB400030F8281C008DA3EB010118F8F5
:10064000013CABEB00000193002B52D04A4B002938
:1006500003EB840656F8047CACBF0B464B4207EB19
:10066000030B464B46F804BC03EB8403002853F805
:1006700004ECB4BF47420746774402EB840243F8D8
:10068000047C52F8042C002AB8BF5242ABEB0202A1
:1006900046F8042C0CEB840252F8042C002AB8BF54
:1006A0005242BA1A43F8042C354A1268138B594344
:1006B000138A91FBF3F6518B4843518A90FBF1F773
:1006C000019878B32F4802212044069000F8011CBD
:1006D0002D4800EB040B0BF8011C9AF8DC000328F2
:1006E00061D15DE018F8010C01280CBF13202846E9
:1006F0009DE7214A002902EB840252F804CCB4BFE2
:100700004B420B46634442F8043C1C4A002802EB6F
:10071000840252F804CCB4BF43420346634442F817
:10072000043CC1E7FFE71948002E00EB440030F815
:10073000022CB4BF714231468A4205DA002EACBFAA
:100740003146714220F8021C4288002FB4BF794222
:1007500039461DE07C9F00207AA1002052A1002094
:1007600066A1002086070020880700208A07002055
:10077000089B002098070020B0070020B807002041
:1007800060070020F49A0020FE9A0020A8070020AD
:100790008A4297DA002FACBF39467942418091E70F
:1007A000FDF733FF68B1204600F0A4FBBDF8100050
:1007B000A9F80400BDF81400A9F8060009B0BDE8C6
:1007C000F08F18F8010C012803D0D8B9691C07294B
:1007D00018D3282ED8BF282F09DCFE4901EB44018D
:1007E00031F8022C282A9CBF4988282919D9009859
:1007F00090F85A02012805D10699032001F8010C4E
:100800000BF8010C0898089910F8010C401CC0B2B4
:1008100001F8010C1428C9D30899002001F8010C33
:10082000C4E7ED494FF0000C01EB840151F8042CB2
:10083000EA4901EB840151F8041C8A42C8BF4FF019
:10084000010C05A904AA1423CDE90003CDE9022176
:1008500007982B4600F12802A0F12801604600F01D
:1008600071FB01280CBF01200020069901F8010C42
:100870000BF8010CC6E72DE9F04F8DB00446FDF7EB
:1008800055F90490FDF755F90890FDF731FE8146C2
:10089000FDF70EFE079094F85960FDF709FE827A85
:1008A00094F859100127002A04BF427D002A06D17E
:1008B000027D012A1CBF90F85D22012A01D180F837
:1008C0005A7200258DF819508DF818708DF8175050
:1008D00090F85A02DFF808830028D8F800007DD08D
:1008E000826DC2F3C0438DF81430C2F340428DF8DC
:1008F0001520806D2246C0F380408DF8160002203E
:10090000FFF772F9B648D0F8008098F8580010F058
:10091000010F00F0438294F85B10B4F8B400ADF816
:100920000800B4F8B630C1EB411109EBC101ADF8D4
:100930000A300B9194F8591094F8F4C0A94A01EBCD
:100940004101BCF1020F02EB81017CD031F80AAC0D
:1009500021F808AC31F80C2C21F80A2C21F80C0CE9
:1009600031F8049C21F8029C31F806CC21F804CC23
:1009700021F8063C81B261F30F0062F31F409142FF
:1009800084BF62F30F0061F31F40010C514588BF23
:100990006AF31F4081B2020C914284BF62F30F00E0
:1009A00061F31F40000C63F30F016CF31F416345BB
:1009B00084BF6CF30F0163F31F410A0C4A4588BFE3
:1009C00069F31F418BB20A0C934284BF62F30F019B
:1009D00063F31F410B0CADF80C0000E00EE09DF836
:1009E0001410ADF80E30012904BFADF80800ADF8C1
:1009F0000A3094F8F40002283AD0AFE090F858207A
:100A0000C2F3C0038DF81430C2F340028DF81520F4
:100A100090F85820C2F380028DF816202279022A1D
:100A20001EBF032A224600207FF46AAF826DC2F304
:100A3000C0438DF81430C2F340428DF81520806D0C
:100A4000C0F3804000E006E08DF816002246022048
:100A5000FFF7CAF856E721F8080C21F80A0C21F82C
:100A60000C0C21F8023C21F8043C21F8063CB2E7CA
:100A70005D484FF0000C304400F8015C5B48019584
:100A8000304400F8017C5A4800EB46100A9059485F
:100A900000EB46100990584800EB46100090099969
:100AA000002001EB0C1E009901EB0C1B0A9901EBD5
:100AB0000C1900210EEBC0020BEBC00309EBC007C1
:100AC00002EB810A4AF8205C03EB810A4AF8205CB9
:100AD00007EB810A491C09B24AF8205C0229EFDBC6
:100AE000401C00B20228E4DB0CF101000FFA80FC8C
:100AF000BCF1020FD3DB019A0998DFF800E100EBAB
:100B0000021A0098002100EB02193D4A002002EB76
:100B1000C1070AEBC10C09EBC1050EEBC103814211
:100B200007D1B8F8622043F82020B8F8602047F8D1
:100B3000202053F820200CEB800B02EB82025200A5
:100B40004BF8202C05EB800B401C00B24BF8202CFE
:100B50000228E4DB481C01B20229D6DBBDF80820DC
:100B600000212046FFF7E7FA0546BDF80A200121DB
:100B70002046FFF7E0FA002DB8BF00250028B8BFD7
:100B80000020174F3968B1F91020531EAB42B8BF8F
:100B90001D46B1F912104A1E8242B8BF1046AAB2D1
:100BA00083B211481149ADF80C20ADF80E30304435
:100BB000314410F801CC11F8015C00F8015C01F837
:100BC00001CC9DF81600012804BFADF80820ADF84F
:100BD0000A3017E0A8070020B0070020B80700205F
:100BE00060070020909F00207C9F0020869F0020AF
:100BF0003C9E0020BC9B0020FC9C0020C0070020E5
:100C0000D007002020460B9900F08AFA94F858107B
:100C10000B98022918BF002529D0C4F8C450B4F895
:100C2000B410B0F8B420DFF86C84891AC4F8C81086
:100C3000B4F8B610B0F8B60008F10A09081AC4F8FA
:100C4000CC00022E9CBF9DF81700012823D008EB92
:100C50000601022001F8010C09EB060101F8010C64
:100C600008EB0601002011F8011CB1BB36E0B4F816
:100C7000B410B0F8B430CA1A48BF5A1AB4F8B63033
:100C8000B0F8B6C0B3EB0C0148BFACEB0301524364
:100C900001FB0125C1E72A4602A92046FFF743FCD4
:100CA000079890F85A020028DAD1FB48304410F82F
:100CB000010C012808D00028D2D1F848304410F89F
:100CC000010C401C1428CBD9BDF80C00ADF808006D
:100CD000BDF80E00ADF80A00C2E704E009EB06011A
:100CE00011F8011C01B10120009007982B4602A9C0
:100CF000427C2046FFF73DF89DF81500012840D0C2
:100D0000BDF80800A4F8B800BDF80A00A4F8BA00BD
:100D1000BDF80800049ABDF80A109042B8BF10460A
:100D2000089A9142B8BF11463A68049BB2F910C0C4
:100D3000ACEB0303A3F1010C8445B8BF6046B2F9E4
:100D40001230089A9A1A531E8B42B8BF194680B2C5
:100D5000A4F8B8008AB2A4F8BA200B99B1F8B81078
:100D6000411AC4F8D4100B98B0F8BA00101A4943CD
:100D7000C4F8D80000FB0010C4F8D0000DB0BDE8E6
:100D8000F08FBDF80C00ADF80800BDF80E10ADF8FE
:100D90000A10A4F8B800BDF80E00B7E7B4F8B40024
:100DA000A4F8B800B4F8B600A4F8BA000DB0BDE8D5
:100DB000F08FBB4A30B4146894F8542012F0040F3A
:100DC0001ABF012323EA020502F00105B0F900C0B1
:100DD000B1F900301DB1E58AEB1A5B1E1BB212F0AF
:100DE000020F06D0A48AA4EB0C0CACF1010C0FFA94
:100DF0008CFC12F0040F19BF0380A1F800C0A0F80A
:100E000000C00B8030BC7047A54A30B41268B2F8FD
:100E1000983013F0FF024FEA132308BF6422002B1F
:100E200008BF64230488B1F800C062439D4CA4FB52
:100E30000252520902800CFB03F0A4FB002040097F
:100E4000088030BC70472DE9F0470446944882B0D2
:100E50000068B0F818A0B0F81A90858AC68A078A88
:100E6000B0F812800020ADF80000ADF80400FDF7E6
:100E70001FFBB4F8B810B4F8BA0001FB0AF292FBF9
:100E8000F7F2A4F8BC2000FB09F292FBF8F26943E8
:100E9000704391FBF7F190FBF8F0A4F8BE20ADF899
:100EA0000010ADF8040001A96846FFF782FFBDF904
:100EB0000000711E8842A8BF084600B2BDF90410A8
:100EC0006A1EADF800009142A8BF114609B2ADF804
:100ED00004100028D8BF0020ADF800000029D8BFBA
:100EE0000021ADF80410A4F8C000A4F8C21002B0AC
:100EF000BDE8F087694A0021024402F8011C6A4AF1
:100F0000024402F8011C644A024402F8011C674AC8
:100F100002EB800242F8041C654A02EB800242F8B0
:100F2000041C644A02EB800242F8041C624A02EB91
:100F3000800242F8041C614A02EB400020F8021CC7
:100F4000418070472DE9F0439BB01F468C46DDE998
:100F500023350021DDF888800646259C12911391E7
:100F60001491159116911791189138461991B8F16D
:100F7000000F14BFA3F10A07471C052F40F2CC80D5
:100F80004FFA80F909F1010189B28B4298BF002123
:100F9000B8F1000F6ED03CF81180CDF8488032F8DF
:100FA00011101391A9EB530109B2002901DA194478
:100FB00009B23CF81180CDF8508032F8111015912B
:100FC000F9B2CDE900310DF1100813460146CDF814
:100FD00008806246304600F004FA16902A88039290
:100FE0002F492088069009684B8AB1F81AC0C3EBD4
:100FF0000313B3FBFCF317934B8AB1F81AC0C3EB8E
:101000000313B3FBFCF318934B8A498B03EB830365
:101010005B00B3FBF1F11991DDF85CC0002E4FF0DD
:1010200000014DD0129B059A5A43049B03EB2242C8
:10103000139BD31A44BF139B9B1A634568D2149B1E
:10104000059ADDF860C05A43049B03EB2242159BCE
:10105000D31A44BF159B9B1A634559D2169A199B04
:10106000821A44BF169A121A9A4251D2169880B226
:1010700006904CE0BCF80080CDF84880B2F80080C3
:1010800021F00101CDF84C803CF80180CDF8508072
:10109000515A94E7F49A00208A070020880700201C
:1010A000600700201F85EB5186070020B007002055
:1010B000B807002098070020A0070020A8070020FC
:1010C000139B05985843049B03EB2040129BC31AC3
:1010D00044BF129B1B1A63451AD2159B0598DDF875
:1010E00060C05843049B03EB2040149BC31A44BFC9
:1010F000149B1B1A63450BD21698199B101A44BFF8
:101100001698801A984203D2169880B20390012153
:1011100003982880069820801BB00846BDE8F0831D
:101120002DE9FF4F8BB09B468A460546FDF7C0F977
:1011300090F85A22BAB114204FF002080290287990
:1011400095F85940FE49022818BF032815D0012AF6
:101150001CBFFC4886681AD095F8F400FA4A0027AC
:10116000022840D11DE03C210291407C02282CBF86
:101170004FF003084FF00F08E1E708686423428A44
:10118000408B5A43B2FBF0F000FB00F6E4E708683E
:10119000428A408BC2EB0212B2FBF0F000FB00F679
:1011A000DAE7101900F8017CE848204400F8017CD7
:1011B0004772E748204400F8017C4772E54800EB9D
:1011C000440020F8027C4782E34885F8DC70204424
:1011D00000F8017C4772E148204400F8017CE048B7
:1011E000204400F8017CDF4802EB040900EB041303
:1011F00019F8010CDDF834C003EB400222F810CCE2
:10120000A2F890B095F8F420032A46D1C01D00F052
:1012100007008DF8207003EB40008DF8247030F843
:10122000102C0D9BB0F890009A1AABEB00030868E5
:10123000018B5143028A91FBF2F10791418B408A65
:10124000594391FBF0FB08AB224601200799FFF7B9
:10125000CBF8059009AB224659460220FFF7C4F8A7
:1012600003909DF820100798CDE900012146012048
:10127000029B059AFFF7EDF89DF82400DDE90232A4
:10128000CDE900B021460220FFF7E3F8B048059908
:10129000204400F8011C0399417219F8010C012245
:1012A000401CC0B209F8010C082808D309F8017CD9
:1012B0009AF8DC00002808BF8AF8DC2002E09AF8DF
:1012C000DC0018B195F85800022809D085F8DC70C8
:1012D000A148204400F8017C47720FB0BDE8F08FB0
:1012E000A04B0021084603EB041C0CEB4003401C00
:1012F00033F8103C80B219440828F6D34FEAD10ADB
:1013000000210846E9460CEB400333F8103CA3EB00
:101310000A035B4349F82030401C80B21944082876
:10132000F1D34FEAD109904B0021084603EB041C8E
:101330000CEB4003401C33F8103C80B219440828E1
:10134000F6D34FEAD10A00210846EB460CEB4003E6
:1013500033F8103CA3EB0A035B434BF82030401CEE
:1013600080B219440828F1D3C80803234E4528BF8A
:10137000864208D37548204410F8011C08299CBFF8
:10138000407A082811D9754885F8DC30204400F8E7
:10139000017C7348204400F8012C95F8DC000328F8
:1013A00004BF0FB0BDE8F08F92E76C48204410F8FE
:1013B000011CC8293CBF491C00F8011C6849214494
:1013C00011F8011C012908D110F8010C40459EBFFD
:1013D00085F8DC300FB0BDE8F08F022085F8DC0026
:1013E00076E72DE9F04FAFB00FFA81F9DDE9388CDF
:1013F0000124CA466946002848D032F81A002B90CA
:10140000BCF1010011D441F8204001EB800632F814
:101410001A503565AAF101050FFA85FABAF1000FE5
:10142000B8BFA8F1010A401EEDD500242546484664
:10143000BCF101020FD433F8107051F82260401E45
:101440007E43341900B245EBE6750028B8BFA8F119
:101450000100521EEFD500263746BCF101005DD4D5
:1014600001EB800233F819A0126DA9F1010902FB0A
:101470000AF296190FFA89F947EBE277B9F1000FF2
:10148000B8BFA8F10109401EEAD547E033F81A00B9
:101490002B90BCF1010011D441F8204001EB8006F3
:1014A00033F81A503565AAF101050FFA85FABAF139
:1014B000000FB8BFA8F1010A401EEDD50024254653
:1014C0004846BCF101030FD432F8107051F8236084
:1014D000401E7E43341900B245EBE6750028B8BFC4
:1014E000A8F101005B1EEFD500263746BCF10100D4
:1014F00014D401EB800332F819A01B6DA9F1010986
:1015000003FB0AF39E190FFA89F947EBE377B9F168
:10151000000FB8BFA8F10109401EEAD54FF000083E
:101520004046CDF8A080BCF1000F24DD51F820200A
:10153000289B524312EB080843EBE27216E00000CE
:10154000600700208407002048A1002066A1002039
:1015500052A100207AA10020A2A10020B6A1002063
:10156000A89B002008A00020A8A0002000F10100F6
:1015700028928445DADC0022964610462992BCF176
:10158000000F11DD01EB800351F820201B6DDDF809
:10159000A4905A434FEAE27A12EB0E0E4AEB09038B
:1015A000401C29938445EDDC4FF00009CA464846AB
:1015B000BCF1000F0DDD01EB800251F82030126DFF
:1015C00000F101005A4312EB09094AEBE27A844523
:1015D000F1DC002003460246BCF1000F0CDD694639
:1015E00001EB8001096D49434FEAE17B8A184BEB1F
:1015F0000303401C8445F2DC1046A8FB002C28990C
:10160000CDE92C0301FB00C0AEFB09CB29992E913B
:1016100008FB030301FB09B10EFB0A10B2EB0C013E
:1016200063EB0000CDE92901084333D0DDE92C024A
:10163000A0FB0413AEFB06CB02FB04322E9B00FB87
:10164000052203FB06B30EFB0733B1EB0C0062EB84
:101650000301DDE9293206F03BF93A990860A8FB5D
:101660000602289901FB0621A9FB04230AFB043387
:1016700008FB071109FB0533801A61EB030109041C
:10168000DDE9293241EA1041000406F021F93A99D6
:10169000486004E03A99002008603A9948603A9816
:1016A000D0E900122B98504311EB204048BF002096
:1016B0002FB0BDE8F08F70B5ADF5166D0E4605463E
:1016C000FCF7F6FE0446FCF707FF4FF41661684688
:1016D00006F0C3F96A463146284606F0AFF80246DE
:1016E000E0736946284603F07BFE20740DF5166D05
:1016F00070BD0000F84A0020411C1154C8B20528F2
:10170000FAD37047F54910B50020C1F88400C1F83C
:101710008800A1F88C0081F88E00C1F89A00C1F809
:101720009E00A1F8A20081F8A400C1F88F00C1F8C2
:101730009300A1F8970081F899000860486008813B
:101740008872C1F80B00C1F80F00A1F813004875AA
:1017500002F06EF9E04A0020411C1154C8B205287D
:10176000FAD310BDDC49084410F8011C21F08001B7
:1017700000F8011C70470020D74A0146535C13F063
:10178000800F04D0491CC9B20529F7D37047535CB8
:1017900003F00F0043F080035354704770B50D46BB
:1017A0000446FCF783FE00231A46A05CA95C88422D
:1017B00001D0012303E0501CC2B20A2AF5D3184617
:1017C00070BD2DE9F0418AB0002000900190029098
:1017D000039004900590069007900890FCF768FE2F
:1017E0000446FCF779FE0546FCF76CFE0746FCF75D
:1017F0007FFE0646FCF75AFE0346B4F90200B0F538
:10180000FA7F79DC94F85802012802D1607C002824
:1018100072D1A07A032818BF05286DD094F85E0213
:10182000012804BF0AB0BDE8F0810021207C4FF000
:10183000010C002888BF0DF1FF3811D9C1EB411010
:1018400007EBC00090F8F320022A12BF032A90F899
:10185000590000F808C0481CC1B2207C8842EDD86D
:10186000297C0020002988BF0DF10B0411D9C0EBA1
:10187000401106EBC10191F8F320022A12BF032A9E
:1018800091F8591001F804C0401C297CC0B2814273
:10189000EDD8002006A933F92020002AC8BF01F89E
:1018A00000C0401CC0B20A28F5D3687C002804BFE1
:1018B0000AB0BDE8F08193F8280003AC6D46F8B19A
:1018C000FCF7F4FD00231846215C2A5C914204D108
:1018D000401CC0B20A28F7D303B306AC6D46FCF730
:1018E000E5FD00231846215C2A5C914204D1401C8E
:1018F000C0B20A28F7D38BB10AB00120BDE8F0814D
:10190000FCF7D4FD00231846215C2A5C9142F3D1F8
:10191000401CC0B20A28F7D3002BEDD10AB000203A
:10192000BDE8F0812DE9F0410026FCF7CBFD07462C
:10193000FCF7BEFD0446FCF7B9FD0546B4F902000C
:10194000B0F5BE7F06DD0221A172B0F5E17FC4BF14
:101950000120607394F85E0201281FBF94F85702BB
:10196000012894F85A02012809D0FCF743FE30B947
:10197000FCF76CFE18B994F85802012802D1FFF761
:1019800020FF06460020411E25F8201005EB8002AE
:10199000401CC0B251800A28F6D3012E20D1207CF1
:1019A000002100281CD9C1EB411007EBC00090F8C2
:1019B000F320022A18BF032A0DD190F85930C288AB
:1019C00005EB830323F8042C028990F8590005EBFA
:1019D000800020F8022C481CC1B2207C8842E2D84A
:1019E00094F8580268B900223D49002E08BF4A7099
:1019F00007D04878401CC0B24870052884BF4A70A0
:101A0000002685F828603046BDE8F0812DE9F05FBA
:101A100034480025006890F85260FCF775FDFCF72B
:101A200047FD0446FCF74EFD8146B4F902004FEA3B
:101A30006008207C002898BFBDE8F09F2A4B012752
:101A40004FF0000CC5EB451009EBC00292F85900AD
:101A5000401EC1B292F8F300022802D0032845D0FC
:101A600026E003EB410080F801C092F8E000012875
:101A70001CD0B2F90200B0F5C87F17DC94F814A0AE
:101A8000BAF1010F03D1B4F902A050450ED1B4F957
:101A900002A0504505D1B2F818A0B4F804B0DA4558
:101AA00001D0404502DD03F8117030E003F8116009
:101AB00013F81100B0B303EB410013F811B090F824
:101AC00001A0DA4523D380F801C003F811C082F8E1
:101AD000E0C082F8E1701EE065A20020C0A10020F5
:101AE000E0070020600700206FA2002013F811001B
:101AF000C0B1B4F90200B0F5C87FDCDA03EB4100F5
:101B000090F801A00AF1010A80F801A0D3E782F859
:101B1000E07082F8E1C0681CC5B2207CA84291D870
:101B2000BDE8F09FFFE782F8E0C0F2E770B5FCF790
:101B3000BFFC0646FCF7C6FC0546307C00240028A6
:101B400012D9C4EB441005EBC00090F8E310012952
:101B500005D190F85900002818BF01F057FF601C0C
:101B6000C4B2307CA042ECD8002070BD70B5FCF748
:101B70009FFC0446FCF7A6FC227C0021002A84BFBF
:101B800002234FF0030C13D9C1EB411200EBC20248
:101B900092F8E350012D01BF92F8F350022D82F824
:101BA000F3C082F85830491C227CC9B28A42EBD873
:101BB000002070BD2DE9F041FCF77AFC867AC57AE9
:101BC000FCF7DCFCFCF7E0FC01F032FFFCF770FCFA
:101BD0000746FCF777FC8046387C0024002812D9A1
:101BE000C4EB441008EBC00090F8E310012905D1C4
:101BF00090F85900002818BF01F008FF601CC4B21B
:101C0000387CA042ECD8FCF753FC0446FCF75AFCA5
